:1000000087C60000B6C60000B4C60000B2C6000035
:10001000B0C60000AEC60000ACC60000AAC6000014
:10002000A8C60000A6C60000A4C60000A2C6000024
:10003000A0C600000C94BD829CC600009AC60000B9
:1000400098C600000C94698094C6000092C6000017
:1000500090C600008EC600008CC600000C94957EF1
:1000600088C600000C94B57B0C948B7B82C6000084
:1000700080C600007EC600007CC600007AC6000074
:100080000C943C8076C6000074C6000072C6000066
:100090000C94617B0C94377B6CC600000C946983D4
:1000A00068C6000066C600000C940F8062C600009F
:1000B00060C600005EC600005CC600000C94E27FD3
:1000C00058C6000056C6000054C600000C940D7BB4
:1000D0000C94E37A4EC600000C94B97A0C948F7A93
:1000E00048C600004E414E494E495459494E46CDEE
:1000F000CCCC3D0AD7233C17B7D13877CC2B3295DF
:1001000095E6241FB14F0A000020410000C84200BC
:10011000401C4620BCBE4CCA1B0E5AAEC59D740086
:10012000407A10F35A00A0724E18090010A5D4E8C6
:100130000000E87648170000E40B54020000CA9A59
:100140003B000000E1F505000080969800000040AB
:10015000420F000000A086010000001027000000F0
:1001600000E803000000006400000000000A000036
:100170000000000100000000002C76D888DC674FEA
:100180000823DFC1DFAE59E1B1B796E5E3E453C61A
:100190003AE651997696E8E6C28426EB898C9B6212
:1001A000ED407C6FFCEFBC9C9F40F2BAA56FA5F4BC
:1001B00090055A2AF75C936B6CF9676DC11BFCE0E4
:1001C000E40D47FEF520E6B500D0ED902E03009437
:1001D0003577050080841E080000204E0A000000CC
:1001E000C80C333333330F986E12831141EF8D21D6
:1001F00014893BE65516CFFEE6DB18D1844B381B3D
:10020000F77C1D901DA4BBE424203284725E228101
:1002100000C9F124ECA1E53D27485454502F312E5C
:10022000302034303020426164205265717565732E
:10023000740D0A5365727665723A2057656264756B
:10024000696E6F2F312E370D0A436F6E74656E74B1
:100250002D547970653A20746578742F68746D6CCC
:100260000D0A0D0A3C68313E45504943204641493C
:100270004C3C2F68313E00485454502F312E3020D2
:10028000323030204F4B0D0A5365727665723A203A
:100290005765626475696E6F2F312E370D0A4163A1
:1002A000636573732D436F6E74726F6C2D416C6C4C
:1002B0006F772D4F726967696E3A202A0D0A436F76
:1002C0006E74656E742D547970653A2000436F6EBC
:1002D0006E656374696F6E3A20636C6F73650D0AA7
:1002E000436F6E74656E742D547970653A20617039
:1002F000706C69636174696F6E2F782D7777772DD5
:10030000666F726D2D75726C656E636F64656400E7
:10031000506F7374206661696C65640055706C6F12
:100320006164204661696C65643A2000234E6F2049
:1003300073656E736F7220666F722074656D7020C6
:10034000262068756D696469747921004E6F2053A9
:10035000656E736F72210020666F722074656D7018
:1003600020262068756D69646974792100235365BE
:100370006E736F72204572726F72200053656E73D8
:100380006F72204572726F7221002357726F6E6711
:100390002073656E736F7220666F722074656D7066
:1003A00020262068756D6964697479210057726F21
:1003B0006E672053656E736F7221004320483D00C5
:1003C000543D0020202020202020202020202020FC
:1003D000202020002020202020202020202020203D
:1003E000202020002020202020202020202020202D
:1003F00020202000495020616464726573733A20A4
:1004000000496E76616C696420534D207374657089
:10041000732070657220616E676C653D00534D20DE
:1004200073746570732070657220616E676C653DD2
:10043000003C68343E436F70797269676874284382
:1004400029323031382D3230323020456455484B16
:10045000204861732043656E7472652E3C2F6834AA
:100460003E3C2F626F64793E3C2F68746D6C3E0099
:100470003C703E4C616D7020616E64204F74686505
:100480007220537461747573EFBC9A3C2F703E00F8
:100490003C68313E43616E6E6F74206765742073F3
:1004A000656E736F722072656164696E6773213C5B
:1004B0002F68313E003C21646F6374797065206859
:1004C000746D6C3E3C68746D6C3E3C686561643E66
:1004D0003C6D65746120636861727365743D22755B
:1004E00074662D38223E3C7469746C653E4F6E6CA8
:1004F000696E65206578706572696D656E74206FD0
:100500006E20706F6C6172697A6174696F6E206FB2
:1005100066206C696768743C2F7469746C653E3C36
:100520002F686561643E3C626F64793E3C68313E91
:100530004F6E6C696E65206578706572696D656E69
:1005400074206F6E20706F6C6172697A6174696F6C
:100550006E206F66206C696768743C2F68313E00BE
:10056000506172616D657465727320726573657434
:1005700020646F6E652100736573757365722F73E8
:100580006D6C69676874706F2F73312F00616E67CF
:100590006C6520646972656374696F6E3A2000430C
:1005A000757272656E7420534D2069732023005359
:1005B0004D3A5461626C6520737465707320706588
:1005C0007220616E676C653D00534D3A506F6C61EF
:1005D000726F696420737465707320706572206136
:1005E0006E676C653D00234448543D00236E65747E
:1005F0003D424C4500236E65743D576946690023B2
:100600006E65743D42540023667470207573657284
:100610006E616D653A003A0023486F73742073650C
:100620007276657220495020616E6420506F72743A
:100630003A002352656C617920646576696365735D
:100640003A002352656C617920737461747573206C
:100650006C6162656C733A20002352656C6179208D
:100660007374617465733A002352656C617920700C
:10067000696E733A00234E6F2E206F662072656C90
:100680006179733D0046696E64696E6720576946FB
:1006900069204950004E45543D426C7565746F6F3A
:1006A0007468204C45004E45543D426C7565746F2E
:1006B0006F7468004E45543D5769466900696E7015
:1006C00075742044535463616C6962726174653A55
:1006D000005344206F70656E206661696C004E6542
:1006E00077206461746120636F6C6C656374696FFB
:1006F0006E20737461727465640043757272656E06
:10070000742073657474696E67733A0053797374F7
:10071000656D2072657365742061742000234453F5
:1007200020546865726D6F6D657465722063616CCD
:100730006962726174656420666F72202300496E7D
:1007400076616C696420616E676C6520666F7220EB
:10075000002073746570732070657220616E676C21
:10076000653D002073746570732070657220616E42
:10077000676C653D00576946692049503A004C6FE7
:1007800067676572204E616D653A20005265626F41
:100790006F74696E672E2E2E005365727665722017
:1007A000506F727420757064617465640053504FAB
:1007B00052543D0049502075706461746564005363
:1007C00049503D0074696D6520696E74657276618B
:1007D0006C3D002377656273657276657220626591
:1007E00067696E73005461626C65205365742030D4
:1007F00000235475726E7461626C652053657420B9
:100800003000506F6C6172697A6572205365742094
:10081000300023506F6C6172697A65722053657481
:1008200020300053797374656D2072657374617242
:1008300074656421002053797374656D207265734B
:10084000746172746564210023436F6D6D616E6421
:10085000400054657374204C616D70732F46616E57
:1008600073004448435020537563636573730044B9
:10087000484350204641494C4544007765627365C2
:1008800072766572202E2E2E006572726F72206F46
:1008900070656E696E672066696C653A20004C6110
:1008A0006D70204F74686572002354696D65202057
:1008B000202020204461746520202020205365637F
:1008C0006F6E647320506F6C61726F696420546145
:1008D000626C652054286F43292048282529202050
:1008E00000646F6E652100696E69742E20646F6EFE
:1008F000652E00534420696E69742E206661696C10
:1009000065642100696E69742E206661696C656496
:10091000210057656C636F6D6520746F20456455C9
:10092000484B00496E697469616C697A696E672029
:10093000534420636172642E2E2E0075706C6F61BB
:100940006420627920465450206661696C65642198
:100950000075706C6F616420627920465450204F9E
:100960004B21007C3C3E5E2B3D3F2F5B5D3B2C2AA8
:10097000225C00005EBCE2613FDD83C29C7E20A35E
:10098000FD1F419DC3217FFCA2401E5F01E3BD3ED0
:100990006082DC237D9FC1421CFEA0E1BF5D03801D
:1009A000DE3C62BEE0025CDF81633D7C22C09E1DB6
:1009B00043A1FF4618FAA427799BC584DA3866E577
:1009C000BB5907DB856739BAE406581947A5FB7898
:1009D00026C49A653BD987045AB8E6A7F91B45C6D1
:1009E000987A24F8A6441A99C7257B3A6486D85B7E
:1009F00005E7B98CD2306EEDB3510F4E10F2AC2F2B
:100A00007193CD114FADF3702ECC92D38D6F31B267
:100A1000EC0E50AFF1134DCE90722C6D33D18F0C84
:100A200052B0EE326C8ED0530DEFB1F0AE4C12914D
:100A3000CF2D73CA947628ABF517490856B4EA69E6
:100A400037D58B5709EBB536688AD495CB2977F41F
:100A5000AA4816E9B7550B88D6346A2B7597C94A48
:100A600014F6A8742AC896154BA9F7B6E80A54D705
:100A7000896B3500002100240027002A002D00305A
:100A800000330001010000040107010A01000022F7
:100A900000250028002B002E003100340002010048
:100AA00000050108010B0100002000230026002999
:100AB000002C002F00320000010000030106010994
:100AC0000105050505070508080808020202020AD3
:100AD0000A080804040404010101010101010103E1
:100AE00003030303030303040707070C0C0C0C0C9C
:100AF0000C0C0C0202020206060606060606060B8F
:100B00000B0B0B0B0B0B0B01021020200808102005
:100B10004010204080020102010804020101020489
:100B20000810204080804020100804020180040248
:100B3000018040201008040201080402010102049F
:100B40000810204080010204081020408000000AA4
:100B50000B02090C0D0E0807030401000000000041
:100B60000000000000000000000000000000000085
:100B70000000000000000000001211100000000042
:100B80000000000000000000000000000000000065
:100B90000000002346616E73207377697463686593
:100BA00064206F6E20666F72200023486561746553
:100BB00072207377697463686564206F6E20666F56
:100BC000722000000001000100101002000100016D
:100BD00000B0000000160000002800000010000017
:100BE00000200000000100010000000000000000E3
:100BF00000000000000000000000000000000000F5
:100C00000000000000FF000000FFFF0000FFFF00E9
:100C100000FFFF0000CFBF0000C7BF0000C3BF0040
:100C200000C1BF0000C0BF000000000000C0BF0046
:100C300000C1BF0000C3BF0000C7BF0000CFBF009E
:100C400000FFFF0000FFFF000000000000000000A8
:100C50000000000000000000000000000000000094
:100C60000000000000000000000000000000000084
:100C70000000000000000000000000000000000074
:100C8000000000000000000000557365722D6167D0
:100C9000656E743A202A0D0A446973616C6C6F7733
:100CA0003A202F0D0A004E6574776F726B206D61CC
:100CB000696E7461696E65642061742000417070B2
:100CC000656E64206D6561732E200053696E676CDC
:100CD00065206D6561732E200053617665206D651A
:100CE000617375726520746F3A00202020202020E7
:100CF0002020202020202020202000202020202014
:100D00002020202020202020202020001D9D5398DE
:100D100011241FBECFEFD1E2DEBFCDBF00E00CBF7C
:100D20001AE0A0E0B2E0EEE9FDE601E00BBF02C090
:100D300007900D92A637B107D9F728E1A6E7BAE0E8
:100D400001C01D92AC35B207E1F716E0C7E8D6E066
:100D500000E006C021970109802FFE010E944DB1DD
:100D6000C638D10780E00807A9F70E942CA10C948F
:100D7000BEB646C9CF93DF93EC01898D9A8D892B3E
:100D800041F0E881F9810284F385E02DCE011995C7
:100D9000F4CFDF91CF910895CF93DF931F92CDB71A
:100DA000DEB76983DC01ED91FC910280F381E02DD7
:100DB00041E050E0BE016F5F7F4F19950F90DF91CA
:100DC000CF910895FC01818D928D0895FC01848955
:100DD0009589089523E334E0FC0131832083FB01EE
:100DE0004089518962897389FC01428353836483FA
:100DF00075830895DC01ED91FC91048CF58DE02D57
:100E00001994CF93DF931F92CDB7DEB76983DC01CE
:100E1000ED91FC910280F381E02D41E050E0BE01B4
:100E20006F5F7F4F19950F90DF91CF910895FC016F
:100E30009485FB018485981303C081E0943009F404
:100E400080E0089521E0FC018485843009F420E0ED
:100E5000822F08950895CF93DF931F92CDB7DEB709
:100E60006983DC01ED91FC910280F381E02D41E08A
:100E700050E0BE016F5F7F4F19950F90DF91CF91CA
:100E80000895DC01ED91FC91068CF78DE02D19950C
:100E900091E089270895862F089581E08627089597
:100EA0000A96D9CF90E080E0089590E0982F8827A7
:100EB00044E050E0845F9B4F0C941595DF92EF92D5
:100EC000FF920F931F93CF93DF93D82E02E11CE084
:100ED000E801EE24E394F12C22968091AE029091E9
:100EE000AF028E159F059CF061E088810E94F57C21
:100EF00060910D0C88810E94DF7B64EF71E080E0DF
:100F000090E00E94267D8FEFE81AF80AE5CFDD20F9
:100F100009F45EC0C2E1DCE0EE24E394F12C2296F9
:100F20008091AE029091AF02E816F9062CF560911F
:100F30000F0C88810E94DF7B68EE73E080E090E018
:100F40000E94267DAFEFEA1AFA0A60910F0C8A819F
:100F50000E94DF7B68EE73E080E090E00E94267DD7
:100F600060910D0C88810E94DF7B68EE73E080E069
:100F700090E00E94267DD3CF68EE73E080E090E0A1
:100F80000E94267D93E4E92E92E0F92EC1E0D0E0A4
:100F9000B2E0EB0EF11C0E5F1F4F8091AE029091FC
:100FA000AF028C179D07A4F0D701ED91FC91EE0FD5
:100FB000FF1FE35FF34F6081F80180810E94DF7BB8
:100FC00068EC70E080E090E00E94267D2196E0CF02
:100FD000DF91CF911F910F91FF90EF90DF900895D7
:100FE0009F92AF92BF92CF92DF92EF92FF920F93B8
:100FF0001F93CF93DF935C017B018B01D0E0C0E0B6
:10100000F80191908F016501CC0EDD1EC6010E9492
:10101000A6AF981621F0692DC6010E94AEAF2196A9
:10102000CA32F1E0DF0761F7C701DF91CF911F916D
:101030000F91FF90EF90DF90CF90BF90AF909F9077
:10104000089581E08093E1028091E202882341F0DB
:1010500088E08093BA1360E08FEA93E10C94968065
:101060000895CF93DF93EC01FB01248135810E9429
:101070001779CE01DF91CF9108958091E202882304
:10108000F9F08091E1028823D9F081E00E94D480B8
:101090008BE39FE10197F1F760E080E00E94E3803D
:1010A00064EE73E08FEA93E10E945F7A61E080E092
:1010B0000E94E38064ED73E08FEA93E10C945F7A21
:1010C00008958F929F92AF92BF92CF92DF92EF924C
:1010D000FF920F931F93CF93DF938C01862F0B30DA
:1010E000110509F092C090913813992309F0F894F2
:1010F00062E10E94597DEC0180913813882309F048
:101100007894209701F180E090ECA9E7B4EC80930B
:101110002B1390932C13A0932D13B0932E13809325
:101120002F1390933013A0933113B0933213CE3F0B
:101130008FEFD80709F49DC0CF3FDC0709F4F5C154
:10114000CCEFDFEF24C1C0913313E09034136E2D48
:1011500070E090E080E00E9493AE2DEC3CEC4CEC13
:101160005DE30E94F2AE4B015C016C2F70E090E0F9
:1011700080E00E9493AE9B01AC01C501B4010E94C6
:1011800029B060932B1370932C1380932D1390939D
:101190002E13D0913513F09036136D2F6F7770E0CA
:1011A00090E080E00E9493AE4B015C016F2D70E0F7
:1011B00090E080E00E9493AE2DEC3CEC4CEC5DE3C3
:1011C0000E94F2AE9B01AC01C501B4010E9429B09E
:1011D000D7FD19C060932F13709330138093311390
:1011E00090933213CE0DCD0FCF0D81E090E0209182
:1011F0003713C21302C090E080E0892B09F487C046
:10120000CFEFDFEF92C19058E5CFCFEFDFEF0631A0
:10121000110509F0BCC090913813992309F0F89496
:1012200061E00E94597DEC0180913813882309F018
:101230007894209709F180E090ECA9E7B4EC8093D2
:101240002B1390932C13A0932D13B0932E138093F4
:101250002F1390933013A0933113B0933213CF3FD9
:10126000DC0709F462C1209709F451C0229609F005
:1012700067CFCEEFDFEF8BC0C0913413D091331323
:10128000609133137091341376276727762790E0A7
:1012900080E00E9491AE2DEC3CEC4CEC5DE30E94B2
:1012A000F2AE60932B1370932C1380932D139093B5
:1012B0002E13E0903613F09035136F2D6F77762F45
:1012C0006E2D90E080E00E9491AE2DEC3CEC4CEC59
:1012D0005DE30E94F2AEF7FC18C060932F13709389
:1012E000301380933113909332138C2F8D0F8E0D0A
:1012F0008F0DC1E0D0E090913713891302C0D0E088
:10130000C0E0D195C195D109AACF9058E6CFC09041
:101310002B13D0902C13E0902D13F0902E1320E07F
:1013200030E048EC52E4C701B6010E9426B1D0E09B
:10133000C0E0181614F4CBEFDFEF20E030E0A90195
:10134000C701B6010E948DAE87FF02C0CAEFDFEF72
:10135000C0902F13D0903013E0903113F0903213DF
:1013600020E030E048EC52ECC701B6010E948DAE9F
:1013700087FF02C0C9EFDFEF20E030E040EF52E42A
:10138000C701B6010E9426B118160CF4C9C00C3072
:10139000110509F0CAC081E08093CE0C8CE58093E2
:1013A000D00C1092CF0C1092D10C90E080E00E94F3
:1013B0004D7481E00E94F07365E08CE50E947D75BC
:1013C0001092940C8093930CC82FD0E0209709F4CE
:1013D000AAC0C530D1050CF4B8C006E31BE086E412
:1013E0009FE00E949772F80180870F5F1F4FC8012E
:1013F00086539B408C179D0794F3C0913E0B009140
:101400003F0B602F70E090E080E00E9493AE2DECE7
:101410003CEC4CEC5DE30E94F2AE6B017C016C2F66
:1014200070E090E080E00E9493AE9B01AC01C701A8
:10143000B6010E9429B06B017C01C092360BD0929C
:10144000370BE092380BF092390BD091400B109192
:10145000410B6D2F6F7770E090E080E00E9493AEBB
:101460004B015C01612F70E090E080E00E9493AE40
:101470002DEC3CEC4CEC5DE30E94F2AE9B01AC0128
:10148000C501B4010E9429B0D7FD5DC060933A0B3D
:1014900070933B0B80933C0B90933D0BC00FCD0F93
:1014A000C10F8091420BC813ABCE20E030E048EC76
:1014B00052E4C701B6010E9426B1D0E0C0E0181680
:1014C00014F4CBEFDFEF20E030E040EA50E4C70156
:1014D000B6010E948DAE87FF02C0CAEFDFEFC09059
:1014E0003A0BD0903B0BE0903C0BF0903D0B20E092
:1014F00030E040EF51ECC701B6010E948DAE87FF8E
:1015000002C0C9EFDFEF20E030E040EF52E4C70156
:10151000B6010E9426B1181644F4C8EFDFEF05C0EB
:10152000C8EFDFEF34CFCEEFDFEFCE01DF91CF9109
:101530001F910F91FF90EF90DF90CF90BF90AF90F1
:101540009F908F9008959058A1CFCDEFDFEFEDCF12
:101550002C9A08952C9808958EBD00000DB407FEB6
:10156000FDCF8EB508959B0190E00496982F8827B3
:10157000642F820F931F0C94A295CF93DF93C82FF3
:10158000D62F472F60E170E0EEDF4D2F61E170E074
:101590008C2FDF91CF91E7CFCF93DF93C82FD0E08F
:1015A0002496DC2FCC27C60FD71FD4DF8FE0D4DFE3
:1015B0008D2FD2DF8C2FD0DF80E0CEDFC82FC8DFA9
:1015C0008C2FDF91CF9108951F93CF93DF93182F26
:1015D00066E270E0E1DFC82F67E270E0812FDCDFB8
:1015E0009C2FDF91CF911F9108951F93CF93DF938D
:1015F000182F60E270E0D0DFC82F61E270E0812F29
:10160000CBDF9C2FDF91CF911F91089544E050E0F4
:10161000BC018FE090E00C94159508958CBD9DBDA4
:101620000895EF92FF920F931F93CF93C82F7B01E2
:1016300080E590E0F3DF68E270E08C2FADDF082FEB
:1016400069E270E08C2FA8DF282F302FB90121E04C
:1016500030E0A7018C2F0E94027681E090E0CF91CC
:101660001F910F91FF90EF900895CF93DF931F92FA
:10167000CDB7DEB7FC01218D328D8FEF9FEF232B8D
:1016800039F0BE016F5F7F4F808DCBDF898190E0A5
:101690000F90DF91CF9108950F931F93CF93DF9316
:1016A0001F92CDB7DEB78C01DC01ED91FC91008477
:1016B000F185E02D1995892B71F0BE016F5F7F4F89
:1016C000F8018485AEDF898190E00F90DF91CF91A2
:1016D0001F910F9108958FEF9FEFF7CFFF920F9318
:1016E0001F93CF93DF93F82E80E590E097DF10E013
:1016F00000E08F2D69DFEC01892B19F08F2D64DF5D
:101700008C01C017D107A9F7CE01DF91CF911F91AE
:101710000F91FF900895FC018485843009F0DECF9D
:1017200090E080E00895AF92BF92CF92DF92EF9267
:10173000FF921F93CF93DF93182F6B017A0180E5FF
:1017400090E06CDFB12CA12C812F3EDFEC01892BC6
:1017500019F0812F39DF5C01CA15DB05A9F7209745
:10176000E1F463E070E0812F17DF843159F08823C2
:1017700049F0C1E0D0E08C3111F4D0E0C0E0D19567
:10178000C195D109CE01DF91CF911F91FF90EF90CC
:10179000DF90CF90BF90AF900895EC16FD060CF44B
:1017A000E7011C161D0674F768E270E0812FF4DE75
:1017B000E82E69E270E0812FEFDE282F3E2D7901BF
:1017C0009E01A601B701812F0E940276EC0EFD1E3C
:1017D0004F2D68E270E0812FC6DE4E2D69E270E089
:1017E000812FC1DE60E470E0812F0E949574CACF22
:1017F000CF93DF93FC01218D328D2115310529F422
:101800008FEF9FEFDF91CF910895EC01808D42170C
:10181000530708F0A90187DF181619068CF7298DE0
:101820003A8D281B390B3A8F298FECCF0F931F93DA
:10183000CF93DF931F92CDB7DEB7FC01218D328DA0
:10184000232B41F48FEF9FEF0F90DF91CF911F91EA
:101850000F9108958C0141E050E0BE016F5F7F4F12
:10186000FC01808D60DF1816190664F7F801818D80
:10187000928D0197928F818F898190E0E5CF0F93B0
:101880001F93CF93DF9300D000D01F921F92CDB74C
:10189000DEB78C01DC01ED91FC910680F781E02D33
:1018A0001995F801808D1ADF18161906ACF548E075
:1018B00050E0BE016F5F7F4FD80158968C9133DFA7
:1018C00018161906F4F4D801509684E0FE013196FA
:1018D00001900D928A95E1F78D8190E0982F8827ED
:1018E0002E81820F911DF801958B848B8F81282F7B
:1018F00030E0322F22278885820F932F911D928FFF
:10190000818F28960FB6F894DEBF0FBECDBFDF9152
:10191000CF911F910F91089590E080E0F2CFFC01EC
:10192000848501CFCF93DF931F92CDB7DEB741E01F
:1019300050E0BE016F5F7F4FFC018485F4DE181616
:10194000190634F4898190E00F90DF91CF910895CA
:101950008FEF9FEFF9CFCF93C82F80E590E05EDE49
:1019600060E170E08C2F0E9495744FEF62E070E0B0
:101970008C2FCF91F8CDFF920F931F93CF93DF93CE
:10198000C82FD62F8A01F22EE6DF80E590E046DEF2
:101990004D2F4F2970E060E08C2FE5DD011511051A
:1019A000B1F0412F64E070E08C2FDDDD402F65E069
:1019B00070E08C2FD8DD61E070E08C2F0E94957470
:1019C00081E0DF91CF911F910F91FF9008950091D9
:1019D0005F0C1091600C0F5F1F4F1093600C009311
:1019E0005F0CDFCFBF92CF92DF92EF92FF920F9307
:1019F0001F93CF93DF9300D000D0CDB7DEB7FC01AB
:101A0000208D243009F059C06A017B018C01B12C72
:101A100063E070E08B2DC0DD811147C0F801B08E0E
:101A2000F801808D843009F448C096E0EDEEF2E0D4
:101A3000DE01119601900D929A95E1F7F7019381DD
:101A40009F779C8394819D8395819E83B7016E5F70
:101A50007F4F2BDAB601F801808D8FDDF801808D84
:101A600090E0982F882746E050E0BE016F5F7F4FDF
:101A70008A5F9B4F0E941595F801128E118E20E807
:101A8000A60162E0808D77DF81E026960FB6F8949C
:101A9000DEBF0FBECDBFDF91CF911F910F91FF90A1
:101AA000EF90DF90CF90BF900895883109F4B6CFC2
:101AB000B394F4E0BF12ACCFB3CF80E0E6CFCF93C6
:101AC000DF93EC01888D843059F045DFE88DF0E03C
:101AD000EE0FFF1FE159F34F1182108284E0888FCF
:101AE000DF91CF910895CF93C82F80E590E096DDE8
:101AF00063E070E08C2FCF914FCDEF92FF921F9358
:101B0000CF93DF93FC01208D243039F080E0DF910A
:101B1000CF911F91FF90EF9008957B01EC0110E0B1
:101B2000812FE1DF81110EC0188F888D843071F311
:101B3000FD86EC861A8E198E20E0A70162E01BDF7D
:101B400081E0E5CF883181F31F5F143049F7EDCF95
:101B5000FC018485843009F0C6CF80E00895CF93DE
:101B6000DF93FC0124852430D1F0EC01F1DF8431D6
:101B700089F0882379F0883169F021E08C3159F4BB
:101B8000E881F9810084F185E02DCE01199521E0ED
:101B9000892B09F420E0822FDF91CF91089580E016
:101BA000FBCFAF92BF92CF92DF92FF920F931F9322
:101BB000CF93DF938C015B01EA01FC01C688D788D3
:101BC000F08C80E590E02ADD8F2D0E94A5748C17A3
:101BD0009D0720F48F2D0E94A574EC019E01A501A4
:101BE000B6018F2D0E944495F801868997898C0F44
:101BF0009D1F978B868BCE01DF91CF911F910F9107
:101C0000FF90DF90CF90BF90AF900895CF93FC01ED
:101C1000C08D80E590E002DD60E270E08C2F0E94D4
:101C2000957462E070E08C2FB7DC84FD13C062E035
:101C300070E08C2FB1DC83FF09C048E162E070E006
:101C40008C2F91DC90E080E0CF91089580E590E0CA
:101C5000E5DCE7CF40E162E070E08C2F84DC81E0DE
:101C600090E0F2CFFF920F931F93CF93DF93EB019E
:101C7000FC01178A168A2A81211109C02B812111A2
:101C800006C02C81211103C02D812223C9F04115EA
:101C90005105B1F08A01FC01F08C80E590E0BEDCDA
:101CA000BE016E5F7F4F8F2D00D9B8018F2D65DC8F
:101CB00081E090E0DF91CF911F910F91FF90089507
:101CC00090E080E0F7CF4F925F926F927F928F9279
:101CD0009F92AF92BF92CF92DF92EF92FF920F93BB
:101CE0001F93CF93DF93CDB7DEB763970FB6F8940A
:101CF000DEBF0FBECDBF7C016B013A01FB0120E0CE
:101D000090E080E06AE03191332309F45EC040ED59
:101D1000430F4A3008F04AC0689FA001699F500DE8
:101D20001124CA01C097830F911D37FD9A958F3FEB
:101D3000910549F340F3F701428153816481758134
:101D40008091A70F9091A80FA091A90FB091AA0F11
:101D5000481759076A077B0709F416C28701085F0D
:101D60001F4F0E94E07D6F7077277C5FC801C5DE42
:101D7000813009F00EC283E394E09A838983F701EE
:101D800082819381A481B5818B839C83AD83BE8343
:101D900045E350E0BE016F5F7F4FC80163DF892BD1
:101DA000A1F5D12CC12CC8018ADE17C03E3209F042
:101DB000C2CF233009F4BFCFD301A20FB11D1296B9
:101DC0008C932F5F90E080E09ECF233009F0B3CF5B
:101DD000F3018583CC24C394D12CC60163960FB63E
:101DE000F894DEBF0FBECDBFDF91CF911F910F9151
:101DF000FF90EF90DF90CF90BF90AF909F908F902B
:101E00007F906F905F904F9008950E94E07DF70162
:101E1000778366837627672776277A83698342E00C
:101E200050E0BE016F5F7F4FC801BBDE81E090E0F4
:101E30009E878D8742E050E0BE01635F7F4FC801FF
:101E4000B0DE80E091E09E878D8742E050E0BE01E9
:101E5000635F7F4FC801A5DE1E861D8642E050E00D
:101E6000BE01635F7F4FC8019CDE42E050E0BE01CF
:101E7000635F7F4FC80195DE42E050E0BE01635FC3
:101E80007F4FC8018EDE5601F60180818823F1F074
:101E90006501F60181912F01882311F08E32A1F4A2
:101EA00046018A189B081814190464F48F8641E0CF
:101EB00050E0BE01615F7F4FC80173DEA401B50130
:101EC000C8016FDE5201E0CF6201E3CF1F8641E01F
:101ED00050E0BE01615F7F4FC80163DEC12CDD248D
:101EE000D394DE86CD8642E050E0BE01635F7F4F33
:101EF000C80157DEDE86CD8642E050E0BE01635F5A
:101F00007F4FC8014EDEC80181DE892B09F449CF1D
:101F1000F3E0AF2EB12C230122E0420E511C5DC034
:101F2000F7014281538164817581808D918DA28DED
:101F3000B38D481759076A077B0709F01BC1848DC9
:101F4000958DC59709F016C181A192A10C970CF44B
:101F500016C14CE050E0BE016F5F7F4FC80148DC06
:101F60008B819C819827892798279A8B898B298137
:101F70003A81322723273227F701468157814217BA
:101F80005307D1F497FF18C08F709270892B09F016
:101F900041C06F807884762467247624D12CC12CAC
:101FA0006114710409F04CC0C8010E94BA066AEFBE
:101FB000C62EDD24DA9407C0C8010E94BA06ECEFF1
:101FC000CE2EDD24DA9481E0A81AB10809F4EBCE14
:101FD000FFEFCF16DF0609F0E6CE0E94E07D3B0161
:101FE0004C01C8014CDC181619060CF499CF0E945C
:101FF000E07D661977098809990969387341810577
:10200000910508F0B3C062E370E080E090E00E94C8
:10201000267DE7CFC8010E94BA067BEFC72EDD24DC
:10202000DA94D1CF8D85811113C0C801FFDBC801BF
:10203000FDDBC801FBDBC801F9DBFFEFCF1ADF0ACC
:102040008D819E81982789279827C816D90698F4EC
:1020500041E050E0BE01635F7F4FC801C9DB8D8561
:10206000882301F38D859FEF980F9D878823D1F2F8
:10207000C801DCDBF7CF912C812C41E050E0BE01A0
:102080006D5E7F4FC801B4DB8B89982F907C59F42B
:10209000882379F08B899FEF980F9B8B882331F0F1
:1020A000C801C4DBF7CFC801C1DB1B8A8B89811152
:1020B000E4CF42E050E0BE01615F7F4FC80198DB92
:1020C00042E050E0BE01635F7F4FC80191DBC80171
:1020D000ADDBC801ABDBC801A9DBC801A7DB42E06F
:1020E00050E0BE016F5E7F4FC80182DB8F8598890B
:1020F00081159140E1F4CD84DE84DC24CD24DC2400
:1021000081E0C816D10499F489899A89811594408F
:1021100041F0C8010E94BA0657EFC52EDD24DA94BB
:1021200052CF44E050E0B201C80162DB4CCFD12C69
:10213000C12C89899A89982789279827C816D90692
:1021400030F4C80173DBFFEFCF1ADF0AF2CF2FEFB5
:10215000821A920A6814790409F08FCFC8010E948C
:10216000BA0646EFC42EDD24DA942DCFCC24CA94CF
:10217000DC2C29CF2EEFC22EDD24DA9424CF9DEF64
:10218000C92EDD24DA941FCF8EEFC82EDD24DA9419
:1021900024CED12CC12C21CECF92DF92EF92FF9290
:1021A0000F931F93CF93DF93CDB7DEB7AF970FB6E3
:1021B000F894DEBF0FBECDBF7C016A0103E314E0DB
:1021C0001A8309831C861B8688EE93E0A0E0B0E0AA
:1021D0008D879E87AF87B88B87EC93E09A87898736
:1021E000188F0F8B198E1A8E1B8E1C8E84E089A37C
:1021F0001BA70AA71CA61DA61EA61FA680919F0F9F
:102200009091A00FA091A10FB091A20F8EA39FA3B8
:10221000A8A7B9A78B839C83AD83BE8318861F8232
:10222000AE01465D5F4FCE0101964DDD81309105D7
:10223000B1F4D701ED91FC910488F589E02D1DA33F
:102240000CA38CA59DA5AEA5BFA58EA39FA3A8A7F3
:10225000B9A7A601BE016C5D7F4FC7011995AF9666
:102260000FB6F894DEBF0FBECDBFDF91CF911F91A7
:102270000F91FF90EF90DF90CF900895CF92DF9273
:10228000EF92FF920F931F93CF93DF93CDB7DEB7FB
:10229000AF970FB6F894DEBF0FBECDBF7C016A01C9
:1022A00003E314E01A8309831C861B8688EE93E0FF
:1022B000A0E0B0E08D879E87AF87B88B87EC93E076
:1022C0009A878987188F0F8B198E1A8E1B8E1C8EFA
:1022D00084E089A31BA70AA71CA61DA61EA61FA6ED
:1022E00080919F0F9091A00FA091A10FB091A20F8C
:1022F0008EA39FA3A8A7B9A78B839C83AD83BE831E
:1023000018861F82AE01465D5F4FCE010196DBDC71
:1023100081309105B1F4D701ED91FC910684F785E8
:10232000E02D1DA30CA38CA59DA5AEA5BFA58EA3D6
:102330009FA3A8A7B9A7A601BE016C5D7F4FC701E7
:102340001995AF960FB6F894DEBF0FBECDBFDF91E3
:10235000CF911F910F91FF90EF90DF90CF90089554
:102360007F928F929F92AF92BF92CF92DF92EF9225
:10237000FF920F931F93CF93DF93CDB7DEB7A6974E
:102380000FB6F894DEBF0FBECDBF8C01762E942E13
:10239000852E20E2A22ECE0101967C01DC01EA2DE1
:1023A0001D92EA95E9F76801F3E4CF0ED11C83E3AF
:1023B00094E09AA389A38FEF8BA38CA38DA38EA304
:1023C00043E450E0BE016F5D7F4FC6014BDC0196D8
:1023D00009F4B8C081E089838A8386E0B82EBB8285
:1023E0001C82D80114966D917D918D919C911797C7
:1023F0000E9455B16D837E838F83988789869A86E4
:1024000080E890E09C878B874CE150E0B701C601E3
:10241000C8DBFE0137968AE1DF011D928A95E9F754
:102420004801B8E08B0E911CF401D70101900D9288
:10243000BA94E1F740E150E0B701C601B2DBF70121
:102440001192AA94E9F796E0A92EB12C40E250E04F
:10245000B701C601A6DBF1E0AF1AB108B9F783E610
:10246000898392E89A8393E59B838C8385E38D83AC
:1024700081E08E837F829DE3988797E099878A87A2
:1024800086E0F401DE011B9601900D928A95E1F73A
:102490008CE0898B8A8B65E374E0CE0143960E94C1
:1024A000B8B3D8011B966C91CE0149960E9448762C
:1024B000F8016485CE014B960E944876D8011D969E
:1024C0006C91CE014D960E9448764EE150E0B701E6
:1024D000C60167DBB3E07B121DC082E3898384E021
:1024E0008A83F80196859B8397859C8390899D8339
:1024F00091899E8396E39F838887828D8987838DC8
:102500008A87848D8B87858D8C874CE050E0B7015E
:10251000C60147DB87E3898386E08A8391E09B835A
:1025200093E09C838D838FE08E838AE38F838BE39C
:1025300088878FEF898749E050E0B701C60131DB1A
:10254000C60164DBA6960FB6F894DEBF0FBECDBF02
:10255000DF91CF911F910F91FF90EF90DF90CF907F
:10256000BF90AF909F908F907F9008958F929F9291
:10257000AF92BF92CF92DF92EF92FF920F931F9391
:10258000CF93DF93CDB7DEB72D970FB6F894DEBFAC
:102590000FBECDBF7C0110E000E038EE832E33E0AB
:1025A000932EA12CB12C4FEEC42E43E0D42E1C82CE
:1025B0001B828D829E82AF82B886DA82C9820D87A5
:1025C000CE010196C5DA811133C0F70144815581EE
:1025D00020E061E0802FCFD980E590E01FD863E054
:1025E00070E0802F0E94CC0A833129F462E070E011
:1025F000802F0E949574F70184819581000F111F2F
:10260000F801E159F34F918380832D960FB6F8942A
:10261000DEBF0FBECDBFDF91CF911F910F91FF9015
:10262000EF90DF90CF90BF90AF909F908F900895E4
:102630000F5F1F4F0430110509F0B9CFE6CFCF92DD
:10264000DF92EF92FF921F93CF93DF93FC011485EB
:10265000143079F1EC0180E590E00E940E0B68E007
:1026600070E0812F0E9495740E94E07D6B017C01D7
:10267000CE016EDA882399F061E070E080E090E0AE
:102680000E94267D0E94E07D6C197D098E099F09BC
:10269000683E73408105910558F38C855CD9EC85C3
:1026A000F0E0EE0FFF1FE159F34F1182108284E03A
:1026B0008C87DF91CF911F91FF90EF90DF90CF90AB
:1026C00008954F925F926F927F928F929F92AF92F6
:1026D000BF92CF92DF92EF92FF921F93CF93DF933F
:1026E000CDB7DEB72D970FB6F894DEBF0FBECDBFC6
:1026F0007C019FE6A92E9CE0B92E10E0D12CC12CC4
:1027000028EE422E23E0522E612C712C3FEE832EB8
:1027100033E0932E1C821B824D825E826F8278860C
:102720009A8289821D87D5012D913D915D01F70126
:10273000848195812817390799F4CE01019608DA2A
:10274000843189F1CE01019603DA8C3149F4CE014E
:1027500001960E948B0B892B19F4CE0101966FDF35
:102760001F5F1430B9F6CD2841F4D701ED91FC91EB
:102770000084F185E02DC70119952D960FB6F894C8
:10278000DEBF0FBECDBFDF91CF911F91FF90EF90C5
:10279000DF90CF90BF90AF909F908F907F906F9081
:1027A0005F904F900895CC24C394D12CD9CF8F92B1
:1027B0009F92AF92BF92CF92DF92EF92FF920F93D0
:1027C0001F93CF936C015B017A01FC01C485C43077
:1027D000A1F481E090E0F60193838283F12CE12C57
:1027E000C701CF911F910F91FF90EF90DF90CF9095
:1027F000BF90AF909F908F9008958A0141305840CC
:1028000010F000E018E080E590E00E940E0B8C2FA5
:102810000E94A5744C0163E070E08C2F0E94CC0AEA
:10282000873111F08C3121F58016910660F380E537
:1028300090E00E940E0B9801A50170E060E08C2FE3
:102840000E94449560E270E08C2F0E94957462E0D3
:1028500070E08C2F0E94CC0A84FD12C063E070E00F
:102860008C2F0E94CC0A811106C08C2F74D8B1CF56
:1028700010E000E0DCCF80E590E00E940E0BE7CF97
:1028800040E162E070E08C2F0E94B30A012B09F056
:10289000A7CF9FCF3F924F925F926F927F928F927E
:1028A0009F92AF92BF92CF92DF92EF92FF920F93DF
:1028B0001F93CF93DF93CDB7DEB72D970FB6F89464
:1028C000DEBF0FBECDBF6C015B014A01FADE8FE6B1
:1028D000E82E8CE0F82E312C10E000E098EE492E26
:1028E00093E0592E612C712C1C821B824D825E82DA
:1028F0006F8278868FEE93E09A8389833D86F70115
:10290000219131917F01F601848195812817390742
:1029100061F4CE0101961CD9873139F4A401B501C7
:10292000CE01019644DF080F191F3394F4E03F12E3
:10293000DBCFC8012D960FB6F894DEBF0FBECDBF1A
:10294000DF91CF911F910F91FF90EF90DF90CF908B
:10295000BF90AF909F908F907F906F905F904F90BF
:102960003F9008950A9623CFCF92DF92FF920F9364
:102970001F93CF93DF93FC012485243051F090E026
:1029800080E0DF91CF911F910F91FF90DF90CF906A
:1029900008956A01EB018C01F12C8F2DA4D88111CF
:1029A00029C0F801F486F8018485843041F3209130
:1029B0009202309193022F5F3F4F21F130939302A7
:1029C00020939202409192025091930220E061E0A4
:1029D0000E94BB0C8A818F3FC1F48B818F3F01F530
:1029E0008C818F3FE9F48D818F3FD1F484E0F80131
:1029F0008487C5CF8B7F8831A1F2F394F4E0FF1276
:102A0000CCCFD1CF20E030ECD9CF811109C08B8160
:102A1000811106C08C81811103C08D81882331F31F
:102A2000C114D10419F3F801F48480E590E00E9408
:102A30000E0BBE016E5F7F4F8F2D0E945507B601B2
:102A40008F2D0E94BD0A64E070E08F2D0E94957466
:102A5000C8017ED8873159F061E070E080E090E0F5
:102A60000E94267DC80174D88111F2CFBFCF81E0CA
:102A700090E087CFCF93CFB7F89480915E0C81110F
:102A800027C0E6EFFAE08491ECE3FBE09491E82FB5
:102A9000F0E0EE0FFF1FED58F54FA591B491EC91CA
:102AA000E92321F461E085E30E94DF7B61E085E3B7
:102AB0000E94F57C8CB580618CBD8CB580648CBD2A
:102AC00061E084E30E94F57C61E083E30E94F57C91
:102AD00080915E0C8F5F80935E0CCFBFCF91089585
:102AE000EF92FF920F931F93CF93DF938C01E091AE
:102AF0003E108E2F90E0FC01EE0FFF1FE80FF91F34
:102B0000E555F04F808186FD06C069E370E08EE3F5
:102B100090E10E945B7F64E670E080E090E00E94BC
:102B2000267D80919A0290919B0297FF04C010929B
:102B30009B0210929A02C0919A02D0919B02BE0110
:102B40008EE390E10E94DF7E64E670E080E090E03A
:102B50000E94267D80919A0290919B020817190786
:102B6000C4F07E01C53BD1051CF054EBE52EF12CE1
:102B7000C017D10714F5B7018EE390E10E94DF7E04
:102B80006EE170E080E090E00E94267DE7012196F2
:102B9000E8CF0C171D078CF4D7FF02C0D0E0C0E0CF
:102BA000BE018EE390E10E94DF7E6EE170E080E086
:102BB00090E00E94267D2197ECCFCE01C53BD10548
:102BC00014F084EB90E0E0913E102E2F30E0F901FC
:102BD000EE0FFF1FE20FF31FE555F04F20812F7B13
:102BE000208397FF02C090E080E0DF91CF911F919A
:102BF0000F91FF90EF900895EF92FF920F931F9324
:102C0000CF93DF938C01E0913B108E2F90E0FC017D
:102C1000EE0FFF1FE80FF91FE555F04F808186FD8D
:102C200006C069E370E08BE390E10E945B7F64E69D
:102C300070E080E090E00E94267D80919802909163
:102C4000990297FF04C01092990210929802C091C5
:102C50009802D0919902BE018BE390E10E94DF7E41
:102C600064E670E080E090E00E94267D809198020A
:102C70009091990208171907C4F07E01C53BD10550
:102C80001CF054EBE52EF12CC017D10714F5B70159
:102C90008BE390E10E94DF7E6DE270E080E090E0E7
:102CA0000E94267DE7012A96E8CF0C171D078CF4B9
:102CB000D7FF02C0D0E0C0E0BE018BE390E10E94EC
:102CC000DF7E6DE270E080E090E00E94267D2A9732
:102CD000ECCFCE01C53BD10514F084EB90E0E09140
:102CE0003B102E2F30E0F901EE0FFF1FE20FF31F14
:102CF000E555F04F20812F7B208397FF02C090E0A5
:102D000080E0DF91CF911F910F91FF90EF90089598
:102D10004F925F926F927F928F929F92AF92BF92EB
:102D2000CF92DF92EF92FF920F931F93CF93DF9397
:102D3000EC018090AE029090AF02E5E4F2E081E019
:102D400090E0512C412C8816990654F02191319134
:102D50002130310519F42FEF421A520A0196F3CFB0
:102D60001C161D060CF04AC08C169D060CF446C0BD
:102D70004E018E01000F111F7E01EE0CFF1CEE0CA8
:102D8000FF1C8C169D060CF4D9C0C701895C9D4FB1
:102D90006C01FC0180819181A281B3819701215B4B
:102DA0003D4F5901181619061A061B0654F50E94C4
:102DB0005F81F5012081318142815381621B730B58
:102DC000840B950BF60120813181428153812617B6
:102DD00037074807590758F410821182128213826C
:102DE0000E945F81F50160837183828393832196C2
:102DF0000E5F1F4FF4E0EF0EF11CC3CFC1E0D0E037
:102E0000B8CF980128553D4F3901F9018081918152
:102E100098012D5B3D4F6901F901208131818217B5
:102E20009307F1F0F3E04F16510414F00097C1F44A
:102E3000880F991FFC01E35FF34F6081F801EE5E9C
:102E4000F34F80810E94DF7BF30180819181F60145
:102E5000918380836CE271E080E090E00E94267DA7
:102E6000F50180819181A281B381181619061A0695
:102E70001B060CF0BCCF0E945F81F50120813181DF
:102E800042815381621B730B840B950BF701E4564F
:102E9000FD4F208131814281538126173707480732
:102EA000590708F0A4CFF501108211821282138213
:102EB0009801275B3D4F5901F90180819181F6010D
:102EC000208131818217930709F491CF6091AE027E
:102ED0007091AF02E5E4F2E041E050E030E020E044
:102EE000641775074CF0A191B191119711F42F5F00
:102EF0003F4F4F5F5F4FF4CF233031051CF00097F9
:102F000009F075CF880F991FFC01E35FF34F6081D3
:102F1000F801EE5EF34F80810E94DF7BF501808136
:102F20009181F60191838083F301918380836CE228
:102F300071E080E090E00E94267D59CFDF91CF9133
:102F40001F910F91FF90EF90DF90CF90BF90AF90C7
:102F50009F908F907F906F905F904F900895CF9348
:102F6000DF93FC0124813581232B69F0EC01BC0146
:102F700089EA9EE00E944D7ABE0182ED9CE0DF91DD
:102F8000CF910C944D7ADF91CF910895CF93DF9339
:102F9000FC0124813581232B69F0EC01BC0189EA15
:102FA0009EE00E943F7ABE0182ED9CE0DF91CF91CE
:102FB0000C943F7ADF91CF910895CF93DF93FB017B
:102FC00022813381DC0113963C932E931297448126
:102FD00055816681778114964D935D936D937C93B3
:102FE0001797408551856285738518964D935D933B
:102FF0006D937C931B971C96EF012C969C01275E8A
:103000003F4F49914D93A217B307D9F7218D328DC8
:10301000FC01328F218FDF91CF910895CF92DF9203
:10302000EF92FF920F931F93CF93DF93CDB7DEB74D
:10303000A0970FB6F894DEBF0FBECDBF7C018B0109
:1030400050E040E06C018AE0C80ED11CCA01019634
:10305000F8012491E1E0F0E0EC0FFD1FE40FF51F13
:103060002083222381F08032910549F440E250E030
:10307000BE016F5F7F4FC6019ADB90E080E00F5F7B
:103080001F4FAC01E3CF029730F0BE016F5F7F4F5F
:10309000C7010A968CDBA0960FB6F894DEBF0FBE70
:1030A000CDBFDF91CF911F910F91FF90EF90DF90F7
:1030B000CF900895EF92FF920F931F93CF93DF93DA
:1030C000EC018B017A0167E772E0A8DFB801CE015D
:1030D0000E94387A8E01065F1F4F42E050E06FE198
:1030E0007AE0C80164DBE114F10421F0B701CE01FC
:1030F0000E94387A42E050E06FE17AE0C801DF9147
:10310000CF911F910F91FF90EF9051CB69E172E049
:1031100085CFCF92DF92EF92FF920F931F93CF93C1
:10312000DF9300D000D0CDB7DEB77C01FB018481F6
:1031300095818A01081B190B101611069CF0C70116
:103140000E94EB78C70126960FB6F894DEBF0FBE3B
:10315000CDBFDF91CF911F910F91FF90EF90DF9046
:10316000CF900895CE0101960E94FB78CC24C394A1
:10317000D12C6BEF75E0CE0101960E94F377FFEF43
:10318000CF1ADF0A0C151D05A4F7BE016F5F7F4F34
:10319000C7010E94EB78CE0101960E947378D2CFCE
:1031A000EF92FF920F931F93CF93DF9300D000D045
:1031B000CDB7DEB78C017B0167E079E00E9403792F
:1031C0008AE0E816F1042CF461EB76E0C8010E9475
:1031D000F377B701CE0101960E946376BE016F5F5F
:1031E0007F4FC8010E94FC77CE0101960E94737840
:1031F000C80126960FB6F894DEBF0FBECDBFDF9193
:10320000CF911F910F91FF90EF9008951F93CF934F
:10321000DF93CDB7DEB72C970FB6F894DEBF0FBEA5
:10322000CDBF2B893C893093AF022093AE02FE01C3
:103230007396A2E1BCE090E080E03296281739074F
:1032400034F0408151814D935D930196F6CF8B8D83
:103250009C8D90930E0C80930D0C8D8D9E8D909374
:10326000100C80930F0CAC968FADAC97BE016559D6
:103270007F4F8F3209F0B2C1CE0107960E940379C9
:103280006CE374E0CE0101960E940379BE01695F90
:103290007F4FCE0101960E949A77BC0187E593E1AA
:1032A0000E942578CE0101960E947378CE01079680
:1032B0000E94737867E573E1CE0101960E94FB7866
:1032C000CE0101964CDECE0101960E94737862E534
:1032D00074E0CE0101960E940379BE016F5F7F4FBB
:1032E00087E593E10E944B77182FCE0101960E944B
:1032F000737840915B1350915C13112309F475C1ED
:10330000BA016250710987E593E10E943A77682F0C
:10331000CE0101960E94D378BE016F5F7F4F89E393
:1033200093E10E943A78CE0101960E94737861E39E
:1033300072E1CE0107960E94037964E574E0CE0144
:1033400001960E940379BE01695F7F4FCE0101960D
:103350000E949A77BC0181E593E10E942578CE0115
:1033600001960E947378CE0107960E947378239687
:103370008FAD23971F928F9322968FAD22971F9226
:103380008F9321968FAD21971F928F938FAD1F92B0
:103390008F938AE594E09F938F938CE49CE09F93B6
:1033A0008F930E94F6B3CF52DF4F88819981C15D20
:1033B000D04090937A0280937902BE016D527F4F84
:1033C000CE0101960E940379BE016F5F7F4F8BE4AF
:1033D00093E10E943A78CE0101960E947378BE0173
:1033E00062527F4FCE0101960E940379BE016F5F4A
:1033F0007F4F85E493E10E943A78CE0101960E94C6
:1034000073784091491350914A134250510965E431
:1034100073E1CE0101960E943108CE0101960E940F
:10342000D2766C596093B902CE0101960E947378EE
:10343000CD5EDE4F688179818A819B81C351D14005
:103440000E9493AE0FB6F894DEBF0FBECDBF9B01B6
:10345000AC010E942AB1882389F08CE390E0A0E0BF
:10346000B0E0CD5EDE4F88839983AA83BB83C351CE
:10347000D140CE5EDE4F1882C251D140CE5EDE4FCB
:103480008881C251D140882399F0CD5EDE4F88817A
:103490009981AA81BB81C351D1408093B00290939E
:1034A000B102A093B202B093B30281E08093970C73
:1034B000C95EDE4F688179818A819B81C751D14085
:1034C0009B01AC010E942AB1882361F080E090E06A
:1034D000A0E7B2E4C95EDE4F88839983AA83BB83E9
:1034E000C751D140C55EDE4F68817981CB51D14053
:1034F000072E000C880B990B0E9493AE9B01AC0128
:103500000E942AB1882341F082E090E0C55EDE4F40
:1035100099838883CB51D140C55CDE4F6881798126
:10352000CB53D140072E000C880B990B0E9493AE11
:103530009B01AC010E942AB1882341F080E590E014
:10354000C55CDE4F99838883CB53D140C55CDE4F89
:1035500088819981CB53D140909336028093350274
:1035600088E2FE01E651FF4FA0E2BCE001900D921F
:103570008A95E1F7CF5CDE4F88819981AA81BB8172
:10358000C153D1408093200290932102A093220244
:10359000B0932302CB5CDE4F88819981AA81BB81E5
:1035A000C553D14080931C0290931D02A0931E022C
:1035B000B0931F02C75CDE4F88819981C953D14007
:1035C00090935C0280935B022C960FB6F894DEBF5A
:1035D0000FBECDBFDF91CF911F910895CE01079609
:1035E0000E94037961E474E04DCE4150510967E5D2
:1035F00073E1CE0101960E943108BE016F5F7F4FDB
:1036000089E393E10E943A78CE0101960E94737893
:1036100067E573E1CE0101960E94FB7862E574E0F4
:10362000CE0101960E948677BC0187E593E10E9456
:10363000257879CE0F931F93CF93DF9300D000D0DE
:10364000CDB7DEB72091110C2223A9F08C0169E9D6
:1036500077E0CE0101960E940379B801CE01019670
:103660000E949A77BC0189EA9EE00E944D7ACE01C1
:1036700001960E94737826960FB6F894DEBF0FBEAF
:10368000CDBFDF91CF911F910F910895DF92EF92FF
:10369000FF920F931F93CF93DF93CDB7DEB762975F
:1036A0000FB6F894DEBF0FBECDBF8C011092430B56
:1036B00067E079E0CE010D960E940379FF24F39430
:1036C00089EA9EE00E94C4702091430B18161906E7
:1036D00074F521112CC089EA9EE00E94A2708A3004
:1036E00009F07DC089899A89892B09F480C0F092FC
:1036F000430B66E674E0CE0101960E940379BE0199
:10370000635F7F4FCE0101960E949A77BC01CE0184
:1037100007960E94FB78CE0107968CDFCE010796B4
:103720000E947378CE0101960E94737860C0F12CDC
:10373000E12CDD24D394222309F460C089899A897D
:10374000019709F045C06BEC74E0CE0107960E942A
:103750000379BE01695F7F4FCE010D960E946B77A2
:10376000F12C811115C066E774E0CE0101960E942C
:103770000379BE016F5F7F4FCE010D960E946B777C
:10378000FF24F3948111F12CCE0101960E947378ED
:10379000CE0107960E947378FF20A1F050E040E030
:1037A000BE01635F7F4FCE0101960E943108BE01CA
:1037B0006F5F7F4F8EEE90E10E943A78CE010196C6
:1037C0000E94737864E170E080E090E00E94267DC2
:1037D000BE01635F7F4FC8010E94EB7894C08D30BB
:1037E00009F480CF682FCE010D960E94D4776AE04D
:1037F00070E080E090E00E94267D62CF82ED9CE048
:103800000E94C4701816190614F582ED9CE00E94FF
:10381000A2708A30A9F08D3099F09091430B9111EC
:103820000FC0682FCE010D960E94D4778FEFE81A53
:10383000F80A65E070E080E090E00E94267DDECF2F
:1038400089899A89892BA9F3D092430BF2CF64E13D
:1038500070E080E090E00E94267DEF2809F43DC0F2
:1038600089899A89892BC9F18091110C882379F172
:1038700069E977E0CE0101960E940379BE016F5F8E
:103880007F4FCE010D960E946B77F82ECE010196E8
:103890000E947378F1101BC06FE674E0CE010196B0
:1038A0000E940379CE01019671DBCE0101960E9440
:1038B0007378BE01635F7F4FCE0101960E94FB7853
:1038C000CE0101964CDBCE0101960E94737864E133
:1038D00070E080E090E00E94267D89899A8920919D
:1038E000430B21112DCF009709F02ACF64E670E039
:1038F00080E090E00E94267D0E94E07D67E079E014
:10390000C8010E940379CE010D960E947378C80108
:1039100062960FB6F894DEBF0FBECDBFDF91CF9198
:103920001F910F91FF90EF90DF9008950F931F93D9
:10393000CF93DF93CDB7DEB72C970FB6F894DEBFE9
:103940000FBECDBF8C010E94B782BC01C80128DC2C
:103950000E94B182BC01CE01079622DC6FED76E0B9
:10396000CE0101960E940379BE01695F7F4FCE01AF
:1039700001960E949A77BC01C8010E94FC77CE0193
:1039800001960E947378CE0107960E9473786BEFC0
:1039900075E0C8010E94F3770E94AB82BC01CE01A2
:1039A0000196FEDBBE016F5F7F4FC8010E94FC776E
:1039B000CE0101960E94737868E774E0C8010E9406
:1039C000F3770E94A582BC01CE010196E9DBBE011E
:1039D0006F5F7F4FC8010E94FC77CE0101960E9465
:1039E000737868E774E0C8010E94F3770E949D82B3
:1039F000BC01CE010196D4DBBE016F5F7F4FC801D1
:103A00000E94FC77CE0101960E947378C8012C9623
:103A10000FB6F894DEBF0FBECDBFDF91CF911F91DF
:103A20000F9108950F931F93CF93DF93CDB7DEB718
:103A30002C970FB6F894DEBF0FBECDBF8C010E944D
:103A4000B782BC01C801ACDB0E94B182BC01CE01CF
:103A50000796A6DB6FED76E0CE0101960E94037912
:103A6000BE01695F7F4FCE0101960E949A77BC012B
:103A7000C8010E94FC77CE0101960E947378CE01A6
:103A800007960E9473780E945F810E94A4816091D2
:103A9000610C70E0CE01079683DB6FED76E0CE011E
:103AA00001960E940379BE01695F7F4FCE010196A6
:103AB0000E949A77BC01C8010E94FC77CE01019652
:103AC0000E947378CE0107960E9473786BEF75E0C1
:103AD000C8010E94F3770E94AB82BC01CE0101961F
:103AE0005FDBBE016F5F7F4FC8010E94FC77CE0194
:103AF00001960E94737868E774E0C8010E94F3772A
:103B00000E94A582BC01CE0101964ADBBE016F5F17
:103B10007F4FC8010E94FC77CE0101960E94737806
:103B200068E774E0C8010E94F3770E949D82BC019F
:103B3000CE01019635DBBE016F5F7F4FC8010E9449
:103B4000FC77CE0101960E947378C8012C960FB6BF
:103B5000F894DEBF0FBECDBFDF91CF911F910F91C3
:103B600008956115710519F00A960C945B7990E03F
:103B700080E008952F923F924F925F926F927F92D2
:103B80008F929F92AF92BF92DF92EF92FF920F932C
:103B90001F93CF93DF93CDB7DEB7E4970FB6F894BA
:103BA000DEBF0FBECDBF7C014A015B0119010E943F
:103BB000E07D2B013C0187010D5B1F4FC8010E9476
:103BC0003F0C181619069CF00E94E07D64197509D7
:103BD0008609970986169706A806B90608F490C1C3
:103BE00062E370E080E090E00E94267DE7CF42E251
:103BF00050E0BE016F5F7F4FC8010E94F80B8981C2
:103C0000823009F078C1F80184899589833491055F
:103C100009F071C16D817E818F8198850E9455B1B7
:103C20002B013C01F101408251826282738246E0A5
:103C300050E0B701685F7F4FCE014D960E947DB383
:103C4000892B99F4F70180819181A281B381481673
:103C500059066A067B0648F084819581A681B78162
:103C600084159505A605B705E8F4C8010E94BA06B3
:103C7000D12C8D2DE4960FB6F894DEBF0FBECDBFCC
:103C8000DF91CF911F910F91FF90EF90DF90BF9048
:103C9000AF909F908F907F906F905F904F903F90EC
:103CA0002F90089589899A89AB89BC8986879787DF
:103CB000A08BB18B8EECA82EB12CC8010E94160CE3
:103CC000F1E0AF1AB108C9F7D12CC70182969AA7C3
:103CD00089A7F701B696FCA7EBA708969EA78DA724
:103CE0003C974F01899698AB8FA73897FAABE9AB11
:103CF0001701F6E12F0E311CC5979CAB8BABF80179
:103D0000818D928D181619060CF0F6C0C8010E941C
:103D1000160C8333910509F4D4C0A4F581309105C4
:103D200009F474C074F4892B51F3C8010E94160C75
:103D3000B82EBA94FFEFBF1611F3C8010E94160CFB
:103D4000F8CF8330910509F46CC0069771F7C8016C
:103D50000E94160CA82E44E050E06BA97CA9C80173
:103D60000E94F80B712C612CEA2DE450FF0B5F01CF
:103D70006A147B0424F6C8010E94160CFFEF6F1A28
:103D80007F0AF6CF8A33910509F46FC074F5853345
:103D90009105A1F1C69749F6C8010E94160CB82EEC
:103DA000F701828D811109C0838D811106C0848D38
:103DB000811103C0858D8823A1F0EFA5F8A940806B
:103DC000518062807380B401CE0183960E94837A11
:103DD0008DA19EA1AFA1B8A584159505A605B7052F
:103DE000D9F544E050E0B40118C08B33910509F4D3
:103DF00052C08F3F910509F482CF97CFC8010E942E
:103E0000160CC8010E94160CD82E79CFC8010E944A
:103E1000160C44E050E069A97AA9C8010E94F80B89
:103E20006ECFC8010E94160CA82E44E050E0B101EC
:103E3000C8010E94F80B712C612C8A2D8450990BBB
:103E40005C016A147B040CF05ACFC8010E94160C66
:103E50009FEF691A790AF5CFBA94FFEFBF1609F4FC
:103E60004ECFC8010E94160CF7CFC8010E94160C55
:103E700044E050E06BA57CA5C8010E94F80BF70157
:103E800066A177A180A591A50E9455B166A377A3ED
:103E900080A791A734CFC8010E94160C44E050E0DF
:103EA0006DA57EA5C8010E94F80BF70162A573A558
:103EB00084A595A50E9455B162A773A784A795A76D
:103EC0001ECFC8010E94160C44E050E069A57AA5F7
:103ED000C8010E94F80BF70162A173A184A195A10A
:103EE0000E9455B162A373A384A395A366A777A785
:103EF00080AB91AB04CFD12CC8010E94BA06B9CED9
:103F0000DD24DA94B6CE2F923F924F925F926F9259
:103F10007F928F929F92AF92BF92CF92DF92EF9259
:103F2000FF920F931F93CF93DF9300D000D0CDB7B4
:103F3000DEB78C010E9491A82FEC37E040E050E002
:103F40000E94EDAFDC01CB010196A11DB11DF8016E
:103F500084839583A683B78380839183A283B3836D
:103F60005801F3E4AF0EB11CC5010E945F0D64E47B
:103F700070E0C5010E947D0D882309F443C10E94B1
:103F8000E07D2B013C01480182E4880E911C48EE43
:103F9000C42E43E0D42EE12CF12C52E0252E1E82BB
:103FA0001D82D4018C918330B1F1811166C0F8017A
:103FB00084819581A681B7810196A11DB11D84835D
:103FC0009583A683B7830E94E07D641975098609ED
:103FD0009709A70196010E94CBAFA90161E0C80132
:103FE0000E94B01181E0D4018C938D819E81019754
:103FF000C1F20E94E07D6419750986099709D8010C
:10400000D6962D913D914D915C91D9972617370702
:104010004807590720F6C5010E945F0DF801848109
:104020009581A681B7810196A11DB11D84839583D9
:10403000A683B7830E94E07DF801FE9660837183BA
:10404000828393838D819E8126960FB6F894DEBF7E
:104050000FBECDBFDF91CF911F910F91FF90EF90D9
:10406000DF90CF90BF90AF909F908F907F906F9098
:104070005F904F903F902F9008958430F1F4F801B5
:1040800084819581A681B7810196A11DB11D84838C
:104090009583A683B7830E94E07D6419750986091C
:1040A0009709A70196010E94CBAFA90163E0C8015F
:1040B0000E94B011D4012C9298CF813049F5F801BB
:1040C00042AD53AD64AD75AD9E012F5F3F4FC8014A
:1040D00051DD382EF2E08F138FC089819A81AB8138
:1040E000BC81F80184839583A683B7830E94E07D19
:1040F0006419750986099709A70196010E94CBAF3B
:10410000A90163E0C8010E94B011D4013C926DCFB7
:10411000823009F06ACFF80142AD53AD64AD75ADA0
:104120009E012F5F3F4FC80125DD382EF5E08F132C
:104130005DC0E3E0D401EC93F80182A193A1A4A1B6
:10414000B5A1892B8A2B8B2B41F484E893E0A0E066
:10415000B0E082A393A3A4A3B5A3F80186A197A17D
:10416000A0A5B1A5892B8A2B8B2B61F482A193A1E9
:10417000A4A1B5A1B695A7959795879586A397A372
:10418000A0A7B1A7F80182A593A5A4A5B5A5892BE1
:104190008A2B8B2BA9F482A193A1A4A1B5A1AC0178
:1041A000BD0123E076956795579547952A95D1F7F8
:1041B000841B950BA60BB70B82A793A7A4A7B5A743
:1041C000F80186A197A1A0A5B1A586A797A7A0AB46
:1041D000B1AB82A593A5A4A5B5A582AB93ABA4ABC7
:1041E000B5AB81E090E09E838D83FFCE96E089138E
:1041F00003C0D4011C92F9CEBFEF3B12F6CEF401FE
:104200001082F3CE1E821D821DCFEF92FF920F937C
:104210001F93CF93DF93CDB7DEB7E8970FB6F8942F
:10422000DEBF0FBECDBF67E079E0CE0187960E946A
:10423000037967E079E0CE018D960E94037982E0F0
:10424000E82EF12C2496FFAEEEAE249786E0E3EF45
:10425000F2E0DE01D39601900D928A95E1F786E0B7
:10426000FE01F396DE01AC5BBF4F01900D928A9583
:10427000E1F72C961FAE1EAE2C9701E010E02E96B3
:104280001FAF0EAF2E9788E0E9EFF2E0DE015996FE
:1042900001900D928A95E1F788E0FE017996DE01A2
:1042A000A25BBF4F01900D928A95E1F788E1E1E0B2
:1042B000F3E0DE01119601900D928A95E1F788E115
:1042C000FE013196DE01AA5ABF4F01900D928A95E8
:1042D000E1F78091190390911A03A0911B03B0910B
:1042E0001C03E2968CAF9DAFAEAFBFAFE2976AE71B
:1042F00074E0CE0187960E945A7660E0CE018796E0
:104300000E94D4774BA55CA5BE016E587F4FCE01AD
:1043100087960E94DC7567E775E0CE018D960E9456
:10432000027862EC74E089E393E10E945A7660E0DF
:10433000CE018D960E94D47749A95AA9BE0166562E
:104340007F4FCE018D960E94DC7567E079E0CE014B
:1043500087960E945A7667E079E0CE018D960E949A
:104360005A76C250DF4F19821882CE5FD0408091BA
:10437000790290917A02C050DF4F99838883C050B0
:10438000D14080E090E0A0E7B2E4CA5BDE4F8883D2
:104390009983AA83BB83C654D140C65BDE4FF982A2
:1043A000E882CA54D14080E090E0A0E2B2E4C45B6D
:1043B000DE4F88839983AA83BB83CC54D14080E0AD
:1043C00090E0A4E3B2E4C05BDE4F88839983AA83C4
:1043D000BB83C055D14084EB90E0CC5ADE4F99832B
:1043E0008883C455D14088E790E0CA5ADE4F99834C
:1043F0008883C655D1408CE291E0A0E0B0E0C85A75
:10440000DE4F88839983AA83BB83C855D140C45AA1
:10441000DE4F19830883CC55D140C25ADE4FF98252
:10442000E882CE55D14060E08BE493E10E94D477DE
:1044300060E085E493E10E94D47740914F1350915E
:104440005013BE016E5F7E4F8BE493E10E94DC75DA
:104450004091491350914A13BE01635F7E4F85E43A
:1044600093E10E94DC7588E2E0E2FCE0DE01A75EF9
:10447000BE4F01900D928A95E1F78CE390E0A0E0A9
:10448000B0E0CE5BDE4F88839983AA83BB83C2549E
:10449000D140CF5BDE4F1882C154D14084EE98E307
:1044A000AEE8B2E4C05ADE4F88839983AA83BB8307
:1044B000C056D14084EE98E3AEE8B1E4CC59DE4F6B
:1044C00088839983AA83BB83C456D140C859DE4FE1
:1044D00019830883C856D14080E590E0C659DE4F65
:1044E00099838883CA56D14084EF91E090939102DA
:1044F00080939002BE016E5B7F4F0E94F00764EFD5
:1045000071E080E090E00E94267D60E675E0CE01DB
:1045100081960E94F378CE0181960E94AF17CE015A
:1045200081960E947378CE018D960E947378CE0199
:1045300087960E947378E8960FB6F894DEBF0FBE98
:10454000CDBFDF91CF911F910F91FF90EF90089514
:104550009F92AF92BF92CF92DF92EF92FF920F9312
:104560001F93CF93DF93CDB7DEB7C859D1090FB6EC
:10457000F894DEBF0FBECDBF5C017B016A0169E527
:1045800072E1CE0189579F4F0E94037962E574E082
:104590008E010F5F1F4FC8010E940379B801CE0141
:1045A00089579F4F0E946B77982EC8010E9473789D
:1045B000911014C062E574E0C8010E940379BE0145
:1045C00069577F4FC8010E949A77BC01CE01895775
:1045D0009F4F0E942578C8010E947378B501CE01D3
:1045E00083579F4F0E94037962E874E021E0E2164E
:1045F000F10441F06DE874E032E0E316F10411F0EB
:1046000065E974E0CE0189579F4F0E94F37760E01F
:10461000CE0189579F4F0E94D477B601C8010E94EE
:10462000FB786AE0C8010E94E777BC01CE018D5695
:104630009F4F0E94FB78C8010E947378C557DF4FD7
:1046400048815981CB58D040B801CE0189579F4F3E
:104650000E94DC758091980C882399F16DE974E0D3
:10466000CE018F579F4F0E940379CE018F579F4FE6
:104670000E94C617CE018F579F4F0E947378BE01CC
:1046800069577F4FCE018F579F4F0E94FB78CE0115
:104690008F579F4F0E94C617CE018F579F4F0E9482
:1046A0007378B801CE018F579F4F0E940379CE01D6
:1046B0008F579F4F0E94C617CE018F579F4F0E9462
:1046C0007378CC56DF4F8881C459D0408F93CD5634
:1046D000DF4F8881C359D0408F93C257DF4F888105
:1046E000CE58D0408F93C357DF4F8881CD58D040EC
:1046F0008F938DEA94E09F938F9386E7E82E8AE06C
:10470000F82EFF92EF920E94F6B34091350250913D
:1047100036026CE47CE082EE91E10E943E110FB61D
:10472000F894DEBF0FBECDBF019709F07CC01F9388
:104730000F9383EB94E09F938F9308E71BE01F9305
:104740000F930E94F6B3B80182EE91E10E94267A9F
:104750008CE49CE09F938F9384EC94E09F938F93E1
:104760001F930F930E94F6B3B80182EE91E10E946D
:10477000267A6DEC72E082EE91E10E945F7A6FE141
:104780007AE082EE91E10E945B79F70101900020CE
:10479000E9F7CF0187579A409F938F938DEC94E070
:1047A0009F938F931F930F930E94F6B3B80182EEED
:1047B00091E10E94267AB70182EE91E10E94387A57
:1047C00062E370E080E090E00E94267D82EE91E15D
:1047D0000E941F130FB6F894DEBF0FBECDBF11E0CD
:1047E000CE018D569F4F0E947378CE0183579F4F05
:1047F0000E947378CE0189579F4F0E947378812F52
:10480000C856DF4F0FB6F894DEBF0FBECDBFDF91A5
:10481000CF911F910F91FF90EF90DF90CF90BF90BD
:10482000AF909F90089560E173E0CE018F579F4F46
:104830000E94F378CE018F579F4F0E94AF17CE0191
:104840008F579F4F0E9473786CE173E0CE018F57B2
:104850009F4F0E94F378CE018F579F4F0E94C6173B
:10486000CE018F579F4F0E94737866E77AE0CE01A2
:104870008F579F4F0E940379CE018F579F4F0E9401
:10488000AF17CE018F579F4F0E94737810E0A8CFCB
:10489000DF92EF92FF920F931F93CF93DF93CDB7E9
:1048A000DEB762970FB6F894DEBF0FBECDBF209182
:1048B000E202222379F12091E102222359F17A01C7
:1048C0008C016F3F7F4FA1F560E080E00E94E380A4
:1048D000D12CB8018FEA93E10E943F7A63EC73E038
:1048E0008FEA93E10E945F7AF801848160E08D0D88
:1048F0000E94E3800E94E07D60939A0C70939B0C71
:1049000080939C0C90939D0CB701FF0C880B990B26
:104910000E94267D62960FB6F894DEBF0FBECDBF13
:10492000DF91CF911F910F91FF90EF90DF9008954D
:1049300060E080E00E94E3800E94E07D28EE33E0AA
:1049400040E050E00E94CBAFCA01B90120E831E558
:1049500041E050E00E94EDAFAB01BC0120E0CE0190
:1049600001960E94A778BE016F5F7F4FCE01079628
:104970000E94FB786DE878E0CE0107960E9486776A
:10498000BC01CE010D960E94FB78CE0107960E94D5
:104990007378CE0101960E947378BE01635F7F4FEA
:1049A0008FEA93E10E943F7AD98860E08D2D0E94C2
:1049B000E380CE010D960E9473788BCF7F928F9209
:1049C0009F92AF92BF92CF92DF92EF92FF920F939E
:1049D0001F93CF93DF93CDB7DEB762970FB6F894EE
:1049E000DEBF0FBECDBF10E000E034E4C32E3BE0DD
:1049F000D32E40E3E42E53EEB52E66E0A62E7CEED9
:104A0000972EE1E3FE2EFEE48F2EA4E37A2E68EBD0
:104A100072E280E091E10E947D0DF6018E2D1192EF
:104A20008A95E9F7B092440BA092460B9092470BFF
:104A3000F092500B8092510BF092520B7092530BEC
:104A400060E072E0CE0101960E94837A4BE750E06D
:104A5000BE016F5F7F4F80E091E10E94320E40E324
:104A600050E064E47BE080E091E10E94D10D80E0C1
:104A700091E10E94060E68EE73E080E090E00E94F3
:104A8000267D80E091E10E943F0C892B31F50A30B0
:104A9000110509F05CC162EE74E0CE0101960E943E
:104AA0000379CE0101960E94AF17CE0101960E94B4
:104AB000737862960FB6F894DEBF0FBECDBFDF915C
:104AC000CF911F910F91FF90EF90DF90CF90BF900B
:104AD000AF909F908F907F90089540E350E064E402
:104AE0007BE080E091E10E94F80B60916C0B70918B
:104AF0006D0B76276727762790E080E0CB0177273C
:104B00006627C0906E0BD0906F0BDC24CD24DC2484
:104B1000F12CE12C6C297D298E299F297E508A4A0F
:104B200093480E943B810E945F816093740B709355
:104B3000750B8093760B9093770B0A30110509F46F
:104B4000AACF0E945F816093860C7093870C80933C
:104B5000880C9093890C0E945F8160938A0C7093FB
:104B60008B0C80938C0C90938D0CCE0101960E943F
:104B7000121DCE0101960E94AF17CE0101960E9430
:104B800073780E94AB82BC01CE0107960E94D018B8
:104B900068E774E0CE0107960E94F3770E94A58231
:104BA000BC01CE0101960E94D018BE016F5F7F4FFD
:104BB000CE0107960E94FC77CE0101960E94737881
:104BC00068E774E0CE0107960E94F3770E949D8209
:104BD000BC01CE0101960E94D018BE016F5F7F4FCD
:104BE000CE0107960E94FC77CE0101960E94737851
:104BF0006CEE74E0CE0101960E940379BE01695FFC
:104C00007F4FCE0101960E949A77BC01CE010D968E
:104C10000E94FB784AE050E06FEF7FEFCE010D96E7
:104C200037DECE010D960E947378CE0101960E9468
:104C30007378CE0107960E94737868EE73E080E087
:104C400090E00E94267D0E94B782BC01CE010D96A5
:104C50000E94D0180E94B182BC01CE0101960E9430
:104C6000D0186FED76E0CE0107960E940379BE0161
:104C70006F5F7F4FCE0107960E949A77BC01CE01ED
:104C80000D960E94FC77CE0107960E947378CE01A4
:104C900001960E9473780E945F810E94A4816091B6
:104CA000610C70E0CE0101960E94D0186FED76E0A5
:104CB000CE0107960E940379BE016F5F7F4FCE0140
:104CC00007960E949A77BC01CE010D960E94FC7750
:104CD000CE0107960E947378CE0101960E947378E8
:104CE00062EF74E0CE0101960E940379BE01635F1A
:104CF0007F4FCE0101960E949A77BC01CE010796A4
:104D00000E94FB784AE050E06FEF7FEFCE010796FC
:104D1000BFDDCE0107960E947378CE0101960E94F6
:104D20007378CE010D960E94737868EE73E080E090
:104D300090E00E94267DCE0101960E94961C4AE0DA
:104D400050E06FEF7FEFCE010196A2DDAECE0F5F98
:104D50001F4F68EE73E080E090E00E94267D409156
:104D6000740B5091750B6091760B7091770BCE019F
:104D700001960E948E76CE0101960E94AF17CE0159
:104D800001960E94737843CECF93DF9300D000D07A
:104D9000CDB7DEB70E943D08CE0101960E94961C59
:104DA0004AE050E06FEF7FEFCE01019671DDCE015A
:104DB00001960E94737861E080E00E94E380CE015A
:104DC00001960E94BF756FEA73E1CE0101960E94C1
:104DD000CA7968EF74E08FEA93E10E94387A0E9402
:104DE000E07D6093820C7093830C8093840C90938D
:104DF000850C26960FB6F894DEBF0FBECDBFDF91AF
:104E0000CF9108958F929F92AF92BF92EF92FF92AF
:104E10000F931F93CF93DF93CDB7DEB76E970FB687
:104E2000F894DEBF0FBECDBF0091A30F1091A40F69
:104E30000115110509F4D7C00E94E07D4B015C010A
:104E400078012EE3E20EF11CF70180819181A281AD
:104E5000B381A5019401281B390B4A0B5B0BCA01D6
:104E6000B901683E33E0730781059105A0F128EE92
:104E700033E040E050E00E94CBAF861A970AA80AC0
:104E8000B90AD7018D929D92AD92BC921397F80109
:104E900086A597A5A0A9B1A949015A01880C991C1A
:104EA000AA1CBB1C88159905AA05BB0508F0C1C042
:104EB00016A617A610AA11AAF80182A993A9A4A957
:104EC000B5A988159905AA05BB0508F0BBC012AAAB
:104ED00013AA14AA15AAF80186A597A5A0A9B1A995
:104EE000892B8A2B8B2B09F0B6C0EE5BFF4F80819C
:104EF000833009F0B0C084E08083C80104D80196F3
:104F0000D801D2964D915D916D917C91D597452BAD
:104F1000462B472BA1F4F801EE5BFF4F2081233095
:104F200011F021110CC01082F8013E9684E1DF01DE
:104F30001D928A95E9F7C8010E94831F039682306B
:104F4000910519F0049709F04EC080E590E00E94A9
:104F50000E0B6091A30F7091A40F625F7F4FCE0183
:104F600001960E94837ACE0103960E94060B6091FF
:104F7000A30F7091A40F6A5E7F4FCE0101960E942D
:104F8000837A44E050E0BE016D5F7F4F81E090E0A6
:104F90000E9415956091A30F7091A40F6E5E7F4FD4
:104FA000CE0101960E94837A44E050E0BE016D5F1D
:104FB0007F4F85E090E00E9415956091A30F70915E
:104FC000A40F625E7F4FCE0101960E94837A8B818F
:104FD0009C81AD81BE8180939F0F9093A00FA09381
:104FE000A10FB093A20F60ED77E080E090E00E9407
:104FF000267D0E94BD957C0168EE73E080E090E024
:105000000E94267D0BE010E0EF2841F501501109C8
:1050100029F160ED77E080E090E00E94267D0E941B
:10502000BD957C0168EE73E080E090E00E94267DF3
:10503000EBCF821B930BA40BB50B86A797A7A0AB56
:10504000B1AB3ACF821B930BA40BB50B82AB93ABE6
:10505000A4ABB5AB40CF90E080E052CF85E490E1C7
:105060000E94B61291DE67E079E0CE010D960E94B3
:10507000037964EF73E0CE0143960E94F378CE018A
:1050800049960E94BF758E8D1F928F938D8D1F92B2
:105090008F938C8D1F928F938B8D1F928F938AE5A8
:1050A00094E09F938F9388E79BE09F938F930E9458
:1050B000F6B368E77BE0CE0101960E940379BE015A
:1050C0006F5F7F4FCE010D960E943A78CE01019618
:1050D0000E947378BE016D5E7F4FCE0101960E94E3
:1050E000FB78BE01635F7F4FCE0101960E949A77E5
:1050F000BC01CE0107960E94FB78CE0107960E9464
:10510000AF17CE0107960E947378CE0101960E94D8
:105110007378BE01635F7F4FCE0101960E94FB78DA
:10512000AE014F5F5F4F63E070E08BE792E010DA13
:10513000182FCE0101960E9473780FB6F894DEBF47
:105140000FBECDBF111122C06CEF74E0CE010196ED
:105150000E940379BE016D5E7F4FCE0101960E94D1
:105160009A776DE271E10E949A77BC01CE010796B1
:105170000E94FB78CE0107960E94AF17CE010796DA
:105180000E947378CE0101960E947378CE014396F7
:105190000E947378CE010D960E9473786E960FB6BA
:1051A000F894DEBF0FBECDBFDF91CF911F910F915D
:1051B000FF90EF90BF90AF909F908F9008950F93C6
:1051C0001F93CF93DF9300D000D0CDB7DEB78C0113
:1051D000CE0101960E94961C4AE050E06FEF7FEFEF
:1051E000CE01019655DBCE0101960E947378B8017D
:1051F000CE0101960E94FB786AE070E0CE01019634
:105200000E940F81CE0101960E94737826960FB6F8
:10521000F894DEBF0FBECDBFDF91CF911F910F91EC
:105220000895CF92DF92EF92FF920F931F93CF9347
:10523000DF93CDB7DEB768970FB6F894DEBF0FBE29
:10524000CDBF67E079E0CE0143960E94037965E720
:1052500076E0CE0101960E94F378CE0101960E947D
:10526000C617CE0101960E9473786CA17DA1CE0174
:1052700001960E946376CE0101960E94AF17CE017F
:1052800001960E94737868E676E0CE0101960E944E
:10529000F378CE0101960E94C617CE0101960E94B6
:1052A00073787E0188E2E80EF11C01E010E08CA129
:1052B0009DA1801791070CF1F701619171917F0118
:1052C000CE0101960E946376CE0101960E94C61718
:1052D000CE0101960E9473786BEF75E0CE010196C6
:1052E0000E940379CE0101960E94C617CE01019655
:1052F0000E9473780F5F1F4FDACF6BEF75E0CE011E
:1053000001960E940379CE0101960E94AF17CE014B
:1053100001960E94737869E576E0CE0101960E94BD
:10532000F378CE0101960E94C617CE0101960E9425
:10533000737860910D0C70910E0CCE0101960E9455
:105340006376CE0101960E94C617CE0101960E9497
:1053500073786BEF75E0CE0101960E940379CE0160
:1053600001960E94C617CE0101960E947378609143
:105370000F0C7091100CCE0101960E946376CE0145
:1053800001960E94AF17CE0101960E94737862E4E5
:1053900076E0CE0101960E94F378CE0101960E943C
:1053A000C617CE0101960E947378BE01605D7F4FE3
:1053B000CE0101960E940379CE0101960E94C61784
:1053C000CE0101960E9473786BEF75E0CE010196D5
:1053D0000E940379CE0101960E94C617CE01019664
:1053E0000E947378BE016C5C7F4FCE0101960E94D3
:1053F0000379CE0101960E94AF17CE0101960E945B
:10540000737862E376E0CE0101960E94F378CE01D4
:1054100001960E94AF17CE0101960E9473788E010B
:105420000C5D1F4FEE24E394F12C6801F8E0CF0EE1
:10543000D11C8CA19DA18E159F050CF449C0B7010C
:10544000CE0107960E94637669E977E0CE01019666
:105450000E940379BE01695F7F4FCE0101960E94D1
:105460009A77BC01CE010D960E94FB78CE010D9675
:105470000E94C617CE010D960E947378CE01019648
:105480000E947378CE0107960E9473786FED76E0E4
:10549000CE0101960E940379CE0101960E94C617A3
:1054A000CE0101960E947378B801645E7F4FCE01F1
:1054B00001960E940379CE0101960E94AF17CE019A
:1054C00001960E9473788FEFE81AF80A8601ADCF33
:1054D00068E176E0CE0101960E94F378CE01019654
:1054E0000E94C617CE0101960E9473786CE47CE09E
:1054F000CE0101960E940379CE0101960E94C61743
:10550000CE0101960E94737866E176E0CE010196A5
:105510000E94F378CE0101960E94C617CE01019633
:105520000E9473786091350270913602CE01019627
:105530000E946376CE0101960E94AF17CE010196BC
:105540000E94737867E076E0CE0101960E94F378BE
:10555000CE0101960E94C617CE0101960E94737873
:10556000BE016C5A7F4FCE0101960E940379CE0195
:1055700001960E94AF17CE0101960E94737865E0F4
:1055800075E0CE0101960E940379CE0101960E943A
:10559000C617CE0101960E947378BE0164587F4FF2
:1055A000CE0101960E940379CE0101960E94AF17A9
:1055B000CE0101960E947378C052DF4F8881998195
:1055C000C05ED040892B71F46FEF75E0CE0101967B
:1055D0000E94F378CE0101960E94AF17CE0101968A
:1055E0000E947378C052DF4F88819981C05ED0409D
:1055F000019771F465EF75E0CE0101960E94F37892
:10560000CE0101960E94AF17CE0101960E947378D9
:10561000C052DF4F88819981C05ED040029771F4FB
:105620006CEE75E0CE0101960E94F378CE010196F2
:105630000E94AF17CE0101960E94737866EE75E066
:10564000CE0101960E94F378CE0101960E94C61702
:10565000CE0101960E947378CE51DF4F6881798127
:10566000C25ED040CE0101960E946376CE010196C3
:105670000E94AF17CE0101960E94737840917E0C74
:1056800050917F0C6091800C7091810C21E0CE01D3
:1056900007960E94787860E175E0CE0101960E943D
:1056A0000379BE01695F7F4FCE0101960E949A7710
:1056B0006AE175E00E948677BC01CE010D960E94DA
:1056C000FB78CE010D960E94AF17CE010D960E9479
:1056D0007378CE0101960E947378CE0107960E94DE
:1056E000737840917A0C50917B0C60917C0C709196
:1056F0007D0C21E0CE0107960E9478786FE175E07D
:10570000CE0101960E940379BE01695F7F4FCE01F1
:1057100001960E949A776AE175E00E948677BC0143
:10572000CE010D960E94FB78CE010D960E94AF1718
:10573000CE010D960E947378CE0101960E94737877
:10574000CE0107960E94737869EC75E0CE01019650
:105750000E94F378CE0101960E94C617CE010196F1
:105760000E947378409120025091210260912202A0
:105770007091230225E0CE0101960E947878CE0137
:1057800001960E94AF17CE0101960E9473786FEACE
:1057900075E0CE0101960E94F378CE0101960E9439
:1057A000C617CE0101960E94737840911C02509159
:1057B0001D0260911E0270911F0225E0CE0101962C
:1057C0000E947878CE0101960E94AF17CE01019613
:1057D0000E9473786FE975E0CE0101960E94F3781C
:1057E000CE0101960E94C617CE0101960E947378E1
:1057F00060915D0270915E02CE0101960E94637617
:10580000CE0101960E94AF17CE0101960E947378D7
:105810006DE875E0CE0101960E94F378CE01019605
:105820000E94C617CE0101960E947378C65BDE4FB8
:1058300068817981CA54D140CE0101960E94637675
:10584000CE0101960E94AF17CE0101960E94737897
:10585000CE0143960E94737868960FB6F894DEBF27
:105860000FBECDBFDF91CF911F910F91FF90EF90B1
:10587000DF90CF9008952F923F924F925F926F9258
:105880007F928F929F92AF92BF92CF92DF92EF92D0
:10589000FF920F931F93CF93DF93CDB7DEB7EB97B4
:1058A0000FB6F894DEBF0FBECDBF1C018B0170E0B8
:1058B00060E00E943A778F8F67E079E0CE014996E9
:1058C0000E94037980915D0290915E028130910582
:1058D00009F092C088E090E090931B0280931A0236
:1058E00089E090E0909319028093180280910B0C4C
:1058F00090910C0C90930A0C8093090C80911402E7
:1059000090911502A0911602B09117028093100297
:1059100090931102A0931202B093130280912C0273
:1059200090912D02A0912E02B0912F02809330020F
:1059300090933102A0933202B09333028091080C0D
:105940008093070C8091030C9091040CA091050C9E
:10595000B091060C8093FF0B9093000CA093010C68
:10596000B093020C8AE390E090930F0280930E02B2
:1059700080917E0C90917F0CA091800CB091810C55
:105980008093480C9093490CA0934A0CB0934B0C15
:1059900080910C0290910D0290930B0280930A0269
:1059A0008091200290912102A0912202B0912302C5
:1059B0008093240290932502A0932602B09327029D
:1059C0002F8D233509F089C010920A0C1092090C12
:1059D0008091110C882371F066E275E0CE0101968A
:1059E0000E940379CE0101960E94AF17CE01019665
:1059F0000E947378E12C46C1029711F78AE090E08B
:105A000090931B0280931A028BE090E0909319020E
:105A1000809318028091FD0B9091FE0B90930A0CDD
:105A20008093090C8091060290910702A0910802D0
:105A3000B09109028093100290931102A093120278
:105A4000B09313028091280290912902A0912A021A
:105A5000B0912B028093300290933102A0933202D6
:105A6000B09333028091FC0B8093070C8091F80B6C
:105A70009091F90BA091FA0BB091FB0B8093FF0B67
:105A80009093000CA093010CB093020C8BE390E078
:105A900090930F0280930E0280917A0C90917B0C70
:105AA000A0917C0CB0917D0C8093480C9093490C94
:105AB000A0934A0CB0934B0C809104029091050284
:105AC00090930B0280930A0280911C0290911D0218
:105AD000A0911E02B0911F026BCFC80101970297DF
:105AE00008F0D3C181E090E0A0E0B0E08093100224
:105AF00090931102A0931202B0931302D101149655
:105B00008D919C91029748F141E050E0B101CE01A6
:105B100001960E943108BE016F5F7F4FCE0149960A
:105B20000E943A78CE0101960E947378CE01499680
:105B30000130110581F50E94C77620E030E040E297
:105B400051E40E94F2AE0E94F5B06093100270938F
:105B500011028093120290931302BF8D81E090E0B6
:105B600090930A0C8093090CB13401F58091110CCB
:105B7000882309F43FCF6BE275E0CE0101960E94C5
:105B80000379CE0101960E94AF17CE0101960E94C3
:105B90007378E12C44C00E94C77620912402309192
:105BA00025024091260250912702CBCFEF8DE6349B
:105BB00009F037C161E080911A020E94DF7B023058
:105BC0001105C1F4CE0149960E94C7769B01AC0134
:105BD0006091480C7091490C80914A0C90914B0C4B
:105BE0000E9428B06093480C7093490C80934A0C33
:105BF00090934B0C8091110C882371F064E375E055
:105C0000CE0101960E940379CE0101960E94C6172B
:105C1000CE0101960E947378EE24E394F12C8091DA
:105C2000110C882379F1409110025091110260917A
:105C30001202709113022AE0CE0101960E94A77809
:105C4000BE016F5F7F4FCE0107960E94FB7868E42C
:105C500075E0CE0107960E948677BC01CE010D96B5
:105C60000E94FB78CE010D960E94AF17CE010D96D3
:105C70000E947378CE0107960E947378CE01019638
:105C80000E9473788091100290911102A0911202EB
:105C9000B0911302181619061A061B060CF07AC5E5
:105CA0005F8D563409F481C4523509F482C46E2DD7
:105CB00080911A020E94DF7BC12CD12C76019AE0E0
:105CC000892E912CA12CB12C80911002909111025F
:105CD000A0911202B0911302C816D906EA06FB067B
:105CE0000CF069C46091090C809118020E94DF7B5E
:105CF00061E070E080E090E00E94267D60E08091AD
:105D000018020E94DF7B6091300270913102809115
:105D10003202909133020E94267D80913002909150
:105D20003102A0913202B09133024597A105B1052D
:105D30000CF471C0609110027091110280911202F6
:105D400090911302A50194010E94EDAFC701B60125
:105D50000E94EDAF672B682B692B09F05CC0023005
:105D600011050CF458C080915D0290915E0201977C
:105D700031F460E175E082EE90E10E945A76809104
:105D80005D0290915E02029731F46FE175E082EE60
:105D900090E10E945A76C701B6010E9493AE20910D
:105DA00024023091250240912602509127020E9440
:105DB0008DB0AB01BC0121E0CE0107960E9478783E
:105DC00062EE70E1CE0101960E94FB78BE01695F30
:105DD0007F4FCE0101960E949A776AE175E00E949A
:105DE0008677BC0182EE90E10E942578CE01019673
:105DF0000E947378CE0107960E94737862EE70E17C
:105E0000CE0101960E94FB78CE010196D8D9CE0131
:105E100001960E9473788FEFC81AD80AE80AF80A28
:105E200053CFFF8DF23509F0B4CE60E080911A02B5
:105E30000E94DF7B02301105C1F4CE0149960E9419
:105E4000C7769B01AC016091480C7091490C809120
:105E50004A0C90914B0C0E9429B06093480C7093AF
:105E6000490C80934A0C90934B0C8091110C882321
:105E700009F4C0CD6EE375E0CE0101960E9403796E
:105E8000CE0101960E94C61780CE0115110521F0A2
:105E90000330110509F0AECD81E090E090935E02F1
:105EA00080935D0290930A0C8093090C20915B0211
:105EB00030915C023AAB29AB331F3327331F3BAF22
:105EC000632F80911A020E94DF7B8FEF9FEF9093E8
:105ED0000B0280930A02C12CD12C76011DA61EA6AE
:105EE0001FA618AA19A61AA61BA61CA61BA21CA2AE
:105EF0001DA21EA2412C512C32011FAA18AE19AEB0
:105F00001AAE1BAA1CAA1DAA1EAA61E08091180243
:105F10000E94DF7B61E070E080E090E00E94267DDF
:105F200060E0809118020E94DF7B61E070E080E019
:105F300090E00E94267DC701B60123E030E040E0FA
:105F400050E00E94EDAF672B682B692B09F0F8C079
:105F500043E050E058A74FA3812C912C540180912D
:105F60000E02863308F0865320917B00982F98709C
:105F7000277F922B90937B008770806480937C00B6
:105F800080917A00806480937A0080917A0086FD07
:105F9000FCCF8091780060917900762F682F072ED2
:105FA000000C880B990B0E9493AE9B01AC01C501BC
:105FB000B4010E9429B04B015C0162E070E080E016
:105FC00090E00E94267D8FA198A5019798A78FA3A6
:105FD000892B29F620E030ED4FE355E4C501B401EB
:105FE0000E948DB04B015C018091110C882399F1C6
:105FF0002DEC3CEC4CE45EE3C501B4010E9426B1FB
:1060000087FD29C022E0B501A401CE0107960E94B8
:1060100078786FE475E0CE0101960E940379BE01A5
:10602000695F7F4FCE0101960E949A77BC01CE0135
:106030000D960E94FB78CE010D960E94AF17CE01FF
:106040000D960E947378CE0101960E947378CE015E
:1060500007960E9473782AE939E949E95EE3C501A8
:10606000B4010E9426B187FD13C04114510461049C
:10607000710411F42601370129A53AA54BA55CA5A9
:10608000232B242B252B21F4C9A6DAA6EBA6FCA6EC
:106090002DEC3CEC4CE45EE3C501B4010E948DAEF6
:1060A00018160CF448C0411451046104710409F439
:1060B00047C08BA19CA1ADA1BEA1892B8A2B8B2BA4
:1060C00069F42DA53EA54FA558A9232B242B252BDC
:1060D00009F47DC0CBA2DCA2EDA2FEA28BA19CA103
:1060E000ADA1BEA1481659066A067B064CF5809103
:1060F0000A0290910B0297FF6FC010920B02109250
:106100000A022BA13CA14DA15EA1420E531E641EAA
:10611000751ED301C201B595A795979587958FAB4D
:1061200098AFA9AFBAAF1BA21CA21DA21EA2412C00
:10613000512C320105C0411451046104710471F6FF
:10614000A0910A02B0910B02B8A7AFA3A230B1058B
:106150000CF05EC0B7FD03C003301105B1F0BFEF16
:10616000CB1ADB0AEB0AFB0AE0E4CE16ECE9DE060A
:10617000E104F10409F0C9CE0330110531F05BAD43
:10618000E52E0115110509F07DCDC1010E94C776EC
:106190006B017C01C092480CD092490CE0924A0CF1
:1061A000F0924B0C20E030E044EB53E4C701B60121
:1061B0000E9426B187FDDEC020E030E044EB53E4CE
:1061C000C701B6010E9428B06B017C01EBCFCDA6C0
:1061D000DEA6EFA6F8AA7ECF0115110509F0B0CF13
:1061E000019690930B0280930A022BA13CA14DA132
:1061F0005EA1420E531E641E751ED301C201B595E9
:10620000A795979587958BAB9CABADABBEAB8BCF72
:106210006BA97CA98DA99EA92FA938AD49AD5AAD0E
:10622000621B730B840B950B0E9493AE4B015C01B8
:106230004FA158A5BA01550F880B990B0E9493AE38
:106240009B01AC01C501B4010E948DB020E030E09B
:1062500044EB53E40E948DB04B015C018092240218
:1062600090922502A0922602B092270220E030E010
:1062700040E85FE30E9426B187FD58C080915D022F
:1062800090915E0281309105F1F580921F139092FA
:106290002013A0922113B092221380922002909298
:1062A0002102A0922202B09223026DE174E0CE019D
:1062B00001960E94F378CE0101960E94C617CE0186
:1062C00001960E94737840912402509125026091BA
:1062D00026027091270225E0CE0101960E9478786F
:1062E000CE0101960E94AF17CE0101960E947378ED
:1062F00084EF91E0909391028093900261E072E1CB
:106300000E94F00739CF029781F680922313909272
:106310002413A0922513B092261380921C0290920F
:106320001D02A0921E02B0921F02BFCF61E074E076
:10633000CE0101960E94F378CE0101960E94C61705
:10634000CE0101960E94737840912402509125025B
:10635000609126027091270225E0CE0101960E94ED
:106360007878CE0101960E94AF17CE0101960E9467
:10637000737802CF20E030E0A901C701B6010E9486
:106380008DAE87FF0BC020E030E044EB53E4C70143
:10639000B6010E9429B06B017C01ECCFC092FF0BCB
:1063A000D092000CE092010CF092020C4DA45EA47D
:1063B0006FA478A889A59AA5ABA5BCA5481A590AC7
:1063C0006A0A7B0A01151105D9F41092FF0B10928D
:1063D000000C1092010C1092020CA9A9BAA9812CF0
:1063E000912C54018394C12CD12C7601B7FF26C087
:1063F000C12CD12C760188248A94982C54011EC07B
:10640000E9A9FAA9812C912C54018394F7FF04C0C7
:1064100088248A94982C5401C090FF0BD090000CD3
:10642000E090010CF090020C20E030E044E353E4F3
:10643000C701B6010E948DAE87FF92C0C701B601A9
:1064400090582091240230912502409126025091CB
:1064500027020E94F2AE6B017C01A3019201C501EB
:10646000B4010E94BCAF0E9493AE20E030E040E057
:106470005FE30E94F2AE9B01AC01C701B6010E942E
:1064800028B00E94F5B060931002709311028093BF
:106490001202909313028091110C882309F441C0D9
:1064A0002AE04DA55EA56FA578A9CE010D960E94A4
:1064B000A7782AE049A55AA56BA57CA5CE01079629
:1064C0000E94A77866E575E0CE0101960E940379E7
:1064D000BE01695F7F4FCE0101960E949A776BEFF4
:1064E00075E00E948677BE01635F7F4F0E949A77B6
:1064F000BC01CE0143960E94FB78CE0143960E94D8
:10650000AF17CE0143960E947378CE0101960E9488
:106510007378CE0107960E947378CE010D960E9483
:1065200073788091100290911102A0911202B091A3
:106530001302B7FF36C0B095A095909581959F4FF7
:10654000AF4FBF4F8093100290931102A09312029D
:10655000B0931302EE24E394F12C36E43F8F92CBF8
:106560002091240230912502409126025091270269
:106570002F8F38A349A35AA3A701960160E070E0CA
:1065800084EB93E40E9428B06093FF0B7093000C9F
:106590008093010C9093020C2F8D38A149A15AA130
:1065A00058CFE12C42E54F8F6DCBEE24E394F12CD4
:1065B0007ECBE12C7CCB0230110524F401151105B2
:1065C00009F0E0C061E080E00E94E3800330110543
:1065D00021F00115110509F09CC0C090480CD09025
:1065E000490CE0904A0CF0904B0C20E030E044EB7A
:1065F00053E4C701B6010E9426B187FD0BC020E01D
:1066000030E044EB53E4C701B6010E9428B06B01AF
:106610007C01EBCF20E030E0A901C701B6010E9468
:106620008DAE87FF0BC020E030E044EB53E4C701A0
:10663000B6010E9429B06B017C01ECCFC092480CDE
:10664000D092490CE0924A0CF0924B0C80915D0282
:1066500090915E020197B1F460E175E082EE90E105
:106660000E945A768091480C9091490CA0914A0C56
:10667000B0914B0C80937E0C90937F0CA093800C78
:10668000B093810C80915D0290915E020297B1F40B
:106690006FE175E082EE90E10E945A768091480C9D
:1066A0009091490CA0914A0CB0914B0C80937A0CBC
:1066B00090937B0CA0937C0CB0937D0C4091480C84
:1066C0005091490C60914A0C70914B0C21E0CE0125
:1066D00007960E94787862EE70E1CE0101960E94E2
:1066E000FB78BE01695F7F4FCE0101960E949A77C9
:1066F0006AE175E00E948677BC0182EE90E10E941B
:106700002578CE0101960E947378CE0107960E94EB
:1067100073780130110509F0C8C040911002509102
:106720001102609112027091130221E0CE010796CE
:106730000E94A7786EE575E0CE0101960E9403796C
:10674000BE01695F7F4FCE0101960E949A77BC011E
:1067500082EE90E10E942578CE0101960E94737826
:10676000CE0107960E94737862EE70E1CE01019629
:106770000E94FB78CE0101960E94DF28CE0101968F
:106780000E9473781092100210921102109212025D
:106790001092130280915D0290915E02813091050A
:1067A00009F0D9C08091090C90910A0C90930C0CBF
:1067B00080930B0C8091100290911102A091120213
:1067C000B09113028093140290931502A0931602C5
:1067D000B09317028091300290913102A091320261
:1067E000B091330280932C0290932D02A0932E023D
:1067F000B0932F028091070C8093080C8091FF0BBF
:106800009091000CA091010CB091020C8093030CAC
:106810009093040CA093050CB093060C8091480C47
:106820009091490CA0914A0CB0914B0C80937E0C36
:1068300090937F0CA093800CB093810C80910A02FE
:1068400090910B0290930D0280930C02012B81F426
:106850008091240290912502A0912602B0912702F6
:106860008093200290932102A0932202B0932302EE
:10687000CE0149960E947378EB960FB6F894DEBF6E
:106880000FBECDBFDF91CF911F910F91FF90EF9081
:10689000DF90CF90BF90AF909F908F907F906F9040
:1068A0005F904F903F902F9008950230110509F0AE
:1068B0005BCFC090480CD090490CE0904A0CF0900F
:1068C0004B0C20E030E044EB53E4C701B6010E94DA
:1068D00026B187FD0BC020E030E044EB53E4C70154
:1068E000B6010E9428B06B017C01EBCF20E030E0C4
:1068F000A901C701B6010E948DAE87FF0BC020E041
:1069000030E044EB53E4C701B6010E9429B06B01AB
:106910007C01ECCFC092480CD092490CE0924A0C1A
:10692000F0924B0C21E0B701A601CE0107960E9420
:10693000787865E675E0CE0101960E940379BE0184
:10694000695F7F4FCE0101960E949A776BE175E0F7
:106950000E948677FCCE029709F08ACF8091090CBD
:1069600090910A0C9093FE0B8093FD0B8091100286
:1069700090911102A0911202B0911302809306022D
:1069800090930702A0930802B0930902809130020D
:1069900090913102A0913202B0913302809328028B
:1069A00090932902A0932A02B0932B028091070CA6
:1069B0008093FC0B8091FF0B9091000CA091010C37
:1069C000B091020C8093F80B9093F90BA093FA0B03
:1069D000B093FB0B8091480C9091490CA0914A0C0C
:1069E000B0914B0C80937A0C90937B0CA0937C0C11
:1069F000B0937D0C80910A0290910B029093050256
:106A000080930402012B09F033CF809124029091EE
:106A10002502A0912602B091270280931C02909338
:106A20001D02A0931E02B0931F0222CF2F923F920D
:106A30004F925F926F927F928F929F92AF92BF928E
:106A4000CF92DF92EF92FF920F931F93CF93DF933A
:106A5000CDB7DEB7C055D1090FB6F894DEBF0FBE73
:106A6000CDBF6AEF70E1CE018F5B9F4F0E94FB7834
:106A700023960EAD1FAD23970115110571F0D801B6
:106A80008D918D01882349F0082E000C990B0E94EE
:106A900075B3F80131978083F2CF6CE675E0CE01D3
:106AA00001960E940379BE016F5F7F4FCE018F5B1D
:106AB0009F4F0E946B77182FCE0101960E9473782A
:106AC000112309F403C145E050E06AEF70E1CE0103
:106AD00001960E943108BE016F5F7F4F8CED90E1FF
:106AE0000E943A78CE0101960E9473788CED90E175
:106AF0000E94DD7660E08CED90E10E94D4774091B9
:106B0000E0105091E11069E572E18CED90E10E9496
:106B1000DC7562E574E0CE0101960E940379BE0146
:106B20006F5F7F4F8CED90E10E946B77182FCE0145
:106B300001960E9473786CE374E0111102C061E465
:106B400074E0CE0101960E9403796CED70E1CE01F4
:106B500001960E949A77BC0187E593E10E9425780F
:106B6000CE0101960E94737887E593E10E94DD765D
:106B700040915B1350915C134150510967E573E1FB
:106B8000CE0101960E943108BE016F5F7F4F89E3FD
:106B900093E10E943A78CE0101960E94737889E3CE
:106BA00093E10E94D2760E9493AE9B01AC010E94B9
:106BB0002AB1882309F448C060915B1370915C137B
:106BC0006250710987E593E10E943A77682FCE0100
:106BD00001960E94D378BE016F5F7F4F89E393E1F6
:106BE0000E943A78CE0101960E94737862E574E0C3
:106BF000CE0101960E940379BE016F5F7F4F89E34A
:106C000093E10E946B77182FCE0101960E94737852
:106C10001123D1F060915B1370915C136350710983
:106C200087E593E10E943A77682FCE0101960E9492
:106C3000D378BE016F5F7F4F89E393E10E943A787A
:106C4000CE0101960E94737884EF91E090939102B7
:106C50008093900261E072E10E94F00764E670E0C8
:106C600080E090E00E94267D80913402882371F0BC
:106C70006AEF70E1CE0101960E94FB78CE01019689
:106C80000E941A1BCE0101960E947378CE018F5B81
:106C90009F4F0E94737881E0C05BDF4F0FB6F8947E
:106CA000DEBF0FBECDBFDF91CF911F910F91FF903F
:106CB000EF90DF90CF90BF90AF909F908F907F909C
:106CC0006F905F904F903F902F90089562E775E02E
:106CD000CE0101960E940379BE016F5F7F4FCE0106
:106CE0008F5B9F4F0E946B77182FCE0101960E94F9
:106CF0007378112309F447C045E050E06AEF70E172
:106D0000CE0101960E943108BE016F5F7F4F8CED6E
:106D100090E10E943A78CE0101960E9473788CED42
:106D200090E10E94DD7660E08CED90E10E94D477E6
:106D30004091E0105091E11061E372E18CED90E13F
:106D40000E94DC7561E372E1CE014C960E940379EA
:106D500064E574E0CE0101960E940379BE01645E91
:106D60007F4FCE0101960E949A77BC0181E593E1A5
:106D70000E942578CE0101960E947378CE014C9630
:106D80000E94737861CF68E775E0CE0101960E949A
:106D90000379BE016F5F7F4FCE018F5B9F4F0E94D3
:106DA0006B77182FCE0101960E9473781123E1F0C2
:106DB00043E050E06AEF70E1CE0101960E94310895
:106DC000BE016F5F7F4F8CED90E10E943A78CE015B
:106DD00001960E9473786CED70E1CE0101960E94DD
:106DE000FB78CE010196CCCF6CE775E0CE01019621
:106DF0000E940379BE016F5F7F4FCE018F5B9F4F73
:106E00000E946B77182FCE0101960E947378112390
:106E100001F144E050E06AEF70E1CE0101960E947A
:106E20003108BE016F5F7F4F8CED90E10E943A7890
:106E3000CE0101960E9473788CED90E10E94D2768B
:106E40007093C0126093BF1270937A0260937902BC
:106E5000FBCE61E875E0CE0101960E940379BE0188
:106E60006F5F7F4FCE018F5B9F4F0E946B77182F14
:106E7000CE0101960E947378112309F449C045E0C0
:106E800050E06AEF70E1CE0101960E943108BE0128
:106E90006F5F7F4F8CED90E10E943A78CE010196B2
:106EA0000E9473788CED90E10E94D27670931C134F
:106EB00060931B1384EF91E0909391028093900272
:106EC00061E072E10E94F00764E670E080E090E02B
:106ED0000E94267D69E977E0CE0101960E94037940
:106EE0006AEF70E1CE0101960E949A77BC01CE0153
:106EF0004C960E94FB78CE014C960E94AF17CE01B3
:106F00004C960E947378CE0101960E947378ACCEA5
:106F100067E875E0CE0101960E940379BE016F5FBC
:106F20007F4FCE018F5B9F4F0E946B77182FCE0152
:106F300001960E9473781123E1F044E050E06AEF7B
:106F400070E1CE0101960E943108BE016F5F7F4F54
:106F50008CED90E10E943A78CE0101960E94737800
:106F60008CED90E10E94D27670931E1360931D13F6
:106F7000A1CF6CE875E0CE0101960E940379BE01B5
:106F80006F5F7F4FCE018F5B9F4F0E946B77182FF3
:106F9000CE0101960E9473781123A1F044E050E0E5
:106FA0006AEF70E1CE0101960E943108BE016F5F69
:106FB0007F4F8CED90E10E943A78CE0101960E94BD
:106FC000737882CF61E975E0CE0101960E94037962
:106FD000BE016F5F7F4FCE018F5B9F4F0E946B772B
:106FE000182FCE0101960E9473781123A1F047E07B
:106FF00050E06AEF70E1CE0101960E943108BE01B7
:107000006F5F7F4F8CED90E10E943A78CE01019640
:107010000E94737823CE69E975E0CE0101960E9443
:107020000379BE016F5F7F4FCE018F5B9F4F0E9440
:107030006B77182FCE0101960E9473781111D7CF6C
:1070400061EA75E0CE0101960E940379BE016F5F8F
:107050007F4FCE018F5B9F4F0E946B77182FCE0121
:1070600001960E947378112321F081E00E945E074F
:10707000F5CD6BEA75E0CE0101960E940379BE0161
:107080006F5F7F4FCE018F5B9F4F0E946B77182FF2
:10709000CE0101960E947378112319F00E940227F5
:1070A000DDCD62EB75E0CE0101960E940379BE0151
:1070B0006F5F7F4FCE018F5B9F4F0E946B77182FC2
:1070C000CE0101960E947378112309F454C04AE05E
:1070D00050E06AEF70E1CE0101960E943108BE01D6
:1070E0006F5F7F4F8CED90E10E943A78CE01019660
:1070F0000E9473788CED90E10E94D2760E943B81D1
:107100000E945F816093860C7093870C8093880C3B
:107110009093890C0E945F8160938A0C70938B0C12
:1071200080938C0C90938D0CCE014C960E94121D76
:107130006DEB75E0CE0101960E940379BE01645E9D
:107140007F4FCE0101960E949A77BC01CE018A96AC
:107150000E94FB78CE018A960E94AF17CE018A96D4
:107160000E947378CE0101960E947378CE014C96EE
:107170000E94737879CD63E277E0CE0101960E9498
:107180000379BE016F5F7F4FCE018F5B9F4F0E94DF
:107190006B77182FCE0101960E947378112309F4A2
:1071A0006CC045E050E06AEF70E1CE0101960E94AC
:1071B0003108BE016F5F7F4F8CED90E10E943A78FD
:1071C000CE0101960E9473780E945F816093860CC5
:1071D0007093870C8093880C9093890C8CED90E1D0
:1071E0000E94D2766093B0027093B1028093B20293
:1071F0009093B3026093011370930213809303136F
:1072000090930413209100132093970C672B682B05
:10721000692B11F41092970C84EF91E090939102F6
:107220008093900261E072E10E94F00764E670E0F2
:1072300080E090E00E94267D64EC77E0CE0101962C
:107240000E94F378CE0101960E94C617CE010196E6
:107250000E9473784091B0025091B1026091B202E5
:107260007091B302CE0101960E948E76CE010196F6
:107270000E94AF17CE0101967BCF6EEC75E0CE0178
:1072800001960E940379BE016F5F7F4FCE018F5B35
:107290009F4F0E946B77182FCE0101960E94737842
:1072A0001123D9F14AE050E06AEF70E1CE01019676
:1072B0000E943108BE016F5F7F4F8CED90E10E940C
:1072C0003A78CE0101960E9473788CED90E10E948D
:1072D000D276613071058105910519F481E08093C2
:1072E00000138CED90E10E94D276672B682B692BFE
:1072F00011F410920013809100138093970C88234F
:1073000009F4D8CD0E945F816093860C7093870C3E
:107310008093880C9093890CCDCD69ED75E0CE01FA
:1073200001960E940379BE016F5F7F4FCE018F5B94
:107330009F4F0E946B77182FCE0101960E947378A1
:10734000112359F148E050E06AEF70E1CE01019657
:107350000E943108BE016F5F7F4F8CED90E10E946B
:107360003A78CE0101960E9473788CED90E10E94EC
:10737000D276613071058105910519F481E0809321
:10738000920C8CED90E10E94D276672B682B692BD2
:1073900009F0A0CD1092920C9DCD62EE75E0CE0169
:1073A00001960E940379BE016F5F7F4FCE018F5B14
:1073B0009F4F0E946B77182FCE0101960E94737821
:1073C000112321F145E050E06AEF70E1CE01019612
:1073D0000E943108BE016F5F7F4F8CED90E10E94EB
:1073E0003A78CE0101960E9473788CED90E10E946C
:1073F000D2766130710521F481E08093980C34CC11
:10740000672B09F031CC1092980C2ECC68EE75E009
:10741000CE0101960E940379BE016F5F7F4FCE01BE
:107420008F5B9F4F0E946B77182FCE0101960E94B1
:107430007378112309F472C066E070E08AEF90E17E
:107440000E943A77682FCE0101960E94D378BE0140
:107450006F5F7F4F8CED90E10E943A78CE010196EC
:107460000E9473788CED90E10E94DD7660E08CEDF7
:1074700090E10E94D4778CED90E10E94D2766B016E
:10748000CB01181619060CF0EFCB2091AE0230910B
:10749000AF02261737070CF4E7CB48E050E06AEF5D
:1074A00070E1CE0101960E943108BE016F5F7F4FEF
:1074B0008CED90E10E943A78CE0101960E9473789B
:1074C0008CED90E10E94DD768091E0109091E110CA
:1074D0000997A8F028E030E050E040E06CED70E162
:1074E000CE0101960E941779BE016F5F7F4F8CED30
:1074F00090E10E943A78CE0101960E947378B6011D
:10750000E3E0660F771FEA95E1F76B5E7D4E48E09A
:1075100050E08CED90E10E94DC7596CB6FEE75E04B
:10752000CE0101960E940379BE016F5F7F4FCE01AD
:107530008F5B9F4F0E946B77182FCE0101960E94A0
:107540007378112309F402C26BEF75E0CE014C96FB
:107550000E94037966EF75E0CE0101960E940379DF
:10756000AE01445E5F4FBE016F5F7F4FCE018F5B08
:107570009F4F0E945D99CE0101960E947378CE01C3
:107580004C960E9473786BEF75E0CE014C960E948A
:10759000037968EF75E0CE0101960E940379AE0190
:1075A000445E5F4FBE016F5F7F4FCE018F5B9F4F89
:1075B0000E945D99CE0101960E947378CE014C968F
:1075C0000E9473786BEF75E0CE014C960E940379B0
:1075D0006AEF75E0CE0101960E940379AE01445E28
:1075E0005F4FBE016F5F7F4FCE018F5B9F4F0E9449
:1075F0005D99CE0101960E947378CE014C960E944F
:1076000073786EEF75E0CE014C960E9403796DEFB2
:1076100075E0CE0101960E940379AE01445E5F4F92
:10762000BE016F5F7F4FCE018F5B9F4F0E945D99C0
:10763000CE0101960E947378CE014C960E94737819
:107640006EEF75E0CE014C960E94037967E478E016
:10765000CE0101960E940379AE01445E5F4FBE01E8
:107660006F5F7F4FCE018F5B9F4F0E945D99CE0170
:1076700001960E947378CE014C960E947378CE01D9
:107680008F5B9F4F0E94DD760E945F8160936B0C41
:1076900070936C0C80936D0C90936E0C56E0E52EFD
:1076A000F12C64E6462E512C612C712C8824839495
:1076B000912C5701B3E0AB0EB11C27968EAD9FAD58
:1076C00027970197A816B90608F0CECAB701CE01D0
:1076D0008F5B9F4F0E943A77682FCE014C960E9495
:1076E000D3786701E2E0CE0ED11CFFEFEF1AFF0A5C
:1076F0009601A701BE016F5B7F4FCE0101960E94EC
:107700001779CE0101960E94D2768B01CE010196A7
:107710000E9473780130110521F400911B13109120
:107720001C130330110521F400911D1310911E1339
:107730006BEF75E0CE0101960E940379A601BE01B0
:107740006F5F7F4FCE018F5B9F4F0E94559A6C01F8
:10775000CE0101960E94737867E079E0CE01019630
:107760000E9403791C141D0424F59601A501BE0195
:107770006F5B7F4FCE018A960E941779BE01665DCE
:107780007F4FCE0101960E943A78CE018A960E94E0
:107790007378101611061CF176012FEFE21AF20A27
:1077A000CE0101960E947378CE014C960E947378A8
:1077B00080CFA501BE016F5B7F4FCE018A960E94EC
:1077C0003108BE01665D7F4FCE0101960E943A7876
:1077D000CE018A960E947378101611060CF78091DC
:1077E000AE029091AF02801791070CF446C070E092
:1077F00060E0CE014C960E943A77823509F042C093
:10780000CE0101960E94D276672B682B692B39F442
:10781000F801EE0FFF1FE855FD4F11821082CE01D7
:1078200001960E94D276613071058105910529F596
:10783000F801EE0FFF1FE855FD4F91828082000F87
:10784000111F000F111FF801E456FD4F8081918137
:10785000A281B381181619061A061B0624F040826D
:107860005182628273820E945F81015B1D4FD80149
:107870006D937D938D939C9313971C141D040CF4AE
:107880008BCF8ECF8634E9F5CE0101960E94D27659
:10789000672B682B692B39F4F801EE0FFF1FE75BAC
:1078A000FD4F11821082CE0101960E94D276613086
:1078B00071058105910539F4F801EE0FFF1FE75BB3
:1078C000FD4F91828082000F111F000F111FF801E0
:1078D000E456FD4F80819181A281B381181619066B
:1078E0001A061B0624F040825182628273820E9433
:1078F0005F81015B1D4FF8016083718382839383F5
:10790000BCCF843481F4CE0101960E94D276000F60
:10791000111F000F111FF801E95CFD4F6083718397
:1079200082839383A0CF843509F0A7CFCE0101963F
:107930000E94D276000F111F000F111FF801E456AC
:10794000FD4F6083718382839383D1CF6FEB77E0A8
:10795000CE0101960E94F378BE016F5F7F4FCE018A
:107960008F5B9F4F0E946B77182FCE0101960E946C
:107970007378112309F41CC144E050E06AEF70E110
:10798000CE0101960E943108BE016F5F7F4F8CEDE2
:1079900090E10E943A78CE0101960E9473788CEDB6
:1079A00090E10E94DD7660E08CED90E10E94D4775A
:1079B0004091E0105091E1106CE47CE08CED90E19E
:1079C0000E94DC7562E179E0CE01CB960E940379DA
:1079D0006CED70E1CE01C3960E94FB788FA998AD43
:1079E00010E0892BE1F067E079E0CE018A960E94F1
:1079F000037921968EAD9FAD21979E01295B3F4F64
:107A00007901892B09F05DC0CE01C3960E94D27620
:107A1000D7016C93CE018A960E94737811E0CE0153
:107A2000C3960E947378CE01CB960E94737811237F
:107A300009F41AC98E01095B1F4FEDE2EE2EE2E157
:107A4000FE2E6801B4E0CB0ED11CF80181918F01AC
:107A5000D7018D937D011D8E1C8E1F8E1E8E19A247
:107A600018A24AE0BE016F5F7F4F90E00E94A4AA77
:107A7000BE016F5F7F4FCE014C960E945A76CE01B9
:107A80004C960E94AF17CE014C960E947378C01698
:107A9000D106D9F684EF91E0909391028093900201
:107AA00061E072E10E94F00764E670E080E090E03F
:107AB0000E94267D64EB77E0CE0101960E94F37868
:107AC000D5CB50E040E0BE01655C7F4FCE01C39650
:107AD0000E94559A8C01892B11F40FA918AD4E0103
:107AE000BCE18B0E911C67E079E0C4010E94037930
:107AF0005701D12CC12C782C692C45018E189F0878
:107B00001016110684F59801A601BE016D5C7F4F29
:107B1000CE0101960E941779BE016F5F7F4F872DBE
:107B2000962D0E943A78CE0101960E947378872D97
:107B3000962D0E94D276F50161935F016801FFEFF7
:107B4000CF1ADF0AA601BE01655C7F4FCE01C39646
:107B50000E94559A8C018FA998ADC816D90668F273
:107B600010E000E0CACF8FA998ADC816D906D8F4A6
:107B7000A601BE016D5C7F4FCE0101960E943108C7
:107B8000BE016F5F7F4FCE014C960E943A78CE01C6
:107B900001960E947378CE014C960E94D276E80C32
:107BA000F91CD7016C93CE014C960E94737832CFAA
:107BB0006DEA77E0CE0101960E94F378BE016F5F17
:107BC0007F4FCE018F5B9F4F0E946B77182FCE01A6
:107BD00001960E9473781123E9F146E050E06AEFC4
:107BE00070E1CE0101960E943108BE016F5F7F4FA8
:107BF0008CED90E10E943A78CE0101960E94737854
:107C00008CED90E10E94DD768091E0109091E11082
:107C1000892B09F429C88CED90E10E94D2767093EB
:107C20002A1360932913709336026093350284EF10
:107C300091E0909391028093900261E072E10E9442
:107C4000F00764E670E080E090E00E94267D69E93C
:107C500077E032CF60E076E0CE0101960E940379B2
:107C6000BE016F5F7F4FCE018F5B9F4F0E946B778E
:107C7000182FCE0101960E9473781123A9F06CE8A9
:107C800077E0CE0101960E94F37864E670E0CE01C1
:107C900001960E940F81CE0101960E947378F0E058
:107CA000E0E019950C94343667E076E0CE014C960E
:107CB0000E940379BE01645E7F4F8AEF90E10E94CB
:107CC0006B7711E0811115C06FE076E0CE0101966F
:107CD0000E940379BE016F5F7F4F8AEF90E10E949F
:107CE0006B7711E0811101C010E0CE0101960E9476
:107CF0007378CE014C960E947378112389F167E165
:107D000076E0CE0101960E9403796FE373E1CE0124
:107D100001960E949A77BC0182EE90E10E9425783C
:107D2000CE0101960E94737869E977E0CE01019651
:107D30000E94037962EE70E1CE0101960E949A776B
:107D4000BC01CE014C960E94FB78CE014C960E945D
:107D5000AF17CE014C960E947378CE0101966CC588
:107D600061E276E0CE014C960E940379BE01645E2A
:107D70007F4F8AEF90E10E946B7711E0811115C06F
:107D800068E276E0CE0101960E940379BE016F5F42
:107D90007F4F8AEF90E10E946B7711E0811101C063
:107DA00010E0CE0101960E947378CE014C960E949D
:107DB0007378112369F06EE777E082EE90E10E941C
:107DC000027865E473E182EE90E10E94FC77ACCF2B
:107DD0006FE276E0CE0101960E940379BE016F5FEB
:107DE0007F4FCE018F5B9F4F0E946B77182FCE0184
:107DF00001960E947378112331F00E94DE241092C4
:107E000034020C94343668E376E0CE014C960E943E
:107E10000379BE01645E7F4F8AEF90E10E946B7729
:107E200011E0811115C06DE376E0CE0101960E944C
:107E30000379BE016F5F7F4F8AEF90E10E946B77FD
:107E400011E0811101C010E0CE0101960E9473780B
:107E5000CE014C960E947378112309F441C06EEF55
:107E600075E0CE0101960E9403794091FE10509179
:107E7000FF108D819E81481B590BBE016F5F7F4FA4
:107E80008AEF90E10E940F99AC014F5F5F4F6AEF5C
:107E900070E1CE014C960E943108BE01645E7F4FB6
:107EA0008CED90E10E943A78CE014C960E94737856
:107EB000CE0101960E9473788CED90E10E94D276FB
:107EC0006115710531F481E08093E2020E94F89619
:107ED00096CF6130710509F092CF1092E202F6CF91
:107EE00062E476E0CE0101960E940379BE016F5FE5
:107EF0007F4FCE018F5B9F4F0E946B77182FCE0173
:107F000001960E947378112309F43BC143E050E0CD
:107F10006AEF70E1CE0101960E943108BE016F5FE9
:107F20007F4F8CED90E10E943A78CE0101960E943D
:107F300073786CED70E1CE0101960E94FB78CE0162
:107F400001960E941A1BCE0101960E94737884EF5D
:107F500091E090939102809390026CED70E1CE01DC
:107F600001960E94FB7860E0CE0101960E94E777BF
:107F7000BC018BE493E10E942578CE0101960E941A
:107F800073786CED70E1CE0101960E94FB7860E0A1
:107F9000CE0101960E94E777BC0185E493E10E943F
:107FA0002578CE0101960E94737840914F1350912D
:107FB000501361EC72E18BE493E10E94DC75409117
:107FC000491350914A136CEC72E185E493E10E94ED
:107FD000DC7561E072E180919002909191020E94C3
:107FE000F00766E476E0CE0101960E9403796CED1D
:107FF00070E1CE0101960E949A77BC01CE018A966B
:108000000E94FB78CE0101960E9473788091BD1288
:108010009091BE12892B39F4BE01665D7F4F82EDCF
:108020009CE00E943F7A68EB7BE080E090E00E9459
:10803000267D8091BD129091BE12029709F087C0F3
:108040006CED70E1CE01C3960E94FB786EE476E0A1
:10805000CE0101960E940379CE0101960E942497D9
:10806000CE0101960E94737864EF71E080E090E0A9
:108070000E94267D61E576E0CE0101960E9403799B
:10808000CE0101960E942497CE0101960E9473783A
:108090006CED75E080E090E00E94267D6AE576E078
:1080A000CE0101960E940379CE0101960E94249789
:1080B000CE0101960E94737864EF71E080E090E059
:1080C0000E94267D68E676E0CE0101960E94037943
:1080D000CE0101960E942497CE0101960E947378EA
:1080E00064EF71E080E090E00E94267D66E476E037
:1080F000CE0101960E940379BE016D5C7F4FCE01D7
:1081000001960E949A77BC01CE014C960E94FB78A2
:10811000CE0101960E947378CE014C960E94DD76C6
:10812000BE01645E7F4FCE0101960E94FB78CE01B6
:1081300001960E942497CE0101960E947378CE0189
:108140004C960E947378CE01C3960E94737868EBB8
:108150007BE080E090E00E94267D61EC72E1CE0140
:1081600001960E940379CE0101960E941A1BCE014E
:1081700001960E94737810923402CE018A960C9474
:10818000B83866E776E0CE0101960E940379BE0119
:108190006F5F7F4FCE018F5B9F4F0E946B77182FD1
:1081A000CE0101960E947378112309F486C044E041
:1081B00050E06AEF70E1CE0101960E943108BE01E5
:1081C0006F5F7F4F8CED90E10E943A78CE0101966F
:1081D0000E9473786BE776E0CE0101960E940379E6
:1081E0006CED70E1CE0101960E949A77BC01CE0140
:1081F0004C960E94FB78CE0101960E947378809184
:10820000BD129091BE12892B39F4BE01645E7F4F7E
:1082100082ED9CE00E943F7A68E873E180E090E0A4
:108220000E94267D8091BD129091BE12029759F551
:1082300062E876E0CE0101960E9403798091E01019
:108240009091E110892B19F56BE876E0CE0101964B
:108250000E945A76BE01645E7F4FCE018A960E94CC
:10826000FB78CE018A960E942497CE018A960E94BE
:10827000737868E873E180E090E00E94267DCE018B
:1082800001960E947378109234020C94B638BE01A5
:108290006F5F7F4FCE018A960E94FB78CE018A964F
:1082A0000E942497CE018A960E94737860E777E156
:1082B00080E090E00E94267DCDCF64E976E0CE019B
:1082C00001960E940379BE016F5F7F4FCE018F5BE5
:1082D0009F4F0E946B77182FCE0101960E947378F2
:1082E000112309F45CC06AEF70E18CED90E10E940B
:1082F000257881E0809334026AEF70E1CE01019627
:108300000E94FB78CE0101960E941A1BCE010196B5
:108310000E9473788091BD129091BE12029709F16C
:108320006CED70E182ED9CE00E943F7A68EB7BE0AF
:1083300080E090E00E94267DCE0101960E94BD97CC
:10834000BE016F5F7F4F8AEF90E10E943A78CE01C5
:1083500001960E94737860ED77E080E090E00E94E3
:10836000267D8091BD129091BE12029771F46CED42
:1083700070E1CE0101960E94FB78CE0101960E9429
:108380002497CE0101960E9473788091FE109091FF
:10839000FF10892B09F433CD69E977E0BCC668E9A1
:1083A00076E0CE0101960E940379BE016F5F7F4F98
:1083B000CE018F5B9F4F0E946B77182FCE010196E5
:1083C0000E947378112309F492C18091BD1290919B
:1083D000BE12019709F013CD6EE976E0CE01C39687
:1083E0000E940379BE016D5C7F4F82ED9CE00E948C
:1083F0003F7A6CE271E080E090E00E94267DCE0141
:108400008A960E94BD9764E670E080E090E00E944A
:10841000267D10E000E065E0C62ED12C7AE0A72E84
:10842000B12C69EA76E0CE0101960E94037950E012
:1084300040E0BE016F5F7F4FCE018A960E94559A41
:108440007C01CE0101960E947378A7014F5F5F4FB8
:10845000BE01665D7F4FCE0101960E943108BE01CC
:108460006F5F7F4FCE01C3960E943A78CE0101968E
:108470000E9473788FA998AD892B09F170E060E0B4
:10848000CE01C3960E943A77082E000C990BC09734
:108490000A97A8F46BEA76E0CE0101960E94037970
:1084A000BE016F5F7F4FCE01C3960E946B77E82EAF
:1084B000CE0101960E947378FF24F394E110F12C11
:1084C00065E876E0CE0101960E94F37864E170E001
:1084D000CE0101960E94CB9CCE0101960E9473783A
:1084E0000F5F1F4F62E370E080E090E00E94267D06
:1084F000C801B6010E943AB10197C1F4CE010196BC
:108500000E94461B8D819E81892B09F4BBC0BE0150
:108510006F5F7F4F8AEF90E10E9425780E941635A9
:10852000FF24F394CE0101960E947378CE01019648
:108530000E94BD97BE016F5F7F4FCE018A960E9459
:108540003A78CE0101960E94737862E370E080E091
:1085500090E00E94267D0436110519F0FF2009F4F1
:1085600060CF8091110C8823F1F069E977E0CE01AA
:108570004C960E940379BE016D5C7F4FCE014C96F4
:108580000E949A77BC01CE0101960E94FB78CE0131
:1085900001960E94AF17CE0101960E947378CE011A
:1085A0004C960E9473788FA998AD892B69F070E082
:1085B00060E0CE01C3960E943A77082E000C990B1A
:1085C000C0970A9708F477C063EB76E0CE01019676
:1085D0000E940379CE018A960E947378CE01C396D9
:1085E0000E9473788D819E81009709F446C0E981CD
:1085F000FA812081222309F440C00797F0F165E752
:1086000077E0CE014C960E94F37868EC70E0CE01E2
:108610004C960E94CB9CCE014C960E947378BE0172
:108620006F5F7F4FCE014C960E94FB7860ED77E044
:10863000CE014C960E940F81CE014C960E94737819
:108640006FEB76E0CE014C960E9403796AEF70E101
:10865000CE014C960E949A77BC01CE018A960E9468
:10866000FB78CE018A960E94AF17CE018A960E94AF
:108670007378CE014C960E947378CE0101960E94C9
:108680007378BDCB043111050CF44CCFC801B50192
:108690000E943AB1892B09F045CFBE016D5C7F4F36
:1086A00082ED9CE00E943F7A68EC70E080E090E010
:1086B0000E94267D37CF6BEA76E0CE0101960E94BC
:1086C0000379BE016F5F7F4FCE01C3960E946B7727
:1086D000182FCE0101960E947378111175CFBE013B
:1086E0006D5C7F4FCE0101960E94EB7873CF6DECED
:1086F00076E0CE0101960E940379BE016F5F7F4F45
:10870000CE018F5B9F4F0E946B77182FCE01019691
:108710000E947378112309F4E8C025E030E044E0BA
:1087200050E06AEF70E1CE0101960E941779BE0118
:108730006F5F7F4F8CED90E10E943A78CE010196F9
:108740000E9473786AEF70E1CE0101960E94FB7877
:10875000CE0101960E941A1BCE0101960E947378E9
:108760008CED90E10E94D2766130710509F067C00E
:108770007093BE126093BD1264EB76E0CE01019659
:108780000E94F378CE0101960E941A1BCE01019639
:108790000E94737862ED76E0CE014C960E940379D8
:1087A00065E473E1CE014C960E949A77BC01CE013C
:1087B00001960E94FB7848EC50E06FEF7FEFCE010E
:1087C00001960E944824CE0101960E947378CE0142
:1087D0004C960E9473780E94F29840E052EC61E05F
:1087E00070E082ED9CE00E94517484EF91E09093E0
:1087F00091028093900261E072E10E94F00761EEC5
:1088000076E0CE014C960E9403796FE373E1CE01CE
:108810004C960E949A77BC01CE0101960E94FB788B
:1088200060ED77E0CE0101960E940F81CE010196A6
:108830000E947378CE014C960E947378E0CA61154D
:108840007105D1F51092BE121092BD1266EA76E063
:10885000CE0101960E94F378CE0101960E941A1B68
:10886000CE0101960E94737868ED76E0CE014C96B9
:108870000E94037965E473E1CE014C960E949A77D9
:10888000BC01CE0101960E94FB7848EC50E06FEFEE
:108890007FEFCE0101960E944824CE0101960E94EE
:1088A0007378CE014C960E9473780E94F29840E84B
:1088B00055E260E070E095CF6230710509F09FCA23
:1088C0007093BE126093BD1265E976E0CE01019609
:1088D0000E94F378CE0101960E941A1BCE010196E8
:1088E0000E9473786CED76E0C1CF66EE76E0CE0143
:1088F00001960E940379BE016F5F7F4FCE018F5BAF
:108900009F4F0E946B77182FCE0101960E947378BB
:10891000112309F441C047E050E06AEF70E1CE0155
:1089200001960E943108BE016F5F7F4F8CED90E190
:108930000E943A78CE0101960E94737861EB76E04E
:10894000CE0101960E940379BE016F5F7F4F8CEDCF
:1089500090E10E946B77182FCE0101960E947378E8
:1089600011111092960C62EC74E0CE0101960E94F7
:108970000379BE016F5F7F4F8CED90E10E946B77B2
:10898000182FCE0101960E947378112309F404CDAB
:1089900081E08093960C00CD6EEE76E0CE010196DC
:1089A0000E940379BE016F5F7F4FCE018F5B9F4FA7
:1089B0000E946B77182FCE0101960E9473781123C5
:1089C00081F146E050E06AEF70E1CE0101960E942D
:1089D0003108BE016F5F7F4F8CED90E10E943A78C5
:1089E000CE0101960E9473788CED90E10E94C776CB
:1089F00060930513709306138093071390930813E5
:108A000084EF91E0909391028093900261E072E193
:108A10000E94F00764E670E080E090E00E94267D0E
:108A2000BBCC65EF76E0CE0101960E940379BE01D2
:108A30006F5F7F4FCE018F5B9F4F0E946B77182F28
:108A4000CE0101960E947378112301F148E050E0B5
:108A50006AEF70E1CE0101960E943108BE016F5F9E
:108A60007F4F8CED90E10E943A78CE0101960E94F2
:108A700073788CED90E10E94C77660930B1370932E
:108A80000C1380930D1390930E13BACF6EEF76E014
:108A9000CE0101960E940379BE016F5F7F4FCE0128
:108AA0008F5B9F4F0E946B77182FCE0101960E941B
:108AB0007378112301F149E050E06AEF70E1CE01D3
:108AC00001960E943108BE016F5F7F4F8CED90E1EF
:108AD0000E943A78CE0101960E9473788CED90E165
:108AE0000E94C77660930F13709310138093111335
:108AF0009093121385CF68E077E0CE0101960E9433
:108B00000379BE016F5F7F4FCE018F5B9F4F0E9445
:108B10006B77182FCE0101960E9473781123F1F024
:108B200049E050E06AEF70E1CE0101960E94310801
:108B3000BE016F5F7F4F8CED90E10E943A78CE01CD
:108B400001960E9473788CED90E10E94C7760E9496
:108B5000F5B0709316136093151352CF62E177E06E
:108B6000CE0101960E940379BE016F5F7F4FCE0157
:108B70008F5B9F4F0E946B77182FCE0101960E944A
:108B800073781123F1F04AE050E06AEF70E1CE0112
:108B900001960E943108BE016F5F7F4F8CED90E11E
:108BA0000E943A78CE0101960E9473788CED90E194
:108BB0000E94C7760E94F5B070931413609313134C
:108BC0001FCF6DE177E0CE0101960E940379BE01CF
:108BD0006F5F7F4FCE018F5B9F4F0E946B77182F87
:108BE000CE0101960E947378112311F14BE050E001
:108BF0006AEF70E1CE0101960E943108BE016F5FFD
:108C00007F4F8CED90E10E943A78CE0101960E9450
:108C100073788CED90E10E94C7760E94F5B0609366
:108C20001713709318138093191390931A13E8CEA7
:108C300069E277E0CE0101960E940379BE016F5F81
:108C40007F4FCE018F5B9F4F0E946B77182FCE0115
:108C500001960E9473781123E1F045E050E06AEF3D
:108C600070E1CE0101960E943108BE016F5F7F4F17
:108C70008CED90E10E943A78CE0101960E947378C3
:108C80008CED90E10E94D27670930A1360930913E1
:108C9000B7CE6FE277E0CE0101960E940379BE0164
:108CA0006F5F7F4FCE018F5B9F4F0E946B77182FB6
:108CB000CE0101960E947378112309F45BC20E94D1
:108CC0005F8160936B0C70936C0C80936D0C909330
:108CD0006E0C26E030E045E050E06AEF70E1CE0136
:108CE00001960E941779BE016F5F7F4F8CED90E176
:108CF0000E943A78CE0101960E9473788CED90E143
:108D00000E94D2764B016B0181E080930013809327
:108D1000970C0E945F816093860C7093870C809300
:108D2000880C9093890C8114910491F580911B1308
:108D300090911C13FC01EE0FFF1FE855FD4F1182AF
:108D40001082880F991F880F991FFC01E95CFD4F65
:108D5000108211821282138280911D1390911E1332
:108D6000FC01EE0FFF1FE855FD4F11821082880FA6
:108D7000991F880F991FFC01E95CFD4F1082118239
:108D80001282138258E7E52EF12C04EB10E029C182
:108D9000F1E08F16910409F06BC08091FE10909164
:108DA000FF100897C0F047E050E06AEF70E1CE0195
:108DB00001960E943108CE0101960E94C776609309
:108DC0000513709306138093071390930813CE0135
:108DD00001960E94737880911B1390911C13FC01E3
:108DE000EE0FFF1FE855FD4F21E030E03183208377
:108DF000880F991F880F991FFC01E456FD4F84E8E6
:108E000093E0A0E0B0E080839183A283B3830E94CB
:108E10005F81E0911B13F0911C13EE0FFF1FEE0F0B
:108E2000FF1FE15BFD4F6083718382839383809199
:108E30001D1390911E13FC01EE0FFF1FE855FD4F0F
:108E400011821082880F991F880F991FFC01E15B26
:108E5000FD4F1082118212821382895C9D4FDC01CA
:108E60001D921D921D921C921397F12CE12C8DCF17
:108E7000B2E08B16910409F056C18091FE109091DA
:108E8000FF100897C0F047E050E06AEF70E1CE01B4
:108E900001960E943108CE0101960E94C776609328
:108EA0000B1370930C1380930D1390930E13CE013C
:108EB00001960E94737840900B1350900C136090B1
:108EC0000D1370900E13A301920160910F13709116
:108ED000101380911113909112130E948DAE87FF91
:108EE00010C020E030E040EA50E4C301B2010E942B
:108EF00029B060930F137093101380931113909304
:108F000012138091091390910A13019797FD22C0C3
:108F1000880F991F880F991F8C010D5D1C4F20E051
:108F200030E040E251E460910513709106138091A6
:108F30000713909108130E9429B09B01AC01F8011E
:108F400060817181828193810E9426B110E000E0EE
:108F5000181614F004EB10E080911B1390911C1371
:108F6000FC01EE0FFF1FE855FD4F11821082880FA4
:108F7000991F880F991FFC01E95CFD4F1082118237
:108F80001282138280911D1390911E13FC01EE0F2B
:108F9000FF1FE855FD4F21E030E031832083880F2B
:108FA000991F880F991FFC01E456FD4F80EB94E058
:108FB000A0E0B0E080839183A283B3830E945F81AD
:108FC000E0911D13F0911E13EE0FFF1FEE0FFF1F18
:108FD000E15BFD4F608371838283938338E7E32EE7
:108FE000F12C28E0821A910832E08316910408F0EF
:108FF00062C080919802909199028A35910514F48B
:1090000010E000E080911B1390911C13FC01EE0F07
:10901000FF1FE855FD4F11821082880F991F880F9E
:10902000991FFC01E95CFD4F1082118212821382AC
:1090300080911D1390911E13FC01EE0FFF1FE85548
:10904000FD4F21E030E031832083880F991F880F86
:10905000991FFC01E95CFD4F4CE251E060E070E0DB
:10906000408351836283738384569D4F48E552E069
:1090700060E070E0DC014D935D936D937C931397FA
:109080000E945F81E0911D13F0911E13EE0FFF1FF0
:10909000EE0FFF1FE15BFD4F60837183828393833B
:1090A000B8E0CB16D10421F4109200131092970C63
:1090B00068E7E62EF12CC8010E94FC1590939902F6
:1090C00080939802801B910B97FF03C09195819527
:1090D000910903973CF0C8010E94FC1590939902F6
:1090E00080939802C7010E94701590939B02809311
:1090F0009A028E199F0997FF03C091958195910956
:1091000003973CF0C7010E94701590939B028093D7
:109110009A0265E377E0CE0101960E9403796AEF37
:1091200070E10C949C3EF3E08F16910409F09DCE03
:10913000809198029091990204EB10E08A35910594
:1091400014F410E000E080911B1390911C13FC01BB
:10915000EE0FFF1FE855FD4F11821082880F991FF7
:10916000880F991FFC01E95CFD4F10821182128269
:10917000138234CF6DE377E0CE0101960E9403792C
:10918000BE016F5F7F4FCE018F5B9F4F0E946B7759
:10919000182FCE0101960E947378112389F143E0C4
:1091A00050E0BE016F5B7F4FCE0101960E943108F7
:1091B000BE016F5F7F4F8CED90E10E943A78CE0147
:1091C00001960E9473788091E0109091E110892BB4
:1091D00041F08CED90E10E94D27670935E02609334
:1091E0005D0280915D0290915E020197029708F402
:1091F000D3C881E090E090935E0280935D02CCC87A
:1092000066E177E0CE014C960E940379BE01645E70
:109210007F4FCE018F5B9F4F0E946B7711E08111D2
:1092200016C06EE677E0CE0101960E940379BE017A
:109230006F5F7F4FCE018F5B9F4F0E946B7711E076
:10924000811101C010E0CE0101960E947378CE0119
:109250004C960E947378112309F46AC066E177E0A6
:10926000CE0101960E940379BE016F5F7F4FCE0150
:109270008F5B9F4F0E946B77182FCE0101960E9443
:1092800073781123A1F046E050E0BE016F5B7F4F81
:10929000CE0101960E943108BE016F5F7F4F8CEDB9
:1092A00090E10E943A78CE0101960E9473786EE6B2
:1092B00077E0CE0101960E940379BE016F5F7F4F78
:1092C000CE018F5B9F4F0E946B77182FCE010196C6
:1092D0000E9473781123A1F042E050E0BE016F5B61
:1092E0007F4FCE0101960E943108BE016F5F7F4F14
:1092F0008CED90E10E943A78CE0101960E9473783D
:109300008091E0109091E110892B09F445C86CED33
:1093100070E1CE0101960E94FB7861E070E0CE0121
:1093200001960E943B2CCE0101960E94737834C8AE
:109330006AE477E0CE018A960E940379BE01665DF9
:109340007F4FCE018F5B9F4F0E946B7711E08111A1
:109350002BC061E477E0CE014C960E940379BE01F8
:10936000645E7F4FCE018F5B9F4F0E946B7711E051
:10937000811116C069E477E0CE0101960E9403795D
:10938000BE016F5F7F4FCE018F5B9F4F0E946B7757
:1093900011E0811101C010E0CE0101960E947378A6
:1093A000CE014C960E947378CE018A960E94737803
:1093B000112309F4ECC06AE477E0CE0101960E9423
:1093C0000379BE016F5F7F4FCE018F5B9F4F0E947D
:1093D0006B77182FCE0101960E947378112309F440
:1093E00067C046E050E0BE016F5B7F4FCE01019643
:1093F0000E943108BE016F5F7F4F8CED90E10E94AB
:109400003A78CE0101960E9473788CED90E10E942B
:10941000C7766B017C0120E030E0A9010E9426B1F3
:1094200018160CF091C0A701960160E070E08AE781
:1094300094E40E948DB00E94F5B060933002709366
:1094400031028093320290933302809130029091E6
:109450003102A0913202B0913302181619061A0691
:109460001B0664F081E090E0A0E0B0E08093300261
:1094700090933102A0933202B093330280915D0247
:1094800090915E028130910509F06BC080913002AD
:1094900090913102A0913202B091330280932C025C
:1094A00090932D02A0932E02B0932F020C94CC41E6
:1094B00047E050E0BE016F5B7F4FCE0101960E94F6
:1094C0003108BE016F5F7F4F8CED90E10E943A78CA
:1094D000CE0101960E9473786AEF74E0CE01019686
:1094E0000E940379BE016F5F7F4FCE018F5B9F4F5C
:1094F0000E946B77182FCE0101960E94737811237A
:1095000031F081E090E090935E0280935D026FE421
:1095100076E0CE0101960E940379BE016F5F7F4F16
:10952000CE018F5B9F4F0E946B77182FCE01019663
:109530000E947378112309F468CF82E090E0909341
:109540005E0280935D0261CF81E090E0A0E0B0E038
:109550008093300290933102A0933202B093330291
:1095600074CF029711F00C94CC418091300290910D
:109570003102A0913202B09133028093280290937D
:109580002902A0932A02B0932B020C94CC4161E5EE
:1095900077E0CE01C3960E940379BE016D5C7F4FD8
:1095A000CE018F5B9F4F0E946B7701E0811140C01D
:1095B0006EE977E0CE018A960E940379BE01665D6E
:1095C0007F4FCE018F5B9F4F0E946B7701E081112F
:1095D0002BC06DE977E0CE014C960E940379BE0165
:1095E000645E7F4FCE018F5B9F4F0E946B7701E0DF
:1095F000811116C068E577E0CE0101960E940379DB
:10960000BE016F5F7F4FCE018F5B9F4F0E946B77D4
:1096100001E0811101C000E0CE0101960E94737843
:10962000CE014C960E947378CE018A960E94737880
:10963000CE01C3960E947378002309F468C161E5E6
:1096400077E0CE0101960E940379BE016F5F7F4FE4
:10965000CE018F5B9F4F0E946B77082FCE01019642
:109660000E94737846E050E0011118C06EE977E07F
:10967000CE0101960E940379BE016F5F7F4FCE013C
:109680008F5B9F4F0E946B77082FCE0101960E943F
:109690007378002309F467C042E050E0BE016F5BBD
:1096A0007F4FCE0101960E943108BE016F5F7F4F50
:1096B0008CED90E10E943A78CE0101960E94737879
:1096C0008091E0109091E110892B11F40C94CC4121
:1096D00063EB78E0CE014C960E940379BE01645E94
:1096E0007F4F8CED90E10E946B77811114C06CE983
:1096F00079E0CE0101960E940379BE016F5F7F4F32
:109700008CED90E10E946B7711E0811110E0CE01A9
:1097100001960E947378CE014C960E9473781123B3
:1097200009F4E4C08CED90E10E94C7762091480CCA
:109730003091490C40914A0C50914B0C0E9429B039
:109740006B017C0120E030E044EB53E40E9426B141
:1097500087FD55C020E030E044EB53E4C701B6017B
:109760000E9428B0EDCF43E050E0BE016F5B7F4F19
:10977000CE0101960E943108BE016F5F7F4F8CEDD4
:1097800090E10E943A78CE0101960E9473786AEFC8
:1097900074E0CE0101960E940379BE016F5F7F4F96
:1097A000CE018F5B9F4F0E946B77082FCE010196F1
:1097B0000E947378002331F081E090E090935E0284
:1097C00080935D026FE476E0CE0101960E940379FA
:1097D000BE016F5F7F4FCE018F5B9F4F0E946B7703
:1097E000082FCE0101960E947378002309F468CFF8
:1097F00082E090E090935E0280935D0261CF20E072
:1098000030E0A901C701B6010E948DAE87FF0BC0F1
:1098100020E030E044EB53E4C701B6010E9429B0D8
:109820006B017C01ECCFC092480CD092490CE092C5
:109830004A0CF0924B0C8CED90E10E94C77620E030
:1098400030E0A9010E9426B187FD15C06CE979E0DE
:10985000CE0101960E9403796CED70E1CE01019674
:109860000E949A77BC018CED90E10E942578CE0190
:1098700001960E9473788CED90E10E94C77620E0FB
:1098800030E0A9010E948DAE87FF30C08CED90E1E1
:109890000E94C77620E030E0A9010E9426B1181688
:1098A00074F58CED90E10E94C776AB01BC0122E01B
:1098B000CE014C960E94787863EB78E0CE01019659
:1098C0000E940379BE01645E7F4FCE0101960E9423
:1098D0009A77BC018CED90E10E942578CE0101962B
:1098E0000E947378CE014C960E9473786CED70E103
:1098F000CE0101960E94FB7862E070E010CD8CED05
:1099000090E10E94C776AB01BC017058D0CF6DE5E5
:1099100077E0CE018A960E940379BE01665D7F4F93
:10992000CE018F5B9F4F0E946B7711E081112BC09E
:109930006CE577E0CE014C960E940379BE01645E2F
:109940007F4FCE018F5B9F4F0E946B7711E081119B
:1099500016C063E677E0CE0101960E940379BE014E
:109960006F5F7F4FCE018F5B9F4F0E946B7711E03F
:10997000811101C010E0CE0101960E947378CE01E2
:109980004C960E947378CE018A960E9473781123B8
:1099900009F48BC0CE018F5B9F4F0E94DD766DE591
:1099A00077E0CE0101960E940379BE016F5F7F4F81
:1099B000CE018F5B9F4F0E946B77182FCE010196CF
:1099C0000E947378112329F145E050E0BE016F5BDE
:1099D0007F4FCE0101960E943108BE016F5F7F4F1D
:1099E0008CED90E10E943A78CE0101960E94737846
:1099F0008091E0109091E110892B11F40C94CC41EE
:109A00006CED70E1CE0101960E94FB7863E070E09E
:109A100086CC46E050E0BE016F5B7F4FCE010196E1
:109A20000E943108BE016F5F7F4F8CED90E10E9474
:109A30003A78CE0101960E9473786AEF74E0CE0105
:109A400001960E940379BE016F5F7F4FCE018F5B4D
:109A50009F4F0E946B77182FCE0101960E9473785A
:109A6000112331F081E090E090935E0280935D02DB
:109A70006FE476E0CE0101960E940379BE016F5F2C
:109A80007F4FCE018F5B9F4F0E946B77182FCE01C7
:109A900001960E947378112309F4AACF82E090E026
:109AA00090935E0280935D02A3CF6BE677E0CE01D8
:109AB0008A960E940379BE01665D7F4FCE018F5B5F
:109AC0009F4F0E946B7711E081112BC06AE677E00F
:109AD000CE014C960E940379BE01645E7F4FCE0199
:109AE0008F5B9F4F0E946B7711E0811116C061E779
:109AF00077E0CE0101960E940379BE016F5F7F4F30
:109B0000CE018F5B9F4F0E946B7711E0811101C0E6
:109B100010E0CE0101960E947378CE014C960E940F
:109B20007378CE018A960E947378112309F428C1B4
:109B30006BE677E0CE0101960E940379BE016F5F6C
:109B40007F4FCE018F5B9F4F0E946B77182FCE0106
:109B500001960E947378112309F443C045E050E058
:109B6000BE016F5B7F4FCE0101960E943108BE019E
:109B70006F5F7F4F8CED90E10E943A78CE010196A5
:109B80000E9473788091E0109091E110892B61F030
:109B90008CED90E10E94C7766093480C7093490C5D
:109BA00080934A0C90934B0CC090480CD090490C79
:109BB000E0904A0CF0904B0C20E030E044EB53E492
:109BC000C701B6010E9426B187FD57C020E030E0F2
:109BD00044EB53E4C701B6010E9428B06B017C013D
:109BE000EBCF46E050E0BE016F5B7F4FCE010196A8
:109BF0000E943108BE016F5F7F4F8CED90E10E94A3
:109C00003A78CE0101960E9473786AEF74E0CE0133
:109C100001960E940379BE016F5F7F4FCE018F5B7B
:109C20009F4F0E946B77182FCE0101960E94737888
:109C3000112331F081E090E090935E0280935D0209
:109C40006FE476E0CE0101960E940379BE016F5F5A
:109C50007F4FCE018F5B9F4F0E946B77182FCE01F5
:109C600001960E947378112309F48CCF82E090E072
:109C700090935E0280935D0285CF20E030E0A901E1
:109C8000C701B6010E948DAE87FF0BC020E030E017
:109C900044EB53E4C701B6010E9429B06B017C017B
:109CA000ECCFC092480CD092490CE0924A0CF09252
:109CB0004B0C80915D0290915E02019771F4C0920D
:109CC0007E0CD0927F0CE092800CF092810C60E1CF
:109CD00075E082EE90E10E945A768091480C909156
:109CE000490CA0914A0CB0914B0C20915D0230912F
:109CF0005E022230310571F480937A0C90937B0CD4
:109D0000A0937C0CB0937D0C6FE175E082EE90E146
:109D10000E945A764091480C5091490C60914A0C2F
:109D200070914B0C21E0CE014C960E94787862EE47
:109D300070E1CE0101960E94FB78BE01645E7F4F08
:109D4000CE0101960E949A776AE175E00E948677BB
:109D5000BC0182EE90E10E942578CE0101960E941E
:109D60007378CE014C960E94737862EE70E1CE015A
:109D700001960E94FB78CE0101960E94DF28D3CA8B
:109D800069E777E0CE018A960E940379BE01665D9D
:109D90007F4FCE018F5B9F4F0E946B7711E0811147
:109DA0002BC068E777E0CE014C960E940379BE0194
:109DB000645E7F4FCE018F5B9F4F0E946B7711E0F7
:109DC000811116C06EE777E0CE0101960E940379FB
:109DD000BE016F5F7F4FCE018F5B9F4F0E946B77FD
:109DE00011E0811101C010E0CE0101960E9473784C
:109DF000CE014C960E947378CE018A960E947378A9
:109E0000112309F415C2C0903002D0903102E090C5
:109E10003202F090330264E877E0CE0101960E94AE
:109E20000379BE016F5F7F4FCE018F5B9F4F0E9412
:109E30006B77182FCE0101960E947378112309F4D5
:109E400065C044E050E0BE016F5B7F4FCE010196DC
:109E50000E943108BE016F5F7F4F8CED90E10E9440
:109E60003A78CE0101960E94737880915D029091BC
:109E70005E028130910509F095C0C0902C02D0900F
:109E80002D02E0902E02F0902F0281E090E0A0E001
:109E9000B0E080932C0290932D02A0932E02B093F9
:109EA0002F028091E0109091E110892B09F092C06F
:109EB00069E877E08CED90E10E945A768091E0109D
:109EC0009091E110892B81F06CED70E1CE0101964B
:109ED0000E94FB7870E060E0CE0101960E943B2C6E
:109EE000CE0101960E94737880915D0290915E028E
:109EF0008130910509F08EC1C0922C02D0922D02C2
:109F0000E0922E02F0922F020C94CC4145E050E0FA
:109F1000BE016F5B7F4FCE0101960E943108BE01EA
:109F20006F5F7F4F8CED90E10E943A78CE010196F1
:109F30000E9473786AEF74E0CE0101960E94037963
:109F4000BE016F5F7F4FCE018F5B9F4F0E946B778B
:109F5000182FCE0101960E947378112331F081E011
:109F600090E090935E0280935D026FE476E0CE0114
:109F700001960E940379BE016F5F7F4FCE018F5B18
:109F80009F4F0E946B77182FCE0101960E94737825
:109F9000112309F46ACF82E090E090935E028093EF
:109FA0005D0263CF029709F07CCFC0902802D09069
:109FB0002902E0902A02F0902B0281E090E0A0E0DC
:109FC000B0E08093280290932902A0932A02B093D4
:109FD0002B0267CF6FE877E0CE0101960E940379EC
:109FE000BE016F5F7F4F8CED90E10E944B77182F81
:109FF000CE0101960E947378112309F475CF8CED80
:10A0000090E10E94C77620E030E0A9010E948DAE69
:10A01000811128C080915D0290915E02019731F418
:10A0200062E977E08CED90E10E945A7680915D02C2
:10A0300090915E02029731F469E877E08CED90E14F
:10A040000E945A768091E0109091E110892B09F4DA
:10A050004BCF6CED70E1CE0101960E94FB7861E080
:10A0600070E03ACF6EEF75E0CE0101960E94037961
:10A07000BE016F5F7F4F8CED90E10E944B77182FF0
:10A08000CE0101960E947378112309F42DCF41E08F
:10A0900050E06CED70E1CE0101960E943108CE01D6
:10A0A00001960E94C7764B015C01CE0101960E9489
:10A0B000737820E030E0A901C501B4010E948DAEA3
:10A0C000181634F0812C912C50E8A52E5FE3B52EA4
:10A0D00000915D0210915E020130110509F075C01A
:10A0E000A501940160E070E48CE995E40E948DB0D4
:10A0F0006093240270932502809326029093270296
:10A1000060931F1370932013809321139093221355
:10A110006093200270932102809322029093230285
:10A12000B801CE014C960E94637667E977E0CE01D4
:10A1300001960E940379BE01645E7F4FCE010196B5
:10A140000E949A77BC01CE018A960E94FB78CE01CC
:10A150008A960E94C617CE018A960E947378CE0115
:10A1600001960E947378CE014C960E94737863E644
:10A1700077E0CE0101960E94F378CE0101960E940D
:10A18000C617CE0101960E94737840912402509127
:10A190002502609126027091270225E0CE010196EA
:10A1A0000E947878CE0101960E94AF17CE010196E9
:10A1B0000E94737884EF91E09093910280939002D3
:10A1C00061E072E10E94F0078FCE0230110509F0C4
:10A1D000A7CFA501940160E070E48CE196E40E94B1
:10A1E0008DB0609324027093250280932602909391
:10A1F0002702609323137093241380932513909365
:10A20000261360931C0270931D0280931E0290938C
:10A210001F0286CF029711F00C94CC41C092280205
:10A22000D0922902E0922A02F0922B020C94CC41A7
:10A230006CE977E0CE018A960E940379BE01665DE3
:10A240007F4FCE018F5B9F4F0E946B7711E0811192
:10A250002BC06BE977E0CE014C960E940379BE01DA
:10A26000645E7F4FCE018F5B9F4F0E946B7711E042
:10A27000811116C061EA77E0CE0101960E94037950
:10A28000BE016F5F7F4FCE018F5B9F4F0E946B7748
:10A2900011E0811101C010E0CE0101960E94737897
:10A2A000CE014C960E947378CE018A960E947378F4
:10A2B000112309F42EC127968EAD9FAD27970597E0
:10A2C00010F40C94CC4144E050E0BE016F5B7F4F32
:10A2D000CE0101960E943108BE016F5F7F4F8CED69
:10A2E00090E10E943A78CE0101960E9473786CE961
:10A2F00077E0CE0101960E940379BE016F5F7F4F28
:10A30000CE018F5B9F4F0E946B77182FCE01019675
:10A310000E947378112309F49BC044E050E0BE0111
:10A320006F5B7F4FCE0101960E943108BE016F5FC7
:10A330007F4F8CED90E10E943A78CE0101960E9409
:10A3400073788CED90E10E94C77620E030E0A9019F
:10A350000E9426B1181614F00C94CC418CED90E1BB
:10A360000E94C77660932402709325028093260290
:10A370009093270220915D0230915E0221303105D9
:10A3800009F0B2C060931F137093201380932113C0
:10A3900090932213609320027093210280932202F3
:10A3A00090932302B901CE014C960E94637667E92F
:10A3B00077E0CE0101960E940379BE01645E7F4F73
:10A3C000CE0101960E949A77BC01CE018A960E9426
:10A3D000FB78CE018A960E94C617CE018A960E940B
:10A3E0007378CE0101960E947378CE014C960E943C
:10A3F000737861E577E0CE0101960E94F378CE0193
:10A4000001960E94C617CE0101960E947378409172
:10A41000240250912502609126027091270225E0C6
:10A42000CE0101960E947878CE0101960E94AF1766
:10A43000CE0101960E94737884EF91E0909391028F
:10A440008093900261E072E10E94F0070C94CC418D
:10A4500045E050E0BE016F5B7F4FCE0101960E9448
:10A460003108BE016F5F7F4F8CED90E10E943A781A
:10A47000CE0101960E9473786AEF74E0CE010196D6
:10A480000E940379BE016F5F7F4FCE018F5B9F4FAC
:10A490000E946B77182FCE0101960E9473781123CA
:10A4A00031F081E090E090935E0280935D026FE472
:10A4B00076E0CE0101960E940379BE016F5F7F4F67
:10A4C000CE018F5B9F4F0E946B77182FCE010196B4
:10A4D0000E947378112309F434CF82E090E09093C6
:10A4E0005E0280935D022DCF2230310509F05ACFF4
:10A4F0006093231370932413809325139093261352
:10A5000060931C0270931D0280931E0290931F02A1
:10A5100049CF69E875E0CE014C960E940379BE01EF
:10A52000645E7F4FCE018F5B9F4F0E946B7711E07F
:10A53000811116C067EA77E0CE0101960E94037987
:10A54000BE016F5F7F4FCE018F5B9F4F0E946B7785
:10A5500011E0811101C010E0CE0101960E947378D4
:10A56000CE014C960E947378112309F46CC069E8FF
:10A5700075E0CE0101960E940379BE016F5F7F4FA7
:10A58000CE018F5B9F4F0E946B77182FCE010196F3
:10A590000E947378112399F042E050E06AEF70E175
:10A5A000CE0101960E943108BE016F5F7F4F8CED96
:10A5B00090E10E943A78CE0101960E94737867EA92
:10A5C00077E0CE0101960E940379BE016F5F7F4F55
:10A5D000CE018F5B9F4F0E946B77182FCE010196A3
:10A5E0000E947378112399F043E050E06AEF70E124
:10A5F000CE0101960E943108BE016F5F7F4F8CED46
:10A6000090E10E943A78CE0101960E9473788CED19
:10A6100090E10E94D276653B710548F4CB010E941F
:10A62000FC1590939902809398020C94CC416EE3B0
:10A6300077E0CE0101960E94F378CE0101960E9448
:10A64000C6170C9493496BEA77E0CE0101960E94FD
:10A650000379BE016F5F7F4FCE018F5B9F4F0E94DA
:10A660006B77182FCE0101960E947378112309F49D
:10A67000FBC226E030E044E050E06AEF70E1CE013A
:10A6800001960E941779BE016F5F7F4F8CED90E1BC
:10A690000E943A78CE0101960E9473788CED90E189
:10A6A0000E94D2766B018B016EEF75E0CE010196B0
:10A6B0000E9403794091FE105091FF108D819E8180
:10A6C000481B590BBE016F5F7F4F8AEF90E10E94DC
:10A6D0000F99AC014F5F5F4F6AEF70E1CE014C966E
:10A6E0000E943108BE01645E7F4F8CED90E10E94B4
:10A6F0003A78CE014C960E947378CE0101960E9462
:10A7000073788CED90E10E94C7762B013C01F60135
:10A7100031972D96FFAFEEAF2D978091110C8823C6
:10A72000C1F16DEB76E0CE0101960E94F378CE0187
:10A7300001960E94C617CE0101960E947378B60159
:10A74000CE0101960E946376CE0101960E94C61743
:10A75000CE0101960E9473786BEF75E0CE010196F1
:10A760000E940379CE0101960E94C617CE01019680
:10A770000E94737822E0B301A201CE0101960E94EB
:10A780007878CE0101960E94AF17CE0101960E9403
:10A79000737860E088E30E94F57CEFE3FBE0E491EE
:10A7A000EC8FE9EFFAE0E491F0E0EE0FFF1FE955DE
:10A7B000F54F859194919E8F8D8F1FA219A618A693
:10A7C000CE014C9698878F831D821E82198289E064
:10A7D0008A8381E08B838C831C8A1B8A1EA21DA224
:10A7E0001CA21BA21AA219A218A21F8EBB24B394EA
:10A7F000BE01665D7F4F8F8198850E94AC9B882348
:10A8000009F45BC067E0CE018A960E94719A99A90B
:10A810008913EECF898181111DC08F8198850E9497
:10A82000F19ABE01665D7F4F8F8198850E94B09A34
:10A8300040E064EB8F8198850E947D9A8F81988596
:10A840000E94CD9AA82E8F8198850E94F19AA1101E
:10A8500001C0B982AA808AA5803109F4ECC4BE0186
:10A86000665D7F4FCE0101960E94839B8A1590F40E
:10A870008A818A838D818F5F8D838AA5883231F0AA
:10A88000B0F4803119F0823209F0B2CF8E818F5F3F
:10A890008E83AECF8AA5803111F48CE0EACFBE0161
:10A8A000665D7F4FCE0101960E94839BE2CF8B3382
:10A8B00069F3823409F09CCFE9CF8F8198850E949B
:10A8C000F19A40E06CEC8F8198850E947D9A4981D5
:10A8D00064E48F8198850E947D9A8B818823D9F1C9
:10A8E000EA81E9502EEE222E22E0322EE33038F4B7
:10A8F000F0E0EE0FFF1FE35EFC4F208031808C8183
:10A90000882309F470C0898181116DC00E94E07DA7
:10A910004B015C019101330C440B550B61962CAF3C
:10A920003DAF4EAF5FAF61978F8198850E94CD9A02
:10A93000813089F00E94E07D61962CAD3DAD4EAD39
:10A940005FAD6197621B730B840B950B68157905DE
:10A950008A059B0548F38CE08A83B12CA12CBFE7C4
:10A960002B2E8FE1382E9FE3892E8D818A151B04B3
:10A9700009F00CF4A0C04A2DBE016D5C7F4FCE01E2
:10A9800001960E942A9C9A803CE0391598F5ACE02B
:10A990009A2E8BA98031A1F1BE016D5C7F4FCE0153
:10A9A00001960E94839B891509F47CC0AE01465D27
:10A9B0005F4FBE016D5C7F4FCE0101960E94299BC7
:10A9C000882309F46FC08BA9803109F46BC05BE068
:10A9D000951609F46BC08CE09816A1F09AE09912D4
:10A9E00068C08EA610C0B101330C880B990B0E9471
:10A9F000267DB1CF49E0941660F6F9E09F2EC9CFCD
:10AA00008CE0D1CF2EA68F8198850E94F19ABE014D
:10AA10006D5C7F4F8F8198850E94B09A40E06EE414
:10AA20008F8198850E947D9A40E06CA58F819885E2
:10AA30000E947D9A40E06DA58F8198850E947D9A45
:10AA40008BA9803131F040E06EA58F8198850E94FE
:10AA50007D9A8F8198850E94F19ABE016D5C7F4F2F
:10AA60008F8198850E94B09A498168E48F8198858A
:10AA70000E947D9A64E170E080E090E00E94267D73
:10AA80008981882331F06AE070E080E090E00E94E4
:10AA9000267D8F8198850E94F19A8A81891508F414
:10AAA000892D8A83BFEFAB1ABB0A5FCFAFE5AEA794
:10AAB000AACF3EA6A8CFAE80B12CEBE0AE16B10473
:10AAC0001CF0EAE0AE2EB12CFBE5CF16D10408F461
:10AAD0004AC070E2C72E7CE0D72E7601412C512C63
:10AAE000320110E000E0A016B106B1F0602FCE01F7
:10AAF00001960E94619C9B01AC01D7012D933D936F
:10AB00004D935D937D01C301B2010E9429B02B01D9
:10AB10003C010F5F1F4FE7CFB801012E000C880BDF
:10AB2000990B0E9493AE9B01AC01C301B2010E943C
:10AB30008DB04B015C01F12CE12C0E151F05E9F1E4
:10AB4000F6012081318142815381C501B4010E9407
:10AB500028B0D6016D937D938D939D936D01BFEFCA
:10AB6000EB1AFB0AEACF101611060CF05EC0A01615
:10AB7000B10634F4F50131972D96FFAFEEAF2D9766
:10AB80002C966FAD2C97CE0101960E94619C9B0183
:10AB9000AC012D960EAD1FAD2D97000F111F000FAC
:10ABA000111F005E134FC301B2010E9428B0D801EB
:10ABB0006D937D938D939C93139788E2E0E2FCE084
:10ABC000A8EDB2E101900D928A95E1F784EF91E052
:10ABD000909391028093900261E072E10E94F007ED
:10ABE0006DE177E082EE90E10E94027844E050E06F
:10ABF0006AEF70E1CE0101960E943108BE016F5FDD
:10AC00007F4F82EE90E10E94FC77CE0101960E9478
:10AC1000737862EE70E1CE0101960E94FB78CE015E
:10AC200001960E94AF170C943D430115110529F6BA
:10AC300020E2E22E2CE0F22EA016B10609F4BDCFE0
:10AC4000602FCE0101960E94619C9B01AC01C30163
:10AC5000B2010E9428B0F70161937193819391939F
:10AC60007F010F5F1F4FE8CF6FEA77E0CE010196BB
:10AC70000E940379BE016F5F7F4FCE018F5B9F4FB4
:10AC80000E946B77182FCE0101960E9473781111E4
:10AC90000C948B4467EB77E0CE0101960E94037918
:10ACA000BE016F5F7F4FCE018F5B9F4F0E946B771E
:10ACB000182FCE0101960E947378112371F141E0A3
:10ACC0006AEB72E0CE0101960E947B92BE016F5F3B
:10ACD0007F4F8DE593E10E94DD178DE593E10E94A2
:10ACE0002992811104C061ED76E00C945C3D8DE504
:10ACF00093E10E940473892B51F08DE593E10E944A
:10AD00000D8C682F89EA9EE00E941671F0CF8DE5C8
:10AD100093E10E9435920C9434366EEB77E0CE01CD
:10AD200001960E940379BE016F5F7F4FCE018F5B5A
:10AD30009F4F0E946B77182FCE0101960E94737867
:10AD40001123E9F02DB73EB72A5231400FB6F894DF
:10AD50003EBF0FBE2DBFADB7BEB711968AE291E0E0
:10AD6000E1E0F2E101900D920197E1F70E941129D3
:10AD70000FB6F894DEBF0FBECDBF0C94343667EC2F
:10AD800077E0CE0101960E940379BE016F5F7F4F8D
:10AD9000CE018F5B9F4F0E946B77182FCE010196DB
:10ADA0000E947378112309F459C08DB79EB78A5257
:10ADB00091400FB6F8949EBF0FBE8DBFADB7BEB722
:10ADC00011968AE291E0E1E0F2E101900D920197A3
:10ADD000E1F70E9405210FB6F894DEBF0FBECDBF8C
:10ADE0006CE077E0CE0101960E94F378EDB7FEB7F4
:10ADF000EA52F1400FB6F894FEBF0FBEEDBFADB7FB
:10AE0000BEB711968AE291E0E1E0F2E101900D9285
:10AE10000197E1F70E9406190FB6F894DEBF0FBE46
:10AE2000CDBF4DB75EB74A5251400FB6F8945EBFE2
:10AE30000FBE4DBFADB7BEB711968AE291E0E1E01B
:10AE4000F2E101900D920197E1F70E9411290FB6EE
:10AE5000F894DEBF0FBECDBF0C943A3969EC77E0B1
:10AE6000CE0101960E940379BE016F5F7F4FCE0134
:10AE70008F5B9F4F0E946B77182FCE0101960E9427
:10AE800073781123F9F06AEF76E0CE0101960E9403
:10AE9000F378BE016F5F7F4FCE014C960E94FB7826
:10AEA000CE014C960E94AF17CE014C960E9473784B
:10AEB000ADB7BEB7AA52B1400FB6F894BEBF0FBE31
:10AEC000ADBFBACF6DEC77E0CE0101960E94037959
:10AED000BE016F5F7F4FCE018F5B9F4F0E946B77EC
:10AEE000182FCE0101960E947378112309F4F5C042
:10AEF0006EED76E0CE018A960E94F378BE01665D23
:10AF00007F4FCE0101960E94FB78AE014F5F5F4FED
:10AF100062E070E08CE692E00E94A822182FCE0139
:10AF200001960E947378111122C0BE01665D7F4FA9
:10AF3000CE014C960E94FB7861ED77E0CE014C96F5
:10AF40000E9486776DE271E10E949A77BC01CE0182
:10AF500001960E94FB78CE0101960E94AF17CE01A8
:10AF600001960E947378CE014C960E94737868EE29
:10AF700073E080E090E00E94267DBE01665D7F4F19
:10AF8000CE0101960E94FB78AE014F5F5F4F63E0F8
:10AF900070E08FE592E00E94A822182FCE01019662
:10AFA0000E947378111122C0BE01665D7F4FCE01F1
:10AFB0004C960E94FB7861EE77E0CE014C960E94A1
:10AFC00086776DE271E10E949A77BC01CE0101960D
:10AFD0000E94FB78CE0101960E94AF17CE01019628
:10AFE0000E947378CE014C960E94737868EE73E0ED
:10AFF00080E090E00E94267D61E271E1CE01019641
:10B000000E94FB78AE014F5F5F4F61E070E084ED1E
:10B0100092E00E94A822182FCE0101960E94737818
:10B02000111121C061E271E1CE014C960E94FB78C2
:10B0300061EE77E0CE014C960E9486776DE271E179
:10B040000E949A77BC01CE0101960E94FB78CE0146
:10B0500001960E94AF17CE0101960E947378CE012F
:10B060004C960E94737868EE73E080E090E00E9456
:10B07000267D8091960C882311F40C94BD4043E109
:10B0800064ED72E0CE0101960E947B92BE016F5F7B
:10B090007F4F83E993E10E94DD1783E993E10E94EA
:10B0A0002992882311F40C94BD4061E271E183E997
:10B0B00093E10E944D7A66E970E080E090E00E94A2
:10B0C000267D83E993E10E94359262E370E080E09F
:10B0D00090E00E94267D0C94BD406DEE77E0CE019D
:10B0E00001960E940379BE016F5F7F4FCE018F5B97
:10B0F0009F4F0E946B77182FCE0101960E947378A4
:10B10000112301F192E1E92E9CE0F92E01E010E01B
:10B11000F2E0EF0EF11C8091AE029091AF02801729
:10B12000910714F40C94343660E0D7018C910E949E
:10B13000DF7B6CE271E080E090E00E94267D0F5F93
:10B140001F4FE6CF61EF77E0CE0101960E940379B1
:10B15000BE016F5F7F4FCE018F5B9F4F0E946B7769
:10B16000182FCE0101960E947378112301F182E11C
:10B17000E82E8CE0F82E01E010E0B2E0EB0EF11CBE
:10B180008091AE029091AF028017910714F40C9455
:10B19000343661E0F70180810E94DF7B6CE271E070
:10B1A00080E090E00E94267D0F5F1F4FE6CF66EFA4
:10B1B00077E0CE0101960E940379BE016F5F7F4F59
:10B1C000CE018F5B9F4F0E946B77182FCE010196A7
:10B1D0000E947378112311F40C94343627E030E088
:10B1E00046E050E06AEF70E1CE0101960E941779C7
:10B1F000BE016F5F7F4F8CED90E10E943A78CE01E7
:10B2000001960E9473788CED90E10E94D276672BB4
:10B2100071F41092110C6AEF70E1CE0101960E9458
:10B22000FB78CE0101960E941A1B0C943D4381E0ED
:10B230008093110CF0CFFCE0FA1508F419CB2DCB5C
:10B240004F925F926F927F928F929F92AF92BF9236
:10B25000CF92DF92EF92FF920F931F93CF93DF93E2
:10B26000CDB7DEB72C970FB6F894DEBF0FBECDBFBB
:10B2700067E370E08091790290917A020E94610800
:10B2800084E1482E512C612C712CD12CC12CAFEFB4
:10B29000CA1ADA0AC301B2010E94267DE09079023F
:10B2A000F0907A0267E370E0C7010E9461088C01A8
:10B2B000B3E0CB16D10434F08EE1C816D10444F4C7
:10B2C000012B51F094E1490E511C611C711CDFCF20
:10B2D0000115110509F0AEC08BE0E816F10409F084
:10B2E0008EC080902F1390903013A0903113B090A7
:10B2F000321380912B1390912C13A0912D13B091A8
:10B300002E1389879A87AB87BC8764E670E080E05C
:10B3100090E00E94267D60EC73E0CE0101960E94D1
:10B32000F378CE0101960E94DF28CE0101960E949B
:10B33000737861E082E00E94E38021E0B501A4011E
:10B34000CE0101960E947878BE016F5F7F4F8FEA31
:10B3500093E10E943F7ACE0101960E9473786FEDCF
:10B360008FEA93E10E94BF806BEB73E08FEA93E179
:10B370000E945F7A20E049855A856B857C85CE01E5
:10B3800001960E947878BE016F5F7F4F8FEA93E14C
:10B390000E943F7ACE0101960E9473786DEF77E0AC
:10B3A0008FEA93E10E94387A89829A82AB82BC82CA
:10B3B00089859A85AB85BC858D839E83AF83B8874D
:10B3C00029813A814B815C816D817E818F81988555
:10B3D0002C960FB6F894DEBF0FBECDBFDF91CF9194
:10B3E0001F910F91FF90EF90DF90CF90BF90AF90A3
:10B3F0009F908F907F906F905F904F90089596E10F
:10B40000E916F10409F46DCFACE0EA16F10409F095
:10B410007CCF80903A0B90903B0BA0903C0BB0906F
:10B420003D0B8091360B9091370BA091380BB0916A
:10B43000390B67CF0F3F9FEF1907CCF06DEA73E030
:10B44000CE0101960E94F3784AE050E070E060E09F
:10B45000CE0101960E944824CE0101960E94737885
:10B460006AE873E082EE90E10E94027832C00E3FFB
:10B47000AFEF1A07B9F16CE773E0CE0101960E94B5
:10B48000F3784AE050E070E060E0CE0101960E945F
:10B490004824CE0101960E9473786DE673E082EE37
:10B4A00090E10E940278B801CE0101960E94637675
:10B4B000BE016F5F7F4F82EE90E10E94FC77CE016C
:10B4C00001960E94737867E573E082EE90E10E9436
:10B4D000AB7719821A821B821C821D821E821F82F8
:10B4E00018866ECF6CE473E0CE0101960E94F3786B
:10B4F0004AE050E070E060E0CE0101960E944824EE
:10B50000CE0101960E9473786CE273E0ABCF2F926C
:10B510003F924F925F926F927F928F929F92AF92E3
:10B52000BF92CF92DF92EF92FF920F931F93CF9330
:10B53000DF93CDB7DEB7AC970FB6F894DEBF0FBE82
:10B54000CDBF8C0167E079E08BE191E10E945A76F2
:10B5500067E370E08091790290917A020E9461081D
:10B560001C0165EB74E0C8010E940E186FEF77E0D4
:10B57000C8010E94387A69E373E1CE0101960E9406
:10B58000FB78BE016F5F7F4FC8010E943F7ACE01FA
:10B5900001960E94737868E078E0C8010E94387ACA
:10B5A0000E94E07D28EE33E040E050E00E94CBAF07
:10B5B00029013A01CE0109960E94121D6EE078E041
:10B5C000CE0101960E940379BE01675F7F4FCE01D5
:10B5D00001960E949A77BC01CE010F960E94FB78DB
:10B5E000BE01615F7F4FC8010E943F7ACE010F9676
:10B5F0000E947378CE0101960E947378CE0109965D
:10B600000E947378C301B20120E13EE040E050E0C7
:10B610000E94EDAF4B015C01B901CE0187960E94FB
:10B62000D0184CE3C42ED12CE12CF12CC501B4016F
:10B63000A70196010E94EDAFB901CE0109960E94C3
:10B64000D0186FED76E0CE0101960E940379BE011D
:10B65000675F7F4FCE0101960E949A77BC01CE01B1
:10B6600087960E94FC77CE0101960E947378CE01E6
:10B6700009960E947378C301B201A70196010E9446
:10B68000EDAFCE0109960E94D0186FED76E0CE01A5
:10B6900001960E940379BE01675F7F4FCE0101963C
:10B6A0000E949A77BC01CE0187960E94FC77CE015A
:10B6B00001960E947378CE0109960E94737868E122
:10B6C00078E0CE0101960E940379BE01695D7F4F4B
:10B6D000CE0101960E949A776BE178E00E9486770E
:10B6E000BC01CE0109960E94FB78BE01675F7F4FC7
:10B6F000C8010E943F7ACE0109960E947378CE015C
:10B7000001960E94737869E278E0C8010E94387A55
:10B71000CE0101960E94BF75B801CE0101960E942C
:10B72000CA7964E278E0C8010E94267A89DD29831B
:10B730003A834B835C836D837E838F8398874981B3
:10B740005A816B817C8121E0CE0109960E94787834
:10B75000BE01675F7F4FCE010F960E94FB7861E3C9
:10B7600078E0CE010F960E948677BC018BE191E1D3
:10B770000E942578CE010F960E947378CE0109961B
:10B780000E94737868E378E0CE0109960E940379FD
:10B790006BE171E1CE0109960E949A77BC01CE015E
:10B7A0000F960E94FB78BE01615F7F4FC8010E9427
:10B7B0003F7ACE010F960E947378CE0109960E94BF
:10B7C00073784D815E816F81788521E0CE01099685
:10B7D0000E947878BE01675F7F4F8BE191E10E9404
:10B7E0003A78CE0109960E9473786AE478E0CE0137
:10B7F00009960E9403796BE171E1CE0109960E94DE
:10B800009A776BE578E00E948677BC01CE010F96AF
:10B810000E94FB78BE01615F7F4FC8010E943F7AA2
:10B82000CE010F960E947378CE0109960E9473781C
:10B8300040917E0C50917F0C6091800C7091810C36
:10B8400022E0CE010F960E94787862E678E0CE0181
:10B8500009960E940379BE01615F7F4FCE01099670
:10B860000E949A7764E778E00E948677BC01CE0157
:10B8700045960E94FB78BE016B5E7F4FC8010E9417
:10B880003F7ACE0145960E947378CE0109960E94B8
:10B890007378CE010F960E94737840917A0C509184
:10B8A0007B0C60917C0C70917D0C22E0CE010F9698
:10B8B0000E9478786DE778E0CE0109960E940379BE
:10B8C000BE01615F7F4FCE0109960E949A7764E7BF
:10B8D00078E00E948677BC01CE0145960E94FB78F5
:10B8E000BE016B5E7F4FC8010E943F7ACE01459634
:10B8F0000E947378CE0109960E947378CE010F964C
:10B900000E94737886EF28168FEF38062CF460E9D2
:10B9100074E0C8010E940E1860E774E0C8010E943C
:10B920000E1828EAC22E22E0D22EEE24E394F12C47
:10B93000E2E0CE0ED11C8091AE029091AF028E1546
:10B940009F050CF468C0B701CE014B960E94637648
:10B9500069E977E0CE0145960E940379BE01655EF4
:10B960007F4FCE0145960E949A776BEF75E00E945B
:10B970008677BC01CE0181960E94FB78BE016F5D87
:10B980007F4FC8010E943F7AB70183E0660F771F9F
:10B990008A95E1F76B5E7D4ECE010F960E9403798A
:10B9A000BE01615F7F4FC8010E943F7A6BE878E07B
:10B9B000C8010E94387AF60160817181660F771F95
:10B9C000660F771F635F7D4ECE0109960E94037953
:10B9D000BE01675F7F4FC8010E943F7A60E978E04F
:10B9E000C8010E94387ACE0109960E947378CE0170
:10B9F0000F960E947378CE0181960E947378CE01D3
:10BA000045960E947378CE014B960E947378FFEFA3
:10BA1000EF1AFF0A8DCFCE0187960E947378AC96FD
:10BA20000FB6F894DEBF0FBECDBFDF91CF911F914F
:10BA30000F91FF90EF90DF90CF90BF90AF909F90CD
:10BA40008F907F906F905F904F903F902F900895D0
:10BA50002F923F924F925F926F927F928F929F921E
:10BA6000AF92BF92CF92DF92EF92FF920F931F930C
:10BA7000CF93DF93CDB7DEB7CA52D1400FB6F8945B
:10BA8000DEBF0FBECDBFCB5DDE4F59834883C552AD
:10BA9000D1402091780C3091790C2F5F3F4F30933B
:10BAA000790C2093780C2091770C21110EC38B0117
:10BAB0006C0181E08093770C1092790C1092780CD5
:10BAC00067E079E0CE01875E9E4F0E94037967E0D0
:10BAD00079E0CE01815E9E4F0E9403798091AE0293
:10BAE0009091AF028230910594F0209145023091FF
:10BAF00046023093AB022093AA02029741F0809154
:10BB00004702909148029093AD028093AC0250E0BE
:10BB100040E065E978E0C6010E945A18013011053D
:10BB200009F0C9C267E079E08BE491E10E945A769E
:10BB30007E0121E8E20EF11CC701880F991F880FD2
:10BB4000991FFC01E35FFD4EC75DDE4FF983E8837B
:10BB5000C952D140312C212C3AE0832E912CA12CBA
:10BB6000B12C44E6442E512C612C712CCB5DDE4F60
:10BB7000E881F981C552D1408081882309F415C23A
:10BB8000A701BE016F5F7F4FCE018B5D9E4F0E946C
:10BB9000C174049759F3BE016F5F7F4FCE018F5F71
:10BBA0009E4F0E940379BE016F5F7E4FCE01875E7C
:10BBB0009E4F0E943A78CE018F5F9E4F0E9473780D
:10BBC000B701CE018F5F9E4F0E940379BE016F5F68
:10BBD0007E4FCE01815E9E4F0E943A78CE018F5FEC
:10BBE0009E4F0E9473788091110C8823A1F1BE01B1
:10BBF000675E7E4FCE018F5F9E4F0E94FB786EEF97
:10BC000075E0CE018F5F9E4F0E948677BC01CE010A
:10BC1000895F9E4F0E94FB78CE01895F9E4F0E94F4
:10BC2000C617CE01895F9E4F0E947378CE018F5F49
:10BC30009E4F0E947378B701CE018F5F9E4F0E9486
:10BC40000379CE018F5F9E4F0E94AF17CE018F5FA9
:10BC50009E4F0E947378C35EDE4F88819981CD51DB
:10BC6000D140049708F0E0C070E060E0CE01875E4C
:10BC70009E4F0E943A77823531F0843521F08D7FD6
:10BC8000843409F0D1C041E050E0BE01675E7E4FD0
:10BC9000CE018F5F9E4F0E943108CE018F5F9E4F75
:10BCA0000E94D2768B016130710521F400911B1343
:10BCB00010911C130330110521F400911D131091F4
:10BCC0001E13101611060CF0A9C08091AE029091BF
:10BCD000AF02801791070CF4A1C070E060E0CE01C4
:10BCE000875E9E4F0E943A77823509F0BFC0C70138
:10BCF0000E94E9A9892B39F4F801EE0FFF1FE855DE
:10BD0000FD4F11821082C7010E94E9A9813091057F
:10BD1000A1F5F801EE0FFF1FE855FD4F91838083D9
:10BD20009801220F331F220F331FC95DDE4F398365
:10BD30002883C752D140F901E456FD4F808191819B
:10BD4000A281B381181619061A061B0644F00730A3
:10BD500011050CF086C040825182628273820E947B
:10BD60005F81C95DDE4FE881F981C752D140E15B57
:10BD7000FD4F6083718382839383C75DDE4F68814B
:10BD80007981C952D140CE018D5E9E4F0E940379C8
:10BD9000B801E3E0660F771FEA95E1F76B5E7D4E31
:10BDA000CE01835F9E4F0E9403796BE471E1CE0167
:10BDB000895F9E4F0E94FB78BE01635F7E4FCE017C
:10BDC000895F9E4F0E949A776EEA78E00E9486779C
:10BDD000BE016F5F7E4F0E949A776EEF75E00E9402
:10BDE0008677BE016D5E7E4F0E949A776BEF75E09D
:10BDF0000E948677BC018BE491E10E942578CE01F8
:10BE0000895F9E4F0E947378CE01835F9E4F0E9490
:10BE10007378CE018D5E9E4F0E947378CE018F5F46
:10BE20009E4F0E947378A2CEFBE02F1631040CF0D7
:10BE30009DCEF6E0F29D8001F39D100D1124BE0110
:10BE40006F5F7F4FC8018D569E4E0E94BA76B70134
:10BE5000C8018F5A9E4E0E94BA762FEF221A320ADC
:10BE600085CE80829182A282B38279CF863409F016
:10BE700074C0C7010E94E9A9892B39F4F801EE0FBB
:10BE8000FF1FE75BFD4F11821082C7010E94E9A9E5
:10BE90008130910539F4F801EE0FFF1FE75BFD4F8C
:10BEA00091838083C801880F991F880F991FC95DEE
:10BEB000DE4F99838883C752D140FC01E456FD4F81
:10BEC00080819181A281B381181619061A061B067A
:10BED0003CF007301105E4F54082518262827382A2
:10BEE0000E945F81C95DDE4FE881F981C752D14070
:10BEF000E15BFD4F6083718382839383C75DDE4F77
:10BF000068817981C952D140CE018D5E9E4F0E94D9
:10BF10000379B80143E0660F771F4A95E1F76B5E3E
:10BF20007D4ECE01835F9E4F0E9403796BE471E1E9
:10BF3000CE01895F9E4F0E94FB78BE01635F7E4FFA
:10BF4000CE01895F9E4F0E949A7761EB78E03ECFE9
:10BF500080829182A282B382C3CF8434C1F4C701AC
:10BF60000E9406AA000F111F000F111FF801E95CC3
:10BF7000FD4F60837183828393830E945F81015BA5
:10BF80001D4FF801608371838283938347CF84358B
:10BF900009F044CFC7010E9406AA000F111F000F2D
:10BFA000111FF801E456FD4FE4CF81E08093970C18
:10BFB0008091980C882311F0C601A9DA8091980C21
:10BFC000882329F061E374E0C6010E940E181092E4
:10BFD000770C80914F1190915011892B09F46BC00F
:10BFE000CE01895F9E4F0E94121D6FE979E0CE015C
:10BFF0008F5F9E4F0E940379BE01695F7E4FCE0125
:10C000008F5F9E4F0E949A776BEF75E00E94867754
:10C010006BE471E10E949A77BC018BE491E10E948C
:10C020002578CE018F5F9E4F0E947378CE01895F85
:10C030009E4F0E9473786BE471E1CE018F5F9E4F3B
:10C040000E94FB78AE014F5F5E4F62E070E08CE6CD
:10C0500092E00E94A822182FCE018F5F9E4F0E946F
:10C0600073786BE471E1CE018F5F9E4F112309F469
:10C0700046C00E94FB7861EE77E0CE018F5F9E4F55
:10C080000E94867763E371E10E949A77BC01CE013A
:10C09000895F9E4F0E94FB78CE01895F9E4F0E9470
:10C0A000AF17CE01895F9E4F0E947378CE018F5FDC
:10C0B0009E4F0E947378CE01815E9E4F0E947378DE
:10C0C000CE01875E9E4F0E947378C65DDE4F0FB62D
:10C0D000F894DEBF0FBECDBFDF91CF911F910F91BE
:10C0E000FF90EF90DF90CF90BF90AF909F908F9098
:10C0F0007F906F905F904F903F902F9008950E9497
:10C10000FB7861EE77E0CE018F5F9E4F0E948677CD
:10C110006DE271E1B9CFFF920F931F93CF93DF933D
:10C12000EC018B018091780C9091790C01969093A1
:10C13000790C8093780C2091770C222339F06AE0F7
:10C1400070E00E943AB118161906ECF0FF24F3943F
:10C15000F092770C1092790C1092780C50E040E03D
:10C1600065E978E0CE010E945A180230110589F085
:10C17000CE01CDD9F092990C61E374E0CE010E941A
:10C180000E181092770CDF91CF911F910F91FF90B5
:10C19000089560E974E0CE010E940E18EDCFAF92D1
:10C1A000BF92CF92DF92EF92FF920F931F93CF93A4
:10C1B000DF93CDB7DEB7A0970FB6F894DEBF0FBE02
:10C1C000CDBF67E079E085E491E10E945A7667E0AF
:10C1D00079E089E391E10E945A7653E4E52E52E03A
:10C1E000F52E68EAC62E62E0D62E7BE3A72E72E01B
:10C1F000B72E01E010E08091AE029091AF0280175F
:10C2000091070CF482C0F50181919191A191B191B6
:10C210005F01892B8A2B8B2B19F5F6018281938183
:10C22000F7012281338182179307D1F0880F991F7C
:10C23000FC01E35FF34FD801AA0FBB1FAE5EB34F03
:10C2400060818C910E94DF7BF60182819381F701EE
:10C250009383828364E670E080E090E00E94267D14
:10C26000F70162817381CE0145960E946376B80121
:10C27000CE010F960E946376B80123E0660F771F08
:10C280002A95E1F76B5E7D4ECE0109960E940379F7
:10C290006BEF75E0CE0101960E940379BE01675FE6
:10C2A0007F4FCE0101960E949A776EEA78E00E9455
:10C2B0008677BE01615F7F4F0E949A776EEF75E0CF
:10C2C0000E948677BE016B5E7F4F0E949A77BC0109
:10C2D00085E491E10E94FC77CE0101960E9473787B
:10C2E000CE0109960E947378CE010F960E94737852
:10C2F000CE0145960E9473780F5F1F4FF2E0EF0E5C
:10C30000F11C82E0C80ED11C76CFE0911B13F09196
:10C310001C13EE0FFF1FED5BFD4F60817181CE019D
:10C3200001960E94637646E050E0BE016F5F7F4F4A
:10C33000CE0109960E948918BE01675F7F4F89E38D
:10C3400091E10E94FC77CE0109960E947378CE019C
:10C3500001960E947378E0911D13F0911E13EE0F69
:10C36000FF1FED5BFD4F60817181CE0101960E9440
:10C37000637646E050E0BE016F5F7F4FCE010996C5
:10C380000E948918BE01675F7F4F89E391E10E9497
:10C39000FC77CE0109960E947378CE0101960E9427
:10C3A00073786BEF75E0CE0145960E9403790E9489
:10C3B000E07D28EE33E040E050E00E94CBAF690121
:10C3C0007A0167E079E0CE014B960E94037967E03D
:10C3D00079E08BE491E10E945A76CE0101960E94A9
:10C3E000121D44E150E0BE016F5F7F4FCE01099600
:10C3F0000E948918BE01675F7F4F8BE491E10E9424
:10C400003A78CE0109960E947378CE0101960E9477
:10C4100073782AE0B701A601CE0109960E94A77899
:10C4200048E050E0BE01675F7F4FCE010F960E944B
:10C4300089186BE471E1CE0101960E94FB78BE0180
:10C44000615F7F4FCE0101960E949A77BC018FE316
:10C4500091E10E942578CE0101960E947378CE0169
:10C460000F960E947378CE0109960E9473782AE095
:10C47000B701A601CE0109960E94A77865EB78E086
:10C48000CE0101960E940379BE01675F7F4FCE0106
:10C4900001960E949A77BE016B5E7F4F0E949A7749
:10C4A000BC018BE491E10E94FC77CE0101960E94D1
:10C4B0007378CE0109960E94737840917E0C50915A
:10C4C0007F0C6091800C7091810C21E0CE0101966F
:10C4D0000E947878BE016F5F7F4FCE014B960E941D
:10C4E0003A78CE0101960E9473786CEB78E0CE0129
:10C4F00001960E940379BE01655E7F4FCE010196D1
:10C500000E949A77BE016B5E7F4F0E949A77BC01B2
:10C510008BE491E10E94FC77CE0101960E94737832
:10C52000BE01655E7F4FCE0101960E94FB7846E01A
:10C5300050E0BE016F5F7F4FCE0109960E948918BF
:10C54000BE01675F7F4F8FE391E10E94FC77CE01D0
:10C5500009960E947378CE0101960E9473784091EB
:10C560007A0C50917B0C60917C0C70917D0C21E0D9
:10C57000CE0101960E947878BE016F5F7F4FCE0199
:10C580004B960E943A78CE0101960E9473786AEC2D
:10C5900078E0CE0101960E940379BE01655E7F4F6F
:10C5A000CE0101960E949A77BE016B5E7F4F0E947A
:10C5B0009A77BC018BE491E10E94FC77CE01019651
:10C5C0000E947378BE01655E7F4FCE0101960E9486
:10C5D000FB7846E050E0BE016F5F7F4FCE010996C9
:10C5E0000E948918BE01675F7F4F8FE391E10E942F
:10C5F000FC77CE0109960E947378CE0101960E94C5
:10C60000737880915C0C90915D0C892B61F067E3ED
:10C6100070E08091790290917A020E946108909373
:10C620005D0C80935C0C80915C0C90915D0C892B6F
:10C6300009F0EEC00E94205929833A834B835C8322
:10C640006D837E838F83988749815A816B817C813A
:10C6500021E0CE0109960E947878BE01675F7F4F86
:10C66000CE014B960E943A78CE0109960E947378CB
:10C6700064ED78E0CE0109960E940379BE01655E03
:10C680007F4FCE0109960E949A77BE016B5E7F4F65
:10C690000E949A77BC018BE491E10E94FC77CE0165
:10C6A00009960E947378BE01655E7F4FCE010996A0
:10C6B0000E94FB7846E050E0BE01675F7F4FCE01ED
:10C6C0000F960E948918BE01615F7F4F8FE391E151
:10C6D0000E94FC77CE010F960E947378CE010996D6
:10C6E0000E9473784D815E816F81788521E0CE0153
:10C6F00009960E947878BE01675F7F4FCE014B9606
:10C700000E943A78CE0109960E9473786FED78E026
:10C71000CE0109960E940379BE01655E7F4FCE016E
:10C7200009960E949A77BE016B5E7F4F0E949A77AE
:10C73000BC018BE491E10E94FC77CE0109960E9436
:10C740007378BE01655E7F4FCE0109960E94FB782B
:10C7500046E050E0BE01675F7F4FCE010F960E941A
:10C760008918BE01615F7F4F8FE391E10E94FC77E2
:10C77000CE010F960E947378CE0109960E947378BD
:10C7800065E471E18BE491E10E94FC776BEF75E069
:10C79000CE0101960E94037969E371E1CE01019611
:10C7A0000E949A77BC018FE391E10E94FC77CE0151
:10C7B00001960E9473786FE371E1CE0101960E94A9
:10C7C000FB78CE0101960E94AF17CE0101960E9420
:10C7D00073786AE070E080E090E00E94267DCE01F0
:10C7E0004B960E947378CE0145960E947378A0966E
:10C7F0000FB6F894DEBF0FBECDBFDF91CF911F9172
:10C800000F91FF90EF90DF90CF90BF90AF90089581
:10C8100065EE78E08BE491E10E94F37764EF78E0D5
:10C820008FE391E10E94F3776BEF78E08BE491E185
:10C830000E94F37764EF78E08FE391E10E94F37751
:10C840009FCFDF92EF92FF920F931F93CF93DF93CF
:10C85000CDB7DEB7C451D1400FB6F894DEBF0FBEDE
:10C86000CDBFCD5EDE4F59834883C351D140209167
:10C87000780C3091790C2F5F3F4F3093790C2093D7
:10C88000780C2091770C21113EC08B017C01DD24B6
:10C89000D394D092770C1092790C1092780C67E0B8
:10C8A00079E0CE01895F9E4F0E94037967E079E0CD
:10C8B000CE01835F9E4F0E94037950E040E065E91E
:10C8C00078E0C7010E945A180130110591F467E021
:10C8D00079E08BE491E10E945A76CD5EDE4FE881EB
:10C8E000F981C351D140808181111CC058DCD092A4
:10C8F000990CCE01835F9E4F0E947378CE01895FB1
:10C900009E4F0E947378CC5EDE4F0FB6F894DEBF68
:10C910000FBECDBFDF91CF911F910F91FF90EF9090
:10C92000DF900895CD5EDE4FE881F981C351D1409B
:10C930008081882309F465C0AE014F575F4FBE0167
:10C940006F5F7F4FCE018D5E9E4F0E94C174049732
:10C9500049F3BE016F5F7F4FCE018F5F9E4F0E94F4
:10C960000379BE016F5F7E4FCE01895F9E4F0E94AB
:10C970003A78CE018F5F9E4F0E947378BE016F5749
:10C980007F4FCE018F5F9E4F0E940379BE016F5F84
:10C990007E4FCE01835F9E4F0E943A78CE018F5F1B
:10C9A0009E4F0E947378BE01695F7E4F8BE491E1D8
:10C9B0000E94FC77CF5EDE4F88819981C151D140C2
:10C9C000892B09F4AFCF6EEF75E0CE018F5F9E4FDC
:10C9D0000E940379BE01635F7E4FCE018F5F9E4F41
:10C9E0000E949A776BEF75E00E948677BC018BE41A
:10C9F00091E10E94FC77CE018F5F9E4F0E94737879
:10CA000091CF6BE471E187E291E10E94257871CFCB
:10CA10002F923F924F925F926F927F928F929F924E
:10CA2000AF92BF92CF92DF92EF92FF920F931F933C
:10CA3000CF93DF93CDB7DEB7C258D1090FB6F894C4
:10CA4000DEBF0FBECDBF6C015B0188EE482E83E0D8
:10CA5000582E612C712C05E114E09BE5892E912C58
:10CA60008C0E9D1E8CE0880E911C1B019FEF291AD5
:10CA7000390AD6015996ED90FC90F70185818230F4
:10CA800008F493C082859385A485B5858F71992715
:10CA9000AA27BB27892B8A2B8B2B09F086C040E263
:10CAA00050E0BE016F5F7F4FC7010E94F38A803262
:10CAB00009F07BC08981882309F477C0853E79F32A
:10CAC0008E3269F38C8583FDEACF22961FAE1EAEAF
:10CAD00022978FE993E09FAF8EAF24961FAE2497E5
:10CAE000BE016F5F7F4FE0E080E04EE2DB019D9191
:10CAF000BD019032A1F0883049F426E730E02C0FD8
:10CB00003D1F2E0F311DD9014C93EF5F26E730E01A
:10CB10002C0F3D1F2E0F311DD9019C93EF5F8F5FAE
:10CB20008B3021F786E790E08C0F9D1F8E0F911DB3
:10CB3000FC011082D60159966D917C9121E0AE01E5
:10CB40004A585F4FCE01CE960E946F8D882369F1BF
:10CB5000BE01625C7F4FCE0181960E94D991AE01E9
:10CB60004A585F4FBE016F5D7F4FCE01855A9F4F80
:10CB70000E944692CE01855A9F4F0E942992882397
:10CB800009F4ABC0F12CFA141B042CF569E0CE01BA
:10CB900001960E94D378CE0101960E94C617CE015D
:10CBA00001960E947378F394EECF6F961FAE1EAE7F
:10CBB0006F97A3964CAE5DAE6EAE7FAEA3976D96AB
:10CBC0001FAF0EAF6D97E6961FAE1EAEE697A89606
:10CBD0001FAEA897CFCFB401CE0101960E94037972
:10CBE000CE0101960E94C617CE0101960E9473786D
:10CBF000E696EEADFFADE697309709F446C0858125
:10CC0000823008F442C062E574E0CE0101960E94D1
:10CC10000379CE0101960E94AF17CE0101960E94C2
:10CC200073786F968EAD9FAD6F979C838B83A39621
:10CC30008CAD9DADAEADBFADA3978D839E83AF830D
:10CC4000B887A7968CAD9DADAEADBFADA7978987D0
:10CC50009A87AB87BC871A8309838DE0F401DE01D4
:10CC60001D9601900D928A95E1F7E6968EAD9FADE7
:10CC7000E6979B8F8A8FB101CE010196C9DECE0166
:10CC8000855A9F4F0E943592F4CE65E079E0CE013F
:10CC900001960E940379CE0101960E94C617CE012B
:10CCA00001960E947378E696EEADFFADE69740E000
:10CCB00050E0BA01309721F043895489658976891B
:10CCC000CE0101960E948E76CE0101960E94AF178A
:10CCD000CE0101960E947378D2CFCE57DF4F0FB6A8
:10CCE000F894DEBF0FBECDBFDF91CF911F910F91A2
:10CCF000FF90EF90DF90CF90BF90AF909F908F907C
:10CD00007F906F905F904F903F902F9008952F925B
:10CD10003F924F925F926F927F928F929F92AF92CB
:10CD2000BF92CF92DF92EF92FF920F931F93CF9318
:10CD3000DF93CDB7DEB7CB54D1090FB6F894DEBF81
:10CD40000FBECDBF40E052EC61E070E089EA9EE0AA
:10CD50000E94517440E855E260E070E08CE09EE093
:10CD60000E94517440E855E260E070E08FE69DE07B
:10CD70000E94517440E855E260E070E082ED9CE072
:10CD80000E94517461E088E00E94F57C61E089E0D6
:10CD90000E94F57C60E08AE30E94F57C61E088E017
:10CDA0000E94DF7B60E089E00E94DF7B61E08AE037
:10CDB0000E94F57C61E08BE00E94F57C60E08BE3F3
:10CDC0000E94F57C61E08AE00E94DF7B60E08BE0FE
:10CDD0000E94DF7B0E940D7C01E00093CE0C12E5E7
:10CDE0001093D00C1092CF0C1092D10C80EF90E0E9
:10CDF0000E944D7485E590E00E944D7481E00E9490
:10CE0000F0730093CE0C1093D00C1092CF0C1092B4
:10CE1000D10C8BEF90E00E944D7490E080E00E9476
:10CE20004D7481E00E94F07384EF91E09093910241
:10CE30008093900268EE73E080E090E00E94267D8F
:10CE400089EA9EE00E94A270F82E0AE010E0F1103C
:10CE50000BC089EA9EE00E94A270F82E6EE170E09D
:10CE600080E090E00E94267D0150110981F78091B9
:10CE700090029091910201E012E168019C01215021
:10CE800032415901C5018C0D9D1D0E94A6AFF601CE
:10CE900081936F01FBE2CF16F3E1DF0699F7609112
:10CEA0001B1370911C13072E000C880B990B0E940A
:10CEB00093AE9B01AC010E942AB1882331F081E03E
:10CEC00090E090931C1380931B1360911D1370913D
:10CED0001E13072E000C880B990B0E9493AE9B012A
:10CEE000AC010E942AB1882331F082E090E0909357
:10CEF0001E1380931D1325E7F216B1F060911713EE
:10CF0000709118138091191390911A130E9493AE87
:10CF10009B01AC010E942AB1811106C080910112CF
:10CF2000909102128197E8F08DB79EB78A52914096
:10CF30000FB6F8949EBF0FBE8DBFADB7BEB71196AA
:10CF40008AE291E0E1E0F2E101900D920197E1F7D0
:10CF50000E9405210FB6F894DEBF0FBECDBF85E756
:10CF6000F82E2DB73EB72A5231400FB6F8943EBF87
:10CF70000FBE2DBFADB7BEB711968AE291E0E1E0DA
:10CF8000F2E101900D920197E1F70E9406190FB6A8
:10CF9000F894DEBF0FBECDBF95E7F91619F0E3E7B1
:10CFA000FE121BC02DB73EB72A5231400FB6F8947F
:10CFB0003EBF0FBE2DBFADB7BEB711968AE291E05E
:10CFC000E1E0F2E101900D920197E1F70E94112951
:10CFD0000FB6F894DEBF0FBECDBF61E579E083E305
:10CFE00091E10E9402786BE379E08DE291E10E9489
:10CFF00002780E940D7C68E079E089EA9EE00E9458
:10D00000267AD12CC12CB7E2EB2EBB24B394B0927C
:10D01000CE0CE092D00C1092CF0C1092D10C81E08B
:10D020000E94F07381116FC164E179E089EA9EE0AA
:10D030000E94387A8E2D0E94B579E092B31360E396
:10D0400079E089EA9EE00E94387A8E2D0E94B579B7
:10D050009FEFC91AD90AE394E0E4EE12D8CF65E64F
:10D0600079E0CD2811F06BE779E089EA9EE00E9433
:10D07000267A0E940D7C1092B4138091B8138230EE
:10D0800018F098E09093B4139091B913992339F064
:10D09000813029F48091B41384608093B41362E3E7
:10D0A00070E080E090E00E94267D6091BA138FEAE4
:10D0B00093E10E94968068EE73E080E090E00E9429
:10D0C000267D60E38FEA93E10E94A9807BE4C72E6E
:10D0D00076E4D72EC6010197F1F760E38FEA93E17A
:10D0E0000E94A980C6010197F1F760E38FEA93E1FE
:10D0F0000E94A98083E592E00197F1F760E28FEA50
:10D1000093E10E94A9808091B41380620E94D48030
:10D1100084E08093B5138CE00E94D48081E00E946B
:10D12000D480EBE3CE2EEFE1DE2EC6010197F1F7BE
:10D1300082E08093B61386E00E94D48082E00E9451
:10D14000D480C6010197F1F780E40E94D480F8E80A
:10D15000CF2EF2E0DF2EA0E9AA2EA2E0BA2EF60131
:10D1600061916F018FEA93E10E94BF80AC14BD040E
:10D17000B1F70E943D080E94210864E670E080E05B
:10D1800090E00E94267D63E279E0CE0101960E9444
:10D19000F378CE0101960E94AF17CE0101960E944E
:10D1A000737861E085E30E94F57C61E085E30E948D
:10D1B000DF7B61E08AE00E94F57C61E08AE00E940A
:10D1C000DF7B61E084E00E94F57C61E084E00E9406
:10D1D000DF7B61E089E30E94F57C69E370E08EE328
:10D1E00090E10E945B7F68EC70E080E090E00E943C
:10D1F000267D8FEF9FEF90939B0280939A029093EE
:10D2000099028093980268EE73E080E090E00E94BB
:10D21000267D62E179E0CE0101960E94F3784AE032
:10D2200050E06FEF7FEFCE0101960E944824CE01BF
:10D2300001960E94737810925F0F10925D0F10920A
:10D240005A0F1092590F84E08093580F0E94E07D8E
:10D250006B0161E08091580F0E94F57C61E0809144
:10D26000580F0E94DF7B0E943A1582E58093520F8F
:10D270001092530F8091520F9091530F0E940E0BFA
:10D280006AE0E62E8FEF0E94AC0AEA94E110FACF32
:10D2900084E59FE00E948D8420E030E0A90160E0F9
:10D2A00084E59FE00E94CC84E82E80935E0FF1E03D
:10D2B0008F17B1F10E94E07D6C197D09613D7740C7
:10D2C00058F381E08093590F84E59FE00E94A38486
:10D2D00064E079E0CE0101960E94F378CE010196D8
:10D2E0000E94AF17CE0101960E94737863EF78E039
:10D2F000CE0101960E94F3786AE070E0CE010196BB
:10D300000E940F8128C1843009F0A5CE6AE479E03B
:10D3100089EA9EE00E94387A8E2D0E94B5799BCED4
:10D320002AEA31E040E050E068E084E59FE00E94B6
:10D33000CC8482FF2AC0E0925F0F80915F0F812C26
:10D34000912C5401823029F4812C912CA12C40E4A1
:10D35000B42E20E030E0A90167E384E59FE00E945D
:10D36000CC84A501940169E284E59FE00E94CC840D
:10D3700080935E0F8823D1F00E94E07D6C197D09B7
:10D38000613D774030F388E09DCF54E0E52E0E9468
:10D39000B18480935E0FEA94E110F9CF8A3A11F0DC
:10D3A00082E090CF82E080935F0FC7CF80915F0FC4
:10D3B0008230D1F420E030E0A9016AE384E59FE007
:10D3C0000E94CC84882311F086E07CCF0E94B18437
:10D3D000807C803C19F483E080935F0F0E94B184CD
:10D3E0000E94B1840E94B18484E59FE00E94A384DE
:10D3F00080E58093520F1092530F81E00E94B78610
:10D40000882309F463C18091830F811161CF8091DA
:10D41000770F803109F061C182E08093830F109211
:10D42000950F1092960F1092970F1092980F80916F
:10D43000780F9091790FB0E0A0E035E0880F991F48
:10D44000AA1FBB1F3A95D1F78093910F9093920F2B
:10D45000A093930FB093940F80E69FE090939A0F60
:10D460008093990F81E08093820F1092840F109225
:10D47000850F1092860F1092870F1092880F1092CE
:10D48000890F10928A0F10928B0F10928C0F1092AE
:10D490008D0F10928E0F10928F0F1092900F67EEDB
:10D4A00078E0CE0101960E94F378CE0101960E94A9
:10D4B000AF17CE0101960E94737841E062E574E0F7
:10D4C000CE0101960E947B92BE016F5F7F4F88E77D
:10D4D00093E10E94DD1780917A1390917B139C83D6
:10D4E0008B8380917C1390917D13A0917E13B091DA
:10D4F0007F138D839E83AF83B88780918013909133
:10D500008113A0918213B091831389879A87AB8787
:10D51000BC8785E194E09A8389838DE0E4E8F3E1B8
:10D52000DE011D9601900D928A95E1F7809191138D
:10D53000909192139B8F8A8F70E060E0CE010196EC
:10D5400067DA61EE78E0CE0101960E94F378CE01B1
:10D5500001960E94AF17CE0101960E94737868EE83
:10D5600073E080E090E00E94267D43E164ED72E08C
:10D57000CE0101960E947B92BE016F5F7F4F83E9CF
:10D5800093E10E94DD1769EA78E081E291E10E946F
:10D5900002786EE978E081E291E10E94AB7783E95D
:10D5A00093E10E942992882309F4B6C068EB7FE8D2
:10D5B00084ED92E00E940B8F811122C062E879E035
:10D5C000CE0101960E940379CE0101960E94C617F2
:10D5D000CE0101960E94737864ED72E0CE0101964F
:10D5E0000E940379CE0101960E94AF17CE010196E9
:10D5F0000E94737861E271E183E993E10E944D7AC0
:10D6000083E993E10E94359266E970E080E090E062
:10D610000E94267D64E979E0CE0101960E9403799B
:10D62000CE0101960E94AF17CE0101960E94737839
:10D630001092950C6BE778E0CE0101960E94F3788A
:10D64000CE0101960E94AF17CE0101960E94737819
:10D650000E94BD955C0168EE73E080E090E00E945E
:10D66000267DD12CC12CAB2809F00AC58AE0C8164A
:10D67000D10409F4CEC2B601CE0101960E946376B0
:10D68000CE0101960E94AF17CE0101960E947378D9
:10D6900060ED77E080E090E00E94267D0E94BD95DD
:10D6A0005C0168EE73E080E090E00E94267DCE0190
:10D6B00001960E94BF75BE016F5F7F4F89EA9EE0B1
:10D6C0000E94127A9FEFC91AD90ACDCF80E00E943A
:10D6D000B786882309F4FCCD96CE803209F0F8CDC8
:10D6E00083E08093830F40917A0F50917B0F60917C
:10D6F0007C0F70917D0F4093950F5093960F609320
:10D70000970F7093980F21E93FE080E69FE00E9419
:10D71000FF888111A1CEDCCD69E878E0CE010196C9
:10D720000E94F378CE0101960E94C617CE010196A1
:10D730000E94737864ED72E06FCFF4011182108261
:10D740006DE072E1CE0188960E940379B801645EB3
:10D750007F4FCE0182960E940379B701CE014C968D
:10D760000E9463766AE979E0CE0101960E9403790E
:10D77000BE01645E7F4FCE0101960E949A776FEDE5
:10D7800076E00E948677BE016E5D7F4F0E949A7799
:10D790006EEF75E00E948677BE01685D7F4F0E9444
:10D7A0009A77BC012B968FAD2B972C969FAD2C971B
:10D7B0000E94FC77CE0101960E947378CE014C96B0
:10D7C0000E947378CE0182960E947378CE0188966B
:10D7D0000E947378F3011082118212821382F20187
:10D7E0001082118212821382C7010E948816FFEFF5
:10D7F000EF1AFF0A2A960EAD1FAD2A9767C3CE0116
:10D800004C960E94121D6EE979E0CE0101960E94AD
:10D810000379BE01645E7F4FCE0101960E949A7724
:10D820006BEF75E00E948677BE01605C7F4F0E94BF
:10D830009A77BC018BE491E10E942578CE01019694
:10D840000E947378CE014C960E947378CE010196A7
:10D850000E94121D46E150E0BE016F5F7F4FCE0176
:10D860004C960E948918BE01645E7F4FCE0182965D
:10D870000E94FB78BE01665C7F4FCE0182960E94BB
:10D880009A77BC01CE01CA960E942578CE01829675
:10D890000E947378CE014C960E947378CE01019657
:10D8A0000E9473786BE471E1CE0101960E94FB78CF
:10D8B000CE0101960E94AF17CE0101960E947378A7
:10D8C0006BE471E1CE0101960E94FB78AE014F5FDF
:10D8D0005F4F62E070E08CE692E00E94A822182F71
:10D8E000CE0101960E947378111121C06BE471E1A1
:10D8F000CE0101960E94FB7861EE77E0CE010196A1
:10D900000E9486776DE271E10E949A77BC01CE0198
:10D910004C960E94FB78CE014C960E94AF17CE0128
:10D920004C960E947378CE0101960E947378BE01D6
:10D93000665C7F4FCE0101960E94FB78AE014F5F7F
:10D940005F4F63E070E08FE592E00E94A822CE0175
:10D9500001960E947378CE01C4960E947378CE011E
:10D96000CA960E947378C6010E94737801E010E0A5
:10D9700010935E0200935D0210935C0200935B02C1
:10D9800068EA79E08CED90E10E945A7662E178E0F5
:10D99000CE0101960E94F378CE0101960E94AF1746
:10D9A000CE0101960E9473786CED70E1CE01019674
:10D9B0000E94FB7862E070E0CE0101960E943B2C51
:10D9C000CE0101960E94737862E078E0CE01019664
:10D9D0000E94F378CE0101960E94DF28CE010196C5
:10D9E0000E94737861EB76E08CED90E10E945A76AC
:10D9F00061EF77E0CE0101960E94F378CE010196A7
:10DA00000E94AF17CE0101960E9473786CED70E111
:10DA1000CE0101960E94FB7863E070E0CE01019692
:10DA20000E943B2CCE0101960E94737882E090E028
:10DA300090935E0280935D0280912713909128134A
:10DA400090935C0280935B0265EE77E0CE010196D5
:10DA50000E94F378CE0101960E94DF28CE01019644
:10DA60000E94737861EB76E08CED90E10E945A762B
:10DA70006CED70E1CE0101960E94FB7863E070E0EE
:10DA8000CE0101960E943B2CCE0101960E94737834
:10DA900080912713909128139195819591099093E6
:10DAA00028138093271310935C0200935B0284EF8A
:10DAB00091E0909391028093900261E072E10E9464
:10DAC000F00764E670E080E090E00E94267D10930D
:10DAD0005E0200935D028BE890E69093B410809311
:10DAE000B3102091D510822F022E000C990B883094
:10DAF0009105C8F4FC01EE0FFF1FEE0FFF1FEB5462
:10DB0000FF4E4CEA59E0518340832F5F2093D5109C
:10DB1000880F991F880F991FFC01E954FF4E88E276
:10DB20009DE5918380832091D510822F022E000CD9
:10DB3000990B88309105C8F4FC01EE0FFF1FEE0F22
:10DB4000FF1FEB54FF4E42EB59E0518340832F5FA0
:10DB50002093D510880F991F880F991FFC01E95455
:10DB6000FF4E81E294E69183808385E490E10E94F8
:10DB7000B61263ED77E0CE0101960E94F378CE01F4
:10DB800001960E94AF17CE0101960E9473780E9401
:10DB90005F8160936B0C70936C0C80936D0C909311
:10DBA0006E0C1092770C0E94C4260E945F816093D5
:10DBB0008E0C70938F0C8093900C9093910C8091AD
:10DBC00000138093970C882351F00E945F8160932B
:10DBD000860C7093870C8093880C9093890CC55B9E
:10DBE000DF4F0FB6F894DEBF0FBECDBFDF91CF91F0
:10DBF0001F910F91FF90EF90DF90CF90BF90AF906B
:10DC00009F908F907F906F905F904F903F902F905C
:10DC100008956FE678E0CE0101960E94F378CE0178
:10DC200001960E94AF17CE0101960E94737868EEAC
:10DC300073E080E090E00E94267D68EB7FE88BE750
:10DC400092E00E940B8F882331F063EE7FE88BE730
:10DC500092E00E940B8F66E970E080E090E00E9405
:10DC6000267D43E16BE772E0CE0101960E947B9234
:10DC7000BE016F5F7F4F83E993E10E94DD1781E072
:10DC80008093950CCE0101967AD7BE016F5F7F4FCE
:10DC900083E993E10E94127A83E993E10E9435922D
:10DCA00062E370E080E090E00E94267D1092950C87
:10DCB0000E94DE2468EE73E080E090E00E94267D02
:10DCC0000E94022724E6C22ED12CF1100AC089EA54
:10DCD0009EE038D2F82E64E170E080E090E00E948F
:10DCE000267DE1E0CE1AD10881F762E578E0CE0129
:10DCF00001960E94F378CE0101960E94DF28CE01A2
:10DD000001960E947378F2E781E0FF1280E00E94A2
:10DD10005E0768E478E08BE491E10E940278CE012E
:10DD200001960E94121DBE016F5F7F4F8BE491E14F
:10DD30000E94FC77CE0101960E94737865E378E03B
:10DD40008BE491E10E94AB7763E278E0CE0101962B
:10DD50000E94F378CE0101960E94DF28CE01019641
:10DD60000E94737867E370E08091790290917A0263
:10DD70000E94610890935D0C80935C0C6BE471E1F0
:10DD8000CE0101960E94FB78AE014F5F5F4F62E0CB
:10DD900070E08CE692E00E94A822F82ECE01019657
:10DDA0000E947378F11021C06BE471E1CE010196FD
:10DDB0000E94FB7861EE77E0CE0101960E948677A3
:10DDC0006DE271E10E949A77BC01CE014C960E94EF
:10DDD000FB78CE014C960E94AF17CE014C960E9464
:10DDE0007378CE0101960E9473786BE471E1CE01E5
:10DDF00001960E94FB78AE014F5F5F4F63E070E0D9
:10DE00008FE592E00E94A822F82ECE0101960E9492
:10DE10007378F11021C06BE471E1CE0101960E948C
:10DE2000FB7861EE77E0CE0101960E9486776DE285
:10DE300071E10E949A77BC01CE014C960E94FB785A
:10DE4000CE014C960E94AF17CE014C960E9473787B
:10DE5000CE0101960E94737868EE73E080E090E056
:10DE60000E94267D6E0120E4C20ED11C67E079E09D
:10DE7000C6010E94037967E079E0CE01CA960E944C
:10DE8000037967E079E0CE01C4960E94037980911E
:10DE9000AE029091AF0228969FAF8EAF2897A8EA66
:10DEA0008A2EA2E09A2EBCE9AB2EB2E0BB2E8FE404
:10DEB000282E82E0382E21013501EE24E394F12C46
:10DEC0002B96CFAE2B972C96DFAE2C9792E0890E37
:10DED000911CF80138962A96FFAFEEAF2A97F4E02E
:10DEE0006F0E711C24E0420E511C28968EAD9FAD22
:10DEF00028978E159F050CF020CC73E4872E72E0D6
:10DF0000972EE9E4EE2EE2E0FE2E01E010E0F8EEBE
:10DF10004F2EF3E05F2E612C712C22E0820E911CBB
:10DF200034E0A30EB11C82E0E80EF11C94E0290E4F
:10DF3000311C8091AE029091AF02801791070CF4D2
:10DF40005ECCF40160817181CE018896BCD642E03E
:10DF500050E0BE01685D7F4FCE018E960E94891809
:10DF6000B801CE014C96AFD642E050E0BE01645EEF
:10DF70007F4FCE0182960E94891869E977E0CE0131
:10DF800001960E940379BE016E5D7F4FCE0101961E
:10DF9000D1D7BE01625D7F4FCDD7BC01CE01C49603
:10DFA0000E942578CE0101960E947378CE01829658
:10DFB0000E947378CE014C960E947378CE018E96A3
:10DFC0000E947378CE0188960E947378F501608173
:10DFD000718182819381A30192010E94EDAFBA0108
:10DFE000A90120E0CE0101960E94A77848E050E008
:10DFF000BE016F5F7F4FCE014C960E948918BE0113
:10E00000645E7F4FCE01C496F7D7CE014C960E9436
:10E010007378CE0101960E947378F7016081718157
:10E02000CE01019650D643E050E0BE016F5F7F4FB6
:10E03000CE014C960E948918BE01645E7F4FCE01CE
:10E04000C496DAD7CE014C960E947378CE01019621
:10E050000E947378BE016C5C7F4FCE01CA96CCD70C
:10E06000F5011082118212821382F1011082118255
:10E0700012821382C8010E9488160F5F1F4F4DCF76
:10E0800062E678E0C8CD089508958091930C909150
:10E09000940C891B990B08950895AF92BF92CF926B
:10E0A000DF92EF92FF920F931F93CF93DF936C0158
:10E0B0007B018B01040F151FEB015E01AE18BF0839
:10E0C000C017D10759F06991D601ED91FC910190EB
:10E0D000F081E02DC6011995892B79F7C501DF91F3
:10E0E000CF911F910F91FF90EF90DF90CF90BF9055
:10E0F000AF900895FC01A089B1898C91A689B78958
:10E1000082FD0FC09C91818D8F5F8F73228D82174E
:10E1100049F0A18DAE0FBF2FB11D5D969C93818FED
:10E1200008958C910895FC01538D448D252F30E086
:10E13000842F90E0821B930B541710F0CF96089514
:10E1400001970895FC01918D828D981761F0A28D41
:10E15000AE0FBF2FB11D5D968C91928D9F5F9F7307
:10E16000928F90E008958FEF9FEF0895FC01918DBD
:10E17000828D981731F0828DE80FF11D858D90E02A
:10E1800008958FEF9FEF0895FC01918D228D892FC7
:10E1900090E0805C9F4F821B91098F7399270895AF
:10E1A00082ED9CE0F1DF21E0892B09F420E0822F51
:10E1B00008958FE69DE0E8DF21E0892B09F420E057
:10E1C000822F08958CE09EE0DFDF21E0892B09F4A7
:10E1D00020E0822F089589EA9EE0D6DF21E0892B96
:10E1E00009F420E0822F0895FC01A48DA80FB92F17
:10E1F000B11DA35ABF4F2C91848D90E001968F736F
:10E200009927848FA689B7892C93A089B1898C918D
:10E21000837080648C93938D848D981306C00288DC
:10E22000F389E02D80818F7D80830895EF92FF92A6
:10E230000F931F93CF93DF93EC0181E0888F9B8D29
:10E240008C8D98131AC0E889F989808185FF15C0E3
:10E250009FB7F894EE89FF896083E889F989808106
:10E260008370806480839FBF81E090E0DF91CF91D5
:10E270001F910F91FF90EF900895F62E0B8D10E0F7
:10E280000F5F1F4F0F731127E02E8C8D8E110BC067
:10E290000FB607FCFACFE889F989808185FFF5CFB1
:10E2A000CE01A2DFF2CFEB8DEC0FFD2FF11DE35A73
:10E2B000FF4FF0829FB7F8940B8FEA89FB8980812A
:10E2C0008062D0CFCF93DF93EC01888D8823B1F0AB
:10E2D000AA89BB89E889F9898C9185FD03C0808171
:10E2E00086FD0CC00FB607FCF7CF8C9185FFF2CFEF
:10E2F000808185FFEDCFCE0177DFEACFDF91CF912F
:10E30000089580E090E0892B21F065DF81110E9463
:10E31000000080E090E0892B21F054DF81110E9401
:10E32000000080E090E0892B21F043DF81110E9402
:10E33000000080E090E0892B21F032DF81110C9405
:10E34000000008958150823108F05AC0E82FF0E0B3
:10E350008827E255FE488F4F0C944DB1CE71D27193
:10E36000C071C671CA710072D571DB71DF71E57160
:10E37000E971ED71F371F7710072FB710172057251
:10E38000809180008F778093800008958091800035
:10E390008F7DF9CF80918000877FF5CF84B58F770F
:10E3A00084BD089584B58F7DFBCF8091B0008F77B9
:10E3B0008093B00008958091B0008F7DF9CF809157
:10E3C00090008F77809390000895809190008F7DCA
:10E3D000F9CF80919000877FF5CF8091A0008F7753
:10E3E0008093A00008958091A0008F7DF9CF809147
:10E3F000A000877FF5CF809120018F778093200147
:10E400000895809120018F7DF9CF80912001877F31
:10E41000F5CFCF93DF93282F30E0F901E35BF44F82
:10E420008491F901E95FF44FD491F901EF53F54F6D
:10E43000C491CC2399F0811185DFEC2FF0E0EE0F31
:10E44000FF1FE955F54FA591B491EC91ED2381E0C3
:10E4500090E009F480E0DF91CF91089580E090E0B2
:10E46000FACF3FB7F8948091F6149091F714A091E9
:10E47000F814B091F91426B5A89B05C02F3F19F0E8
:10E480000196A11DB11D3FBFBA2FA92F982F882734
:10E49000BC01CD01620F711D811D911D42E0660F0F
:10E4A000771F881F991F4A95D1F7089585ED8093AE
:10E4B000BC008091BC0084FDFCCF1092161808951A
:10E4C0002091E713260F3327331F21323105ECF457
:10E4D00020911618FC0190E080E0243069F082E081
:10E4E0000895A091E7132191AC0149535C4EA40F0C
:10E4F000B52FB11D2C930196861798F38091E713E1
:10E50000680F6093E71380E0089581E0089508950F
:10E51000E091940C8091930CE81730F4F0E0E2560F
:10E52000F34F808190E008958FEF9FEF08959091D1
:10E53000940C8091930C2FEF3FEF981748F4E92F3C
:10E54000F0E0E256F34F208130E09F5F9093940C0F
:10E55000C9010895CF92DF92EF92FF920F931F931C
:10E56000CF93DF937C01CB018A012091CE0C222333
:10E5700089F0EB016B01C40ED51ECC15DD0561F0F1
:10E580006991D701ED91FC910190F081E02DC701D7
:10E590001995F3CF642F94DFC801DF91CF911F91BC
:10E5A0000F91FF90EF90DF90CF900895CF93DF937E
:10E5B0001F92CDB7DEB769832091CE0C2223F9F0EC
:10E5C0002091D10C203258F021E030E0FC0133835F
:10E5D000228390E080E00F90DF91CF9108958091A9
:10E5E000CF0CE82FF0E0E95EF74E998190838F5FC2
:10E5F0008093CF0C8093D10C81E090E0ECCF61E070
:10E60000CE0101965DDFF8CFDC015996ED91FC91CA
:10E610003097B9F083899489A589B6894285538555
:10E6200064857585841B950BA60BB70B811520E8B7
:10E630009207A105B10538F08FEF9FE7A0E0B0E0A9
:10E64000089590E080E00895CF93DF931F92CDB7B7
:10E65000DEB76983DC01ED91FC910280F381E02D4E
:10E6600041E050E0BE016F5F7F4F19950F90DF9141
:10E67000CF9108950E9471B30F931F93CF93DF93AF
:10E68000EC0188819981009759F02A813B812617F6
:10E69000370730F081E0DF91CF911F910F910895FE
:10E6A0008B016F5F7F4F0E9495B2009759F099835D
:10E6B00088831B830A832C813D81232B59F7FC011E
:10E6C0001082E8CF80E0E7CFEF92FF920F931F9385
:10E6D000CF93DF936115710541F480E0DF91CF9115
:10E6E0001F910F91FF90EF90089541155105A9F0EA
:10E6F0007B01EC010C811D81040F151FB801BCDFEB
:10E70000882359F3288139818C819D81B701820F3B
:10E71000931F0E94B8B31D830C8381E0DFCFCF939A
:10E72000DF93EC0188819981009711F00E940CB26F
:10E73000198218821D821C821B821A82DF91CF915E
:10E740000895EF92FF920F931F93CF93DF93EC0105
:10E750007B018A01BA0190DF81110AC0CE01DFDF9F
:10E76000CE01DF91CF911F910F91FF90EF9008950F
:10E770001D830C83B701888199810E94B8B3F0CFC3
:10E78000CF92DF92EF92FF920F931F93CF93DF937D
:10E79000EC017A018B016C01C40ED51ECC15DD0590
:10E7A000A9F00E94AA0A8FE00E94AC0A8D2F0E9455
:10E7B000AC0A8C2F0E94AC0A219680E00E94AC0A21
:10E7C000F80181938F010E94A80AE8CFC701DF9169
:10E7D000CF911F910F91FF90EF90DF90CF90089510
:10E7E000982F2091D10C81E0213208F043C0809114
:10E7F00016188111FCCF8091D00C32E0309316189E
:10E80000909315189FEF909314181092131820935B
:10E810001218A7E1B8E1E2EFF7E190E0291331C067
:10E820001092F1179091F117880F892B8093F117AF
:10E830008091F017813049F51092F0178091F1170F
:10E840008093BB008091BC0083FDF8CF85EC809362
:10E85000BC00809116188230E1F3809114188F3F2C
:10E86000B1F0809114188032A1F080911418803397
:10E8700091F084E01092CF0C1092D10C1092CE0C3B
:10E8800008953D9131939F5FC9CF85EEE0CF80E041
:10E89000F1CF82E0EFCF83E0EDCF682F86E49FE0F9
:10E8A00085CECF93DF93EC019A01AB01E889F9891A
:10E8B00082E08083211581EE38074105510581F101
:10E8C00060E079E08DE390E00E94CBAF2150310908
:10E8D000410951095695479537952795EC85FD8552
:10E8E0001082EE85FF852083188EEC89FD8986E0F5
:10E8F0008083EA89FB89808180618083EA89FB8942
:10E90000808188608083EA89FB8980818068808338
:10E91000EA89FB8980818F7D8083DF91CF91089583
:10E92000E889F989108220E1D9CFCF93C82F462FEB
:10E9300061E070E00E94B30A61E070E08C2F0E94F9
:10E94000CC0A8111F9CFCF910895FF920F931F93B5
:10E95000CF93DF93F82E10E000E08F2D0E94F50A90
:10E96000EC01892B21F08F2D0E94F50A8C01C01734
:10E97000D10799F7CE01DF91CF911F910F91FF90B1
:10E9800008958F929F92AF92BF92CF92DF92EF92B3
:10E99000FF920F931F93CF93DF9300D0CDB7DEB7D5
:10E9A0004C017B016A01DC01ED91FC9180E8DB0107
:10E9B000982F1D929A95E9F7DA011D928A95E9F749
:10E9C000808190E8A92EB12C811119C084E090E0DB
:10E9D00006C08F0181E090E0D4010D931C930F904D
:10E9E0000F900F90DF91CF911F910F91FF90EF90BB
:10E9F000DF90CF90BF90AF909F908F9008958F0140
:10EA00000F5F1F4F6081663229F394F4662309F388
:10EA10006532D1F0B2E0AB16B10444F0F701608387
:10EA2000F1E0AF1AB108C70101967C01F801E7CF08
:10EA30006B3209F45EC06D3369F78181882351F22E
:10EA400080E8A82EB12C45C081818983882311F2EA
:10EA500082818A838F01811103C00E5F1F4FBACF5D
:10EA60000D5F1F4F1B8240E150E070E060E0CE017F
:10EA700001960E94E6A8CECF663281F06B32A1F5F6
:10EA800060E232C0F801818189838823A1F182810B
:10EA90008A83811107C00E5F1F4F7801870183E0D1
:10EAA00090E09ACF7801F3E0EF0EF11C1B8240E179
:10EAB00050E070E060E0CE0101960E94E6A814C02C
:10EAC000D6016C93B1E0AB1AB108F60131966F0133
:10EAD000870178019FEFE91AF90AD8016C91653234
:10EAE00089F254F66623C9F2E2E0AE16B10444F7A7
:10EAF000EFCF60E28FCF8701D0CF909116189111A0
:10EB0000FCCF91E090931618909315182FEF209357
:10EB1000141810921318260F209312189093F117BF
:10EB20009091F117880F892B8093F1178091F0173E
:10EB30008130F9F41092F0178091F1178093BB00A7
:10EB40008091BC0083FDF8CF85EC8093BC00809160
:10EB500016188130E1F380911318861710F4609134
:10EB60001318A2EFB7E1EEE9FCE080E0861303C0E2
:10EB7000089585EEEACF9D9191938F5FF7CFCF9364
:10EB8000DF93EC0183E394E0998388831A821B82EC
:10EB90001C821D8280E590E00E940E0BBE016E5F1C
:10EBA0007F4F44E050E08FE090E0EADD0E940D0BE3
:10EBB000CE01DF91CF9108950F931F93CF93DF93F1
:10EBC0004115510541F0FC01048115810115110524
:10EBD00039F4FB011082DF91CF911F910F910895BD
:10EBE000415051094017510708F48A01EB01FC011B
:10EBF00060817181A801CE010E94CDB3C00FD11FE9
:10EC00001882E9CFAF92BF92CF92DF92EF92FF923C
:10EC10000F931F93CF93DF931F921F92CDB7DEB751
:10EC20007A836983BA01A901E981FA81F770082F13
:10EC300010E0000F111F0A53134FD8018D919C91C2
:10EC40008E0F9F1F9F01240F351F2130384098F0F1
:10EC50005A016B0160E078E07B01EE1AFF0AA70120
:10EC6000B6018EDDA5014E195F09B6016E0D7F1D3F
:10EC7000F801808191810F900F90DF91CF911F91CA
:10EC80000F91FF90EF90DF90CF90BF90AF9078CD35
:10EC900020E3FC0120833296862F82958F706F705F
:10ECA0006A3030F4605D6293682F8111F5CF08956A
:10ECB000695CF9CFFB0101900020E9F73197AF01C2
:10ECC000461B570B3ECD0F931F93CF93DF93CDB7CA
:10ECD000DEB762970FB6F894DEBF0FBECDBF8C01D2
:10ECE000CB01F801118210821382128215821482E4
:10ECF0004AE0BE016F5F7F4F0E9444AABE016F5F72
:10ED00007F4FC801D7DF62960FB6F894DEBF0FBE03
:10ED1000CDBFDF91CF911F910F9108950F931F9356
:10ED2000CF93DF93CDB7DEB7A1970FB6F894DEBFD0
:10ED30000FBECDBF8C01CB01BA01F8011182108248
:10ED400013821282158214822AE0AE014F5F5F4F58
:10ED50000E9483AABE016F5F7F4FC801ABDFA196FF
:10ED60000FB6F894DEBF0FBECDBFDF91CF911F91DC
:10ED70000F910895CF93DF93EC016115710529F090
:10ED800099DFCE01DF91CF910895C9DCFACFFC0164
:10ED900080819181009711F00C94E6A960E070E009
:10EDA000CB010895FC0180819181009711F00C94B2
:10EDB00006AA60E070E0CB010895AF92BF92CF92B7
:10EDC000DF92EF92FF920F931F93CF93DF93DC01BB
:10EDD000CD90DC901197C114D10439F01496CD91E7
:10EDE000DC918C017601209761F4DF91CF911F9126
:10EDF0000F91FF90EF90DF90CF90BF90AF9008956C
:10EE000075015701BFEFAB1ABB0AF7018081082ECD
:10EE1000000C990B0E942CAA892B91F72197CC0DFD
:10EE2000DD1D8881082E000C990B0E942CAA892BCD
:10EE300029F0CE15DF0510F02197F3CFAE014F5F1B
:10EE40005F4F4E195F09D80115965C934E93149746
:10EE5000CE14DF0420F4B701C6010E948AB3D801A2
:10EE6000ED91FC91119714968D919C91E80FF91FEB
:10EE70001082BBCFFC01248135816217730748F4EF
:10EE800080819181009729F0860F971FFC01808176
:10EE9000089580E00895FC0124813581FB014481BF
:10EEA000558124173507A0F0FC01808191810097DE
:10EEB00079F0FB01608171816115710549F0241BB6
:10EEC000350B820F931F0E94AFB321E0892B09F00D
:10EED00020E0822F0895FB0144815581FC012481AB
:10EEE00035812417350778F080819181009759F09A
:10EEF000FB01608171816115710529F00E94BFB32A
:10EF000021E0892B09F020E0822F0895CF93DF9331
:10EF1000EC01FB0101900020E9F73197AF01461B9E
:10EF2000570BD2DB811102C0CE01F9DBCE01DF919C
:10EF3000CF910895CF93DF93EC01FB01448155817C
:10EF400060817181C1DB811102C0CE01E8DBCE019D
:10EF5000DF91CF910895EF92FF920F931F93CF937C
:10EF6000DF93EC017B01CB010E943BAA0097A1F04B
:10EF70000C811D81080F191FB801CE017DDB88238C
:10EF800061F0288139818C819D81B701820F931FA7
:10EF90000E9434AA1D830C8381E0DF91CF911F91E1
:10EFA0000F91FF90EF900895CF93DF931F921F92E0
:10EFB000CDB7DEB769831A8241E050E0BE016F5FD2
:10EFC0007F4F82DB0F900F90DF91CF910895CF9309
:10EFD000DF93EC01E9DF811102C0CE01A0DBCE019D
:10EFE000DF91CF910895FB0101900020E9F731975F
:10EFF000AF01461B570B68CBFB01448155816081F3
:10F00000718162CBEF92FF920F931F93CF93DF93A7
:10F01000EC018B01CB010E943BAA7C01BC01CE011B
:10F020002BDB81110AC0CE017ADBCE01DF91CF91BB
:10F030001F910F91FF90EF900895FD82EC82B8012F
:10F04000888199810E9434AAF0CFCF93DF93EC019D
:10F05000FB018617970741F0608171816115710589
:10F0600039F0448155816DDBCE01DF91CF91089558
:10F0700056DBFACF0F931F93CF93DF938C01EB01F5
:10F08000FC01808191810097E1F0688179816115AF
:10F090007105A9F0428153812C813D8142175307AC
:10F0A00070F00E94B8B38C819D81F80195838483B0
:10F0B0001D821C82DF91CF911F910F9108950E94B4
:10F0C0000CB288819981F801918380838A819B8128
:10F0D000938382838C819D81958384831982188296
:10F0E0001B821A82E5CFFC01808191810C940CB2C5
:10F0F000EF92FF920F931F93CF93DF93CDB7DEB7BD
:10F10000A1970FB6F894DEBF0FBECDBF7C01CB0137
:10F11000BA01F701118210821382128215821482C1
:10F1200042E0420F8E010F5F1F4F0E942BA8BC01CF
:10F13000C70120DEA1960FB6F894DEBF0FBECDBF8B
:10F14000DF91CF911F910F91FF90EF9008950F9352
:10F150001F93CF93DF93CDB7DEB7A2970FB6F89486
:10F16000DEBF0FBECDBF8C01CB01BA01F801118209
:10F170001082138212821582148230E0AE014F5F3A
:10F180005F4F0E944EAABE016F5F7F4FC80192DDA4
:10F19000A2960FB6F894DEBF0FBECDBFDF91CF9120
:10F1A0001F910F910895CF93DF931F921F92CDB7B8
:10F1B000DEB7FC0111821082138212821582148242
:10F1C00069831A82BE016F5F7F4F74DD0F900F90CD
:10F1D000DF91CF910895FC01118210821382128277
:10F1E0001582148247CFFC01118210821382128291
:10F1F0001582148207CFFC011182108213821282C1
:10F200001582148222CFFC01118210821382128295
:10F21000158214826115710549F0FB0101900020EF
:10F22000E9F73197AF01461B570B8BCA0895AF9290
:10F23000BF92CF92DF92EF92FF920F931F93CF93E3
:10F24000DF935C016B017A0189012417350720F4F3
:10F250008F2D7901042F182F67E079E0C501D3DFE6
:10F26000D6011496CD91DC91EC16FD06C0F40C1776
:10F270001D0708F4E801D601ED91FC911197EC0F00
:10F28000FD1F108110826D917C916E0D7F1DC50157
:10F2900071DDF60180819181C80FD91F1883C501E6
:10F2A000DF91CF911F910F91FF90EF90DF90CF9062
:10F2B000BF90AF900895FB0101900020E9F73197CE
:10F2C000AF01461B570BDC01ED91FC910280F381ED
:10F2D000E02D19948F929F92AF92BF92EF92FF927E
:10F2E0000F931F93CF93DF93CDB7DEB7A1970FB6E0
:10F2F000F894DEBF0FBECDBF7C01FA01CB0119A28D
:10F30000223008F42AE08E010F5D1F4F822E912CCF
:10F31000B12CA12CBF01A50194010E94CBAFF90132
:10F32000CA016A3004F5605DD8016E938D01232B0C
:10F33000242B252B79F790E080E0109719F0BD0180
:10F34000C701B9DFA1960FB6F894DEBF0FBECDBFDF
:10F35000DF91CF911F910F91FF90EF90BF90AF90F1
:10F360009F908F900895695CDFCFCF93DF93482FF4
:10F3700050E070E060E020E189EA9EE0ABDFEC0164
:10F380006FE17AE089EA9EE096DF8C0F9D1FDF91A6
:10F39000CF9108958F929F92AF92BF92CF92DF92BA
:10F3A000EF92FF920F931F93CF93DF937C01EB01BA
:10F3B0006C0182E0C80ED11C4701E5E08E0E911C65
:10F3C00010E000E0F60141916F0150E070E060E074
:10F3D0002AE0CE017FDF5C01E881F9810190F081B4
:10F3E000E02D6EE2CE0119958A0D9B1D080F191FA5
:10F3F000C814D90439F7F701458150E070E060E0A6
:10F400002AE0CE0167DF800F911FDF91CF911F911E
:10F410000F91FF90EF90DF90CF90BF90AF909F90B3
:10F420008F9008950F931F93CF93DF93EC01CB013F
:10F43000BE01B0DF8C016FE17AE0CE013CDF800FCE
:10F44000911FDF91CF911F910F9108950F931F93FB
:10F45000CF93DF93EC012FDF8C016FE17AE0CE01D7
:10F460002ADF800F911FDF91CF911F910F91089597
:10F470006115710509F01FCF90E080E00895DB0170
:10F4800014964D915C9115976D917C91DC01ED91F5
:10F49000FC910280F381E02D19940F931F93CF9379
:10F4A000DF93EC01ECDF8C016FE17AE0CE0103DF4A
:10F4B000800F911FDF91CF911F910F910895EF92CF
:10F4C000FF920F931F93CF93DF938C017B01D0E0CA
:10F4D000C0E0F701EC0FFD1F6491662361F0D801D5
:10F4E000ED91FC910190F081E02DC8011995892BD7
:10F4F00011F02196EECFCE01DF91CF911F910F91A8
:10F50000FF90EF900895DC0183E394E08D939D9349
:10F5100084E0FB0101900D928A95E1F708951F9216
:10F520000F920FB60F9211240BB60F922F933F93A9
:10F530004F935F936F937F938F939F93AF93BF93FB
:10F54000EF93FF9382ED9CE00E94F470FF91EF91A6
:10F55000BF91AF919F918F917F916F915F914F91EB
:10F560003F912F910F900BBE0F900FBE0F901F90E9
:10F5700018951F920F920FB60F9211240BB60F928F
:10F580002F933F934F935F936F937F938F939F93AB
:10F59000AF93BF93EF93FF9382ED9CE00E947A704C
:10F5A000FF91EF91BF91AF919F918F917F916F915B
:10F5B0005F914F913F912F910F900BBE0F900FBE17
:10F5C0000F901F9018951F920F920FB60F92112453
:10F5D0000BB60F922F933F934F935F936F937F934D
:10F5E0008F939F93AF93BF93EF93FF938FE69DE02D
:10F5F0000E94F470FF91EF91BF91AF919F918F9115
:10F600007F916F915F914F913F912F910F900BBE22
:10F610000F900FBE0F901F9018951F920F920FB66C
:10F620000F9211240BB60F922F933F934F935F933A
:10F630006F937F938F939F93AF93BF93EF93FF93BA
:10F640008FE69DE00E947A70FF91EF91BF91AF919C
:10F650009F918F917F916F915F914F913F912F91EA
:10F660000F900BBE0F900FBE0F901F9018951F921A
:10F670000F920FB60F9211240BB60F922F933F9358
:10F680004F935F936F937F938F939F93AF93BF93AA
:10F69000EF93FF938CE09EE00E94F470FF91EF9156
:10F6A000BF91AF919F918F917F916F915F914F919A
:10F6B0003F912F910F900BBE0F900FBE0F901F9098
:10F6C00018951F920F920FB60F9211240BB60F923E
:10F6D0002F933F934F935F936F937F938F939F935A
:10F6E000AF93BF93EF93FF938CE09EE00E947A70FC
:10F6F000FF91EF91BF91AF919F918F917F916F910A
:10F700005F914F913F912F910F900BBE0F900FBEC5
:10F710000F901F9018951F920F920FB60F92112401
:10F720000BB60F922F933F934F935F936F937F93FB
:10F730008F939F93AF93BF93EF93FF9389EA9EE0DC
:10F740000E94F470FF91EF91BF91AF919F918F91C3
:10F750007F916F915F914F913F912F910F900BBED1
:10F760000F900FBE0F901F9018951F920F920FB61B
:10F770000F9211240BB60F922F933F934F935F93E9
:10F780006F937F938F939F93AF93BF93EF93FF9369
:10F7900089EA9EE00E947A70FF91EF91BF91AF914C
:10F7A0009F918F917F916F915F914F913F912F9199
:10F7B0000F900BBE0F900FBE0F901F9018951F93C8
:10F7C000CF93DF93282F30E0F901E35BF44F84916E
:10F7D000F901E95FF44FD491F901EF53F54FC4916A
:10F7E000CC23A9F0162F81110E94A271EC2FF0E01A
:10F7F000EE0FFF1FE357F54FA591B4918FB7F89423
:10F80000EC91111108C0D095DE23DC938FBFDF91FE
:10F81000CF911F910895DE2BF8CF1092940C109287
:10F82000930C1092CF0C1092D10C1092161881E00C
:10F83000809315181092F01761E084E1C0DF61E059
:10F8400085E1BDDFE9EBF0E080818E7F8083808100
:10F850008D7F808388E48093B80085E48093BC002A
:10F8600083E490E7909385158093841584E490E772
:10F8700090938315809382150895AF92BF92CF9293
:10F88000DF92EF92FF920F931F93CF93DF936B0161
:10F890007A01EC01C351DB4E28813CE0389F8001A6
:10F8A000399F100D1124A0905518B12C27FF1FC0AF
:10F8B000FB011182108288818F5F88838881980183
:10F8C000280F311D87FD3A95F6012A153B051CF4DA
:10F8D00088818C30BCF180819181049680349C4970
:10F8E00008F471C0F6018081918104966EC0888110
:10F8F0009801280F311D87FD3A952A153B05DCF646
:10F900008881A801480F511D87FD5A95FA01EE0F15
:10F91000FF1FE40FF51FE555F04F808186FFCBCF29
:10F920008881F801E80FF11D87FDFA95CF01EE0FF0
:10F93000FF1FE80FF91FE555F04F808160E08F73DE
:10F940003EDFB9CF808191812881A801420F511DEE
:10F9500027FD5A959A01FA01EE0FFF1FE20FF31FE0
:10F96000E555F04F21813281820F931FF70191837A
:10F97000808388819801280F311D87FD3A95F90110
:10F98000EE0FFF1FE20FF31FE555F04F808186FF5A
:10F9900021C08881080F111D87FD1A95F801EE0F0F
:10F9A000FF1FE00FF11FE555F04F808161E08F737D
:10F9B000DF91CF911F910F91FF90EF90DF90CF904B
:10F9C000BF90AF90FCCE80E49CE9F70191838083E7
:10F9D0008FEF8883DF91CF911F910F91FF90EF9070
:10F9E000DF90CF90BF90AF900895CF93DF9390E0DA
:10F9F000FC01E95FF44F24918F53954FFC018491F2
:10FA00008823D1F090E0880F991FFC01ED58F54F45
:10FA1000A591B491FC01E357F54FC591D4916111C3
:10FA20000EC09FB7F8948C91E22FE0958E238C93B3
:10FA30002881E223E8839FBFDF91CF9108958FB79C
:10FA4000F894EC91E22BEC938FBFF6CF8F929F92BC
:10FA5000AF92BF92CF92DF92EF92FF926B017C0147
:10FA60000E9431724B015C01C114D104E104F10424
:10FA7000B9F00E943172681979098A099B09683EB8
:10FA800073408105910580F321E0C21AD108E10895
:10FA9000F10888EE880E83E0981EA11CB11CE4CF0B
:10FAA000FF90EF90DF90CF90BF90AF909F908F909E
:10FAB0000895AF92BF92CF92DF92EF92FF920F9391
:10FAC0001F93CF93DF93C82FD62F1092331310922A
:10FAD000341310923513109236131092371361E0DD
:10FAE00084DF60E08C2F6BDE6D2F70E090E080E0B3
:10FAF000ADDF60E08C2F79DF8BE990E00197F1F7C3
:10FB000000E911E08C2F0E940972892B81F40150C9
:10FB10001109C1F78EEF9FEFDF91CF911F910F91E8
:10FB2000FF90EF90DF90CF90BF90AF90089500E9E5
:10FB300011E08C2F0E940972019721F401501109E4
:10FB4000C1F7E8CF18E2D0E800E090E9E92EFF2401
:10FB5000F3948C2F0E940972892B29F481E0E81A12
:10FB6000F108B9F7D7CF0E9431726B017C0180E9AF
:10FB7000A82EBB24B3948C2F0E940972019729F4FC
:10FB800081E0A81AB108B9F7C5CF0E9431726C198B
:10FB90007D098E099F09693271058105910538F04B
:10FBA000E02FF0E0E55DFC4E80858D2B8087D695BB
:10FBB00011F40F5FD0E8115041F690E080E0ACCF37
:10FBC0002FB7F8946091F2147091F3148091F414AB
:10FBD0009091F5142FBF0895CF92DF92EF92FF928C
:10FBE000CF93DF9380915710843051F4CFEFDFEF44
:10FBF000CE01DF91CF91FF90EF90DF90CF900895ED
:10FC0000E0917A10E1113CC0DBDF6B017C0128EE52
:10FC1000C20E23E0D21EE11CF11C8BE490E10E9495
:10FC2000AF0D882319F38091B010882331F08091B3
:10FC30007B1090917C10892BC9F28BE490E10E949B
:10FC4000920CEC01CF3FDC0771F08091B01088235B
:10FC500079F280917B1090917C10019790937C10A9
:10FC600080937B10C5CFACDFC616D706E806F90631
:10FC7000A0F610927A108BE490E10E941F13B8CF87
:10FC8000E150E0937A100E2E000CFF0BEF5BFF4E5D
:10FC9000C18DD0E0ADCF0F931F93CF93DF93EC01D5
:10FCA0008C01F80181918F018823B9F195DFF8016A
:10FCB0002291022E000C330B8217930791F38F3F92
:10FCC000980791F0A0917A1091E09A0F90937A1092
:10FCD0000A2E000CBB0BAF5BBF4E59968C93903233
:10FCE00019F48FE180937A102FE1EC17FD07D9F01A
:10FCF00092919F3FD1F3A0917A1081E08A0F809377
:10FD00007A100A2E000CBB0BAF5BBF4E59969C932A
:10FD1000803259F720937A10E8CF81E0DF91CF91BC
:10FD20001F910F91089580E0F9CF1F920F920FB6A7
:10FD30000F9211242F933F938F939F93AF93BF9371
:10FD40008091F2149091F314A091F414B091F514F1
:10FD50003091F11423E0230F2D3758F50196A11DA2
:10FD6000B11D2093F1148093F2149093F314A09397
:10FD7000F414B093F5148091F6149091F714A091B7
:10FD8000F814B091F9140196A11DB11D8093F614D9
:10FD90009093F714A093F814B093F914BF91AF9116
:10FDA0009F918F913F912F910F900FBE0F901F90B9
:10FDB000189526E8230F0296A11DB11DD2CFCF9230
:10FDC000DF92EF92FF92CF93DF93EC01603282E0FB
:10FDD0007807CCF5653B710514F064EB70E0898120
:10FDE00028E830E0281B310987FD3395220F331FA7
:10FDF000220F331F6901330FEE08FF088A8128E5BF
:10FE000032E0281B310987FD3395220F331F220F63
:10FE1000331F032E000C440B550B2C193D094E09C2
:10FE20005F09DB0177FF02C0B0E0A0E00E9413B0E1
:10FE300024EB30E040E050E00E94EDAFC20ED31E54
:10FE4000E41EF51EB601E881E03370F5298188E8EB
:10FE500090E0821B910927FD9395880F991F880FC9
:10FE6000991F681779077CF02A8188E592E0821B48
:10FE7000910927FD9395880F991F880F991F68177F
:10FE800079070CF4CB010297880F991F4FB7F894AC
:10FE90002E2F30E0F901EE0FFF1FE20FF31FE555A3
:10FEA000F04F928381834FBFDF91CF91FF90EF900E
:10FEB000DF90CF9008951F93CF93DF93EC01162F1F
:10FEC0008881803308F04DC061E0812F8EDD88810C
:10FED000282F30E0F901EE0FFF1FE20FF31FE55569
:10FEE000F04F1F736081607C612B608319821A82DE
:10FEF0002CE0622F0E942EB1829FB001112430E0CD
:10FF000020E0AB01420F531FFA01EE0FFF1FE40F79
:10FF1000F51FE555F04F908196FD16C02F5F3F4FBE
:10FF20002C30310571F7813009F51092800082E0A4
:10FF3000809381001092850010928400B19A809184
:10FF40006F00826080936F00E8818E2F90E0FC014B
:10FF5000EE0FFF1FE80FF91FE555F04F8081806419
:10FF600080838881DF91CF911F910895823061F461
:10FF7000109290008093910010929500109294003E
:10FF800088BB80937100E0CF833069F41092A000A9
:10FF900082E08093A1001092A5001092A40089BB7A
:10FFA00080937200D1CF8111CFCF1092200182E0D7
:10FFB0008093210110922501109224018ABB809325
:10FFC0007300C2CF1F920F920FB60F9211240BB67F
:10FFD0000F922F933F934F935F936F937F938F93E2
:10FFE0009F93AF93BF93EF93FF9348E251E064E296
:10FFF00071E090E080E041DCFF91EF91BF91AF9123
:020000021000EC
:100000009F918F917F916F915F914F913F912F9130
:100010000F900BBE0F900FBE0F901F9018951F9260
:100020000F920FB60F9211240BB60F922F933F939E
:100030004F935F936F937F938F939F93AF93BF93F0
:10004000EF93FF9348EA50E064EA70E083E090E0C9
:1000500014DCFF91EF91BF91AF919F918F917F91B0
:100060006F915F914F913F912F910F900BBE0F9029
:100070000FBE0F901F9018951F920F920FB60F9200
:1000800011240BB60F922F933F934F935F936F936F
:100090007F938F939F93AF93BF93EF93FF9348E921
:1000A00050E064E970E082E090E0E7DBFF91EF91DF
:1000B000BF91AF919F918F917F916F915F914F9180
:1000C0003F912F910F900BBE0F900FBE0F901F907E
:1000D00018951F920F920FB60F9211240BB60F9224
:1000E0002F933F934F935F936F937F938F939F9340
:1000F000AF93BF93EF93FF9348E850E064E870E05C
:1001000081E090E0BADBFF91EF91BF91AF919F91B9
:100110008F917F916F915F914F913F912F910F90B0
:100120000BBE0F900FBE0F901F901895FC012481FD
:1001300031E03093CE0C2093D00C1092CF0C109263
:10014000D10C8385862B90E00E944D7481E00C9445
:10015000F0730F931F93CF938C01C62FE7DF6C2FA3
:100160006460C801E3DF6C2F6B7FC801DFDF83ECC5
:1001700090E00197F1F7CF911F910F9108950F93A0
:100180001F93CF938C01C62F607F6160E2DF80E117
:10019000C89FB00111246160C801DBDF81E090E0FD
:1001A000CF911F910F910895CF93C82F682F607F33
:1001B0008FEA93E1CEDF80E1C89FB00111248FEA7E
:1001C00093E1CF91C6CFCF93DF9300D000D01F92A1
:1001D0001F92CDB7DEB798E0EBE4F3E0DE011196B5
:1001E00001900D929A95E1F79091B813961708F443
:1001F0006FEF70E0660F771F21E030E02C0F3D1F9E
:10020000620F731FFB019081890F806828960FB6DB
:10021000F894DEBF0FBECDBFDF91CF91C5CF0F9356
:100220001F93CF93DF932091E2022223F9F02091D4
:10023000E1022223D9F0EB018C0161E080E0C3DF11
:10024000B8018FEA93E11BD96AEE7CE08FEA93E173
:1002500036D961E0F8018481B6DFBE01DD0F880B7D
:10026000990BDF91CF911F910F91F0CBDF91CF913F
:100270001F910F9108956093E9147093EA1480938D
:10028000EB149093EC14645D7E4F8F4F9F4F6093FF
:10029000E5147093E6148093E7149093E81482E0D9
:1002A00090E09093E4148093E3148ADC6093DF146D
:1002B0007093E0148093E1149093E2140895CF9228
:1002C000DF92EF92FF920F931F937ADC8B019C01D8
:1002D000C090DF14D090E014E090E114F090E214AC
:1002E0006091E9147091EA148091EB149091EC14F0
:1002F0000C191D092E093F09083E1340210531053F
:10030000E0F0DC01CB010196A11DB11D8093E91441
:100310009093EA14A093EB14B093EC14B701A601E8
:1003200048515C4F6F4F7F4F4093DF145093E01460
:100330006093E1147093E214C8CF1F910F91FF9066
:10034000EF90DF90CF9008954F925F926F927F92DF
:100350008F929F92AF92BF92CF92DF92EF92FF92D5
:100360000F931F93CF93DF934B015C018091DB14BC
:100370009091DC14A091DD14B091DE1488159905DC
:10038000AA05BB0509F4C6C08CE3C82ED12CE12C0C
:10039000F12CC501A70196010E94CBAF6093610CBF
:1003A000CA01B901A70196010E94CBAF6093620C0C
:1003B000C501B40120E13EE040E050E00E94CBAF37
:1003C000CA01B90128E130E040E050E00E94CBAF23
:1003D0006093630CC501B40120E831E541E050E0D1
:1003E0000E94CBAF69017A01CA01B9016C5F7F4FEE
:1003F0008F4F9F4F27E030E040E050E00E94CBAFAE
:100400006F5F6093640C412C512C320140E004E694
:1004100010E0C0E9D1E0242F30E02E54384FF9012C
:10042000E370FF273097F9F4C901B8010E943AB18F
:10043000892B31F4C901BE010E943AB1892B99F48C
:100440008EE691E0A0E0B0E0480E591E6A1E7B1EC9
:10045000D301C201AA27BB27C816D906EA06FB06A4
:1004600038F04F5FD8CF8DE691E0A0E0B0E0ECCF60
:100470004093670CC90164E670E00E943AB1EC0158
:10048000C90160E971E00E943AB1309721F42097E8
:10049000D9F40097C9F04DE651E060E070E0441AED
:1004A000550A660A770AC418D508E608F708A5E5CC
:1004B000B3E020E0213069F43097E9F5209711F49A
:1004C0000097C9F54DE106C04EE651E060E070E0EE
:1004D000E6CF4C9150E070E060E031E0320FC4169E
:1004E000D506E606F70640F0C41AD50AE60AF70A6A
:1004F0001196232F3C30F1F62F5F2093660CC394A6
:10050000C092650C8092DB149092DC14A092DD14F2
:10051000B092DE14DF91CF911F910F91FF90EF9079
:10052000DF90CF90BF90AF909F908F907F906F9013
:100530005F904F9008954CE1CDCFC1DE05DF8091F3
:10054000670C90E08E54984F0895B9DEFDDE8091DF
:10055000660C90E00895B3DEF7DE8091650C90E0C4
:100560000895ADDEF1DE8091620C90E00895A7DE83
:10057000EBDE8091630C90E008951F920F920FB60E
:100580000F9211240BB60F922F933F934F935F93CB
:100590006F937F938F939F93AF93BF93EF93FF934B
:1005A00080910B140E94097220910E1430910F1447
:1005B0002F5F3F4F30930F1420930E1490910D1422
:1005C000953618F096E090930A1490910A1494309E
:1005D00009F46EC0F8F4923031F1933009F44CC054
:1005E00090910C14992319F0811171C02F9AFF91E9
:1005F000EF91BF91AF919F918F917F916F915F919B
:100600004F913F912F910F900BBE0F900FBE0F9007
:100610001F901895953009F457C0963009F791E06E
:100620009093DA144FC08111DBCF20910E143091DA
:100630000F142436310528F410920F1410920E1462
:10064000CFCF1092DA1410920D14E0910D1491E0B6
:100650009E0F90930D14F0E020910E1430910F1422
:10066000EE0FFF1FE05FFB4E3183208310920F14CB
:1006700010920E1493E019C0813009F0B1CFE091CF
:100680000D1491E09E0F90930D14F0E020910E1444
:1006900030910F14EE0FFF1FE05FFB4E318320837C
:1006A00010920F1410920E1494E090930A1498CFA5
:1006B000882359F220910E1430910F1425363105FC
:1006C00008F48ECF95E0F1CF81118ACFB5CF2F9866
:1006D0008ECF1F920F920FB60F9211240BB60F926E
:1006E0002F933F934F935F936F937F938F939F933A
:1006F000AF93BF93EF93FF938091B900887F8036CB
:1007000009F44DC008F040C0883209F4A9C028F5AA
:10071000803109F49DC0C8F4882309F4FBC08830F7
:1007200009F496C0FF91EF91BF91AF919F918F9186
:100730007F916F915F914F913F912F910F900BBEE1
:100740000F900FBE0F901F901895883109F488C044
:10075000803241F78093141814C0803409F49DC08E
:1007600040F48033B9F38833E9F68093141885ECAC
:10077000B0C0803509F485C0883509F496C0883446
:1007800089F60E945672CECF883909F48CC038F5AC
:10079000883729F050F4883611F0803719F683E055
:1007A000809316181092091457C0883809F47BC03A
:1007B000803919F0803809F0B5CF80910914803262
:1007C00008F071C0E091091481E08E0F8093091444
:1007D0008091BB00F0E0E751FC4E80833DC0803B40
:1007E00039F0E0F4803A09F479C0883A09F09ACFF8
:1007F00084E0809316181092E8131092E713E091AA
:100800008415F091851519958091E71381110FC01A
:1008100081E08093E7131092C71309C0803C09F46C
:10082000A6CF883C09F4A3CF883B09F07BCFE091A9
:10083000E81381E08E0F8093E813F0E0E953FC4E5B
:1008400080818093BB009091E8138091E71329C0C9
:100850008091F1178093BB0085EC8093BC0062CF40
:100860009091131880911218981758F5E091131869
:1008700081E08E0F80931318F0E0EE50F84E8081E7
:10088000E9CFE091131881E08E0F809313188091C7
:10089000BB00F0E0EE50F84E8083909113188091E9
:1008A00012189817C8F285E8D8CFE091131881E0A4
:1008B0008E0F809313188091BB00F0E0EE50F84E3D
:1008C00080838091151881115CCF81E08093F017AF
:1008D00084EA8093BC001092161824CF85EC809394
:1008E000BC001092161880910914803230F4E09107
:1008F0000914F0E0E751FC4E10826091091470E099
:10090000E0918215F091831589EE93E1199510928B
:10091000091408CF1092141834CFCF93DF93EC0151
:100920008091C113811109C081E08093C11380912E
:10093000520F9091530F0E940E0B60E08C81DF915B
:10094000CF910C94DF7B61E0FC0184810E94DF7B0E
:100950008091C113882321F01092C1130C940D0BC8
:1009600008958FEF0C94AC0A0F931F93CF93DF93EE
:10097000EC0126D98B01F5DF8F3F61F021D9601B97
:10098000710B6C177D07B8F380E0DF91CF911F9159
:100990000F91089581E0F9CF8F929F92AF92BF920D
:1009A000FF920F931F93CF93DF93EC01F62E490133
:1009B0005A018E81882379F08F8198859C012F5F61
:1009C0003F4F38872F838230924010F4CADFF4CF34
:1009D000CE01B9DF1E82CE01A0DF8CE291E0C4DF40
:1009E0008F2D80640E94AC0A08E110E0D501C4019B
:1009F000002E04C0B695A795979587950A94D2F7CF
:100A00000E94AC0A08501109083F8FEF180771F7D0
:100A100085E9FF2021F028E087E8F2128FEF0E949D
:100A2000AC0A10E09EDF8A8787FF04C01F3F11F0E9
:100A30001F5FF8CFDF91CF911F910F91FF90BF9073
:100A4000AF909F908F900895AF92BF92CF92DF9218
:100A5000EF92FF920F931F93CF93DF93EC01690105
:100A6000C801820F931F8130924048F58E81882300
:100A700079F088819981AA81BB8184179507A6079F
:100A8000B70731F48F819885C816D90608F03CC0A5
:100A9000488359836A837B838B85833039F089E06F
:100AA000440F551F661F771F8A95D1F79A01AB0136
:100AB00061E1CE0171DF882381F083E08D83CE0177
:100AC00042DF80E0DF91CF911F910F91FF90EF9077
:100AD000DF90CF90BF90AF90089572D85B0141DF57
:100AE0008A878F3F59F46CD86A197B096D3271403F
:100AF000B0F38FE08D83CE0126DFE1CF8E3F81F40E
:100B000018861F8281E08E838F8198858C159D05C4
:100B100048F427DF8F819885019698878F83F4CFDB
:100B20008DE0E8CF6701E00EF11E1BDFF601819337
:100B30006F01EE15FF05C9F78F819885080F191F02
:100B400018870F838985882319F00115124090F0CA
:100B50008E81882379F08F8198859C012F5F3F4F8C
:100B600038872F838230924010F4FBDEF4CFCE0121
:100B7000EADE1E8281E0A6CFEF92FF920F931F93D1
:100B8000CF93DF93EC01790182E1411551056105B5
:100B9000710591F08B85833039F089E0440F551F42
:100BA000661F771F8A95D1F79A01AB0168E1CE01E4
:100BB000F3DE882319F084E08D832CC08EEF0E9431
:100BC000AC0A87018EEFF81AF80181918F010E941B
:100BD000AC0A0E151F05C1F78FEF0E94AC0A8FEF0C
:100BE0000E94AC0ABEDE8A878F71853079F488E571
:100BF00092E0BADE882391F020E030E0A9016DE0B8
:100C0000CE01CADE882361F084E1D6CF81E18D83F5
:100C1000CE0199DECE0197DE80E008C085E1CCCF21
:100C2000A0DE8111F1CFCE018EDE81E0DF91CF9188
:100C30001F910F91FF90EF900895CF93DF938091D4
:100C4000C213882399F1C0918615D09187154091E0
:100C5000940250919502609196027091970220EF54
:100C600035E1CE0189DF811104C080E0DF91CF91B1
:100C700008954091C3135091C4136091C5137091AE
:100C8000C613411551056105710571F020EF35E17D
:100C9000CE0172DF882349F31092C3131092C4135C
:100CA0001092C5131092C6131092C21381E0DECFCA
:100CB0008F929F92AF92BF92EF92FF920F931F93EA
:100CC000CF934B015C01C42F8091940290919502C7
:100CD000A0919602B091970288159905AA05BB05C7
:100CE00039F1ABDF81110BC080E0CF911F910F91E3
:100CF000FF90EF90BF90AF909F908F90089580EFFE
:100D0000E82E85E1F82E00E012E030E020E0B501A9
:100D1000A401809186159091871596DE882321F392
:100D20008092940290929502A0929602B0929702BD
:100D30004091C2134C2B4093C21381E0D6CFCF9386
:100D4000DF93EC016E857F858889998941E0B0DF6A
:100D5000882351F08A8920E2829FC00111248051AA
:100D60009A4EDF91CF91089590E080E0FACF8F9274
:100D70009F92AF92BF92CF92DF92EF92FF92CF936A
:100D800024E53FE03093871520938615882309F4E6
:100D90006BC040E060E070E0CB018ADF81110BC0E6
:100DA00080E0CF91FF90EF90DF90CF90BF90AF9019
:100DB0009F908F9008958091AE178F7789F78091DB
:100DC000BA179091BB17A091BC17B091BD1784368C
:100DD0009105A105B10520F3C090B617D090B717C3
:100DE000E090B817F090B917C114D104E104F104F0
:100DF000B9F240E0C701B6015BDF882389F2809138
:100E0000FB159091FC158115924051F6A0910016AA
:100E1000AA2331F26091FE157091FF1561157105DD
:100E200009F4BECF2091FD15222309F4B9CFA09378
:100E3000720F2093640F90E080E030E0E1E0F0E09A
:100E4000C82FAF01082E02C0440F551F0A94E2F7C5
:100E50002417350769F041E0480F01968930910564
:100E600079F740936D0F9CCFC12CD12C7601C1CF67
:100E700080936D0F209106163091071650E040E0E8
:100E80002115310541F42091141630911516409129
:100E90001616509117162093650F3093660F4093E6
:100EA000670F5093680F46015701860E971EA11CCD
:100EB000B11C8092730F9092740FA092750FB09234
:100EC000760FE0910116F0910216F093790FE093FE
:100ED000780FB0E00E9409B0DC01CB01880D991DAC
:100EE000AA1DBB1D80937A0F90937B0FA0937C0F5C
:100EF000B0937D0F25E0EE0FFF1F2A95E1F7E1503B
:100F0000FE4FEF2FFF27E6958E0F9F1FA11DB11DEE
:100F100080936E0F90936F0FA093700FB093710F2B
:100F20008090031690900416B12CA12C811491048A
:100F300041F48090101690901116A0901216B09067
:100F40001316C81AD90AEA0AFB0AC80CD91CEA1CEB
:100F5000FB1C04C0F694E794D794C794CA95D2F7C3
:100F6000C092690FD0926A0FE0926B0FF0926C0FF3
:100F700085EFC8168FE0D806E104F10428F48CE070
:100F80008093770F81E00DCF80E125EFC2162FEF20
:100F9000D206E104F104A0F380911C1690911D1675
:100FA000A0911E16B0911F1680937A0F90937B0F1D
:100FB000A0937C0FB0937D0F80E2E2CF4F925F92BF
:100FC0006F927F928F929F92AF92BF92CF92DF9259
:100FD000EF92FF920F931F93CF93DF93EC01423078
:100FE00051056105710590F480E0DF91CF911F916B
:100FF0000F91FF90EF90DF90CF90BF90AF909F90B8
:101000008F907F906F905F904F90089589859A851B
:10101000AB85BC850196A11DB11D84179507A60758
:10102000B70710F3CB88DC88ED88FE888F89803184
:1010300009F042C0BB27A72F962F852F48015901E1
:101040002A013B01C80ED91EEA1EFB1E80919402A4
:1010500090919502A0919602B0919702C816D90678
:10106000EA06FB0699F58F898031B9F5B301A20133
:10107000552766277727440F551F40515A4EFA01CE
:10108000918280828091C21381608093C2138A8989
:10109000823080F08D819E81AF81B8858C0D9D1D41
:1010A000AE1DBF1D8093C3139093C413A093C513AB
:1010B000B093C61381E099CFDB01CA01E7E0B69592
:1010C000A79597958795EA95D1F7B8CF40E0C701E6
:1010D000B601EEDD8111C7CF87CFB301A2014F77F3
:1010E000552766277727440F551F440F551F40513A
:1010F0005A4EFA0180829182A282B382C3CF8F922C
:101100009F92AF92BF92CF92DF92EF92FF920F9396
:101110001F93CF93DF93FC0181859285A385B485CE
:101120000196A11DB11D84179507A607B70770F496
:1011300080E0DF91CF911F910F91FF90EF90DF90B2
:10114000CF90BF90AF909F908F90089583889488A0
:10115000A588B6888789803189F5BB27A72F962F68
:10116000852FE9016A017B018F01BC01CD01680D6A
:10117000791D8A1D9B1D8090940290909502A090ED
:101180009602B090970286169706A806B90601F552
:10119000F8018789803109F5DD24EE24FF24F6016A
:1011A000EE0FFF1FE051FA4E80819181B0E0A0E088
:1011B00088839983AA83BB8381E0BBCFDB01CA010B
:1011C000C7E0B695A79597958795CA95D1F7C9CFEA
:1011D00040E06EDD8111DCCFABCFE894C7F8DD24B1
:1011E000EE24FF24F601EE0FFF1FEE0FFF1FE0516C
:1011F000FA4E80819181A281B381BF70D9CF4F9285
:101200005F926F927F92AF92BF92CF92DF92EF92F6
:10121000FF920F931F93CF93DF9300D01F92CDB710
:10122000DEB78C0149835A836B837C835901C12CBF
:10123000D12C7601412C82E0582E612C712C4981F1
:101240005A816B817C819E012F5F3F4FC80157DF20
:10125000882339F1F8018585A301920104C0220F8A
:10126000331F441F551F8A95D2F7DA01C901C80EF2
:10127000D91EEA1EFB1E49815A816B817C818789B8
:10128000803111F188EF9FEFAFEFBFE048175907AA
:101290006A077B07A0F2F501C082D182E282F38265
:1012A00081E00F900F900F900F90DF91CF911F91E1
:1012B0000F91FF90EF90DF90CF90BF90AF907F9015
:1012C0006F905F904F90089588EF9FEFA0E0B0E09F
:1012D000DDCF8F929F92AF92BF92CF92DF92EF922B
:1012E000FF920F931F93CF93DF93EC018D818111B8
:1012F0000EC080E0DF91CF911F910F91FF90EF9092
:10130000DF90CF90BF90AF909F908F9008950B8902
:101310001C892D893E89041715072607370748F3CE
:101320004A015B01823031F48A869B86AC86BD8699
:1013300081E0E0CF81149104A104B10449F41E823C
:101340001F82188619861A861B861C861D86F0CF7A
:101350000A851B852C853D85EB8DFC8D858590E070
:101360000996B901A8014150510961097109082E76
:1013700004C076956795579547950A94D2F77501FD
:101380006401E1E0CE1AD108E108F10804C0F69446
:10139000E794D794C7948A95D2F7C416D506E60683
:1013A000F70620F0012B022B032B09F58F89988D6E
:1013B000A98DBA8D8E839F83A887B9878E010A5F16
:1013C0001F4FC114D104E104F10409F4ADCF4E81E3
:1013D0005F816885798598018B8D9C8D90DE91E089
:1013E000C91AD108E108F1088111EBCF82CFC41AE4
:1013F000D50AE60AF70AE2CF3F924F925F926F92C8
:101400007F928F929F92AF92BF92CF92DF92EF9294
:10141000FF920F931F93CF93DF93CDB7DEB72C9737
:101420000FB6F894DEBF0FBECDBF5C01DC015B964A
:101430008D909C905C9716964D905D906D907C90F1
:101440001997411451046104710409F467C0BFEF96
:101450004B1A5B0A6B0A7B0A312CF4018185928559
:10146000A385B4859C01AD012F5F3F4F4F4F5F4F68
:1014700029873A874B875C87730162011D821E8230
:101480001F821886F40181859285A385B4852D81FC
:101490003E814F815885281739074A075B0708F0B6
:1014A00054C089859A85AB85BC858C159D05AE0594
:1014B000BF0550F482E0C82ED12CE12CF12C92E033
:1014C000492E512C612C712C9E012F5F3F4FB7018B
:1014D000A601C40114DE8823C1F189819A81AB8100
:1014E000BC81892B8A2B8B2B09F1260137019FEFB9
:1014F000491A590A690A790A2D813E814F81588516
:101500002F5F3F4F4F4F5F4F2D833E834F83588751
:101510003FEFC31AD30AE30AF30AB4CFF4014080C1
:101520005180628073803324339497CFC414D504E0
:10153000E604F70409F70FEF1FEF2FEF3FE0B701C5
:10154000A601C4013BDD811119C080E02C960FB6C5
:10155000F894DEBF0FBECDBFDF91CF911F910F91E9
:10156000FF90EF90DF90CF90BF90AF909F908F90C3
:101570007F906F905F904F903F900895F501468166
:10158000578160857185411551056105710531F0FF
:1015900097018601C40112DD8823B9F2D5011696A0
:1015A000CD92DD92ED92FC921997332051F0D70144
:1015B000C6010196A11DB11DF40180839183A28310
:1015C000B383F5018789908DA18DB28D892B8A2BEC
:1015D0008B2B39F4C78AD08EE18EF28E848180689D
:1015E000848381E0B3CF2F923F924F925F926F92AC
:1015F0007F928F929F92AF92BF92CF92DF92EF92A3
:10160000FF920F931F93CF93DF93EC015B012A01AD
:101610008D81811115C08FEF9FEFDF91CF911F91C9
:101620000F91FF90EF90DF90CF90BF90AF909F9081
:101630008F907F906F905F904F903F902F90089584
:101640008C8180FFE8CF0B891C892D893E894A85D2
:101650005B856C857D85C201B0E0A0E06801790101
:10166000C41AD50AE60AF70AC816D906EA06FB061E
:1016700018F42801441A550A42011E0126E0220EE0
:10168000311C8114910409F4B0C04A855B856C85D6
:101690007D856A0181E0D8228B8D9C8D8A019B011A
:1016A000E9E03695279517950795EA95D1F7ED81ED
:1016B000E230D9F5FC01628D738D848D958D600FBC
:1016C000711F821F931F612C22E0722E6C187D08FF
:1016D0008614970408F434012C8126FD04C061149B
:1016E000F2E07F0671F4009194021091950220912E
:1016F000960230919702061717072807390709F055
:1017000051C040E0D5DA882309F485CFC601805165
:101710009A4ED5019C01260D371DFC012E173F075F
:1017200009F45EC041914D93F9CFFC0174807A9425
:101730007022C114D10471F471100CC0452B462BDA
:10174000472B39F58F89988DA98DBA8D8E839F830C
:10175000A887B987EB8DFC8D6E817F8188859985FF
:101760006250710981099109258504C0660F771FB0
:10177000881F991F2A95D2F70685178520893189F8
:10178000600F711F821F931F670D711D811D911DB9
:101790009ACF4E815F81688579859101B0DC811196
:1017A000D9CF39CF750183019601AB01BC0180917E
:1017B00086159091871548D9882309F42CCFA60C5B
:1017C000B71C8A859B85AC85BD85860D971DA11D9F
:1017D000B11D8A879B87AC87BD878618970851CF34
:1017E000281B390BA20EB31EECCFC20116CFCF932C
:1017F000DF931F92CDB7DEB741E050E0BE016F5FCF
:101800007F4FF1DE019731F4898190E00F90DF91F5
:10181000CF9108958FEF9FEFF9CFFC01818D928DCD
:10182000009709F0E4CF8FEF9FEF08950F931F9378
:10183000CF93DF93EC01898D9A8D10E000E0009743
:1018400089F0D5DF8C010F3F100761F0898D9A8DEB
:10185000FC014285538564857585415051096109B4
:10186000710937DDC801DF91CF911F910F91089564
:10187000CF93DF93EC018D81882319F18C8187FF51
:101880001DC0CE015CDAFC01892BD9F08D8182303C
:1018900040F48B899C89AD89BE89848F958FA68FF2
:1018A000B78F8F89988D938F828F8F89988DA98D0F
:1018B000BA8DB58BA48B8C818F778C83DF91CF9180
:1018C000BCC980E0DF91CF9108958F929F92AF9233
:1018D000BF92CF92DF92EF92FF920F931F93CF931D
:1018E000DF9300D01F92CDB7DEB7FC018581813038
:1018F00091F080E00F900F900F900F90DF91CF91BB
:101900001F910F91FF90EF90DF90CF90BF90AF901D
:101910009F908F900895848181FFEBCF8389948974
:10192000A589B689892B8A2B8B2B09F459C07F0195
:1019300040E050E0BA01CF01CCDC8823D1F2F701BE
:10194000C38CD48C8788908CA18CB28C82E090E080
:10195000A0E0B0E0F60180839183A283B3839E016F
:101960002F5F3F4FB501A401C601C9DB882309F4ED
:10197000C0CF00E010E09801B501A401C6011EDB54
:10198000882309F4B6CF89809A80AB80BC80F601A9
:101990008789803101F188EF9FEFAFEFBFE08816B4
:1019A0009906AA06BB06D8F2F701178A108E118E87
:1019B000128E138A148A158A168A84818068848319
:1019C000C70156DF882309F494CF40E050E0BA0104
:1019D000C7017FDC8FCF88EF9FEFA0E0B0E0DFCFC3
:1019E00081E088CFCF92DF92EF92FF921F93CF9347
:1019F000DF93EC0180E2689FF0011124E051FA4E80
:101A00009385917161F0842F827449F080E0DF91B9
:101A1000CF911F91FF90EF90DF90CF900895142FFA
:101A20006A8B8091940290919502A0919602B09158
:101A300097028E879F87A88BB98BC488D588F12C95
:101A4000E12C7601DD24CC24CF8AD88EE98EFA8E63
:101A5000828D938DB0E0A0E0AC01BD014C295D29E1
:101A60006E297F294F8B588F698F7A8F8385887174
:101A7000B1F4848D958DA68DB78D8B8B9C8BAD8BA2
:101A8000BE8B81E08D831F701C831E821F8218868F
:101A900019861A861B861C861D8681E0B8CF803188
:101AA00009F0B4CF9E012D5E3F4F8B8D9C8DA7DB3F
:101AB000882309F4ABCF84E0E5CFCF93DF93EC012B
:101AC000D7DE882311F01D8281E0DF91CF91089548
:101AD000FC01818D928D009709F0CACE08953F9246
:101AE0004F925F926F927F928F929F92AF92BF922E
:101AF000CF92DF92EF92FF920F931F93CF93DF93DA
:101B000000D000D000D01F921F92CDB7DEB77C016D
:101B1000DC0115968C91811115C0FE013196CE0124
:101B20000C966F0130E23193E817F907E1F7DA011B
:101B300030E087E09D91B92E992329F19E3239F446
:101B40008A3011F480E0D6C038E08AE0F3CFE3E6D3
:101B5000F9E04491442321F031969413FACFF2CF67
:101B6000831780F34FED490F4E3560F74FE9490F6A
:101B70004A3118F440EEB42EB90EF601E30FF11D10
:101B8000B0823F5FD7CF89818032E1F2322E8B0164
:101B9000FB01838D948DD7015C969C938E935B970C
:101BA0001682178210861186128613861486158671
:101BB000F80182859385A485B58543895489658913
:101BC000768984179507A607B70708F04CC025E06B
:101BD000B695A795979587952A95D1F7F82FFF7019
:101BE000AF2ED80115968C91823008F4ABCFC80186
:101BF000FEDD97FDA7CFF80182859385A485B58585
:101C00004F96A11DB11D82879387A487B587F0E207
